:020000040002F8
:1070000028A60020C5730200CD730200CF730200D2
:10701000D1730200D3730200D57302000000000098
:10702000000000000000000000000000D773020014
:10703000D973020000000000DB730200DD73020060
:10704000A18C0200DF7302000D9B02009D930200E1
:10705000B1930200DF730200E18B02004591020050
:10706000DD9A0200F59A0200DF730200DF7302006E
:10707000DF730200DF730200DF730200DF730200C0
:107080001D9B0200FD8C0200DF730200DF73020013
:10709000DF730200DF730200D9930200DF73020086
:1070A000DF730200DF730200DF730200DF73020090
:1070B000E98C0200DF730200000000000000000005
:1070C000DF730200DF730200DF730200C59302006A
:1070D000158D0200DF730200DF730200DF73020010
:1070E000DF7302000000000000000000000000004C
:1070F00000000000DF73020000000000DF730200E8
:10710000000000000000000000000000000000007F
:10711000000000000000000000000000000000006F
:10712000000000000000000000000000000000005F
:10713000000000000000000000000000000000004F
:10714000000000000000000000000000000000003F
:10715000000000000000000000000000000000002F
:10716000000000000000000000000000000000001F
:10717000000000000000000000000000000000000F
:1071800000000000000000000000000000000000FF
:1071900000000000000000000000000000000000EF
:1071A00000000000000000000000000000000000DF
:1071B00000000000000000000000000000000000CF
:1071C00000000000000000000000000000000000BF
:1071D00000000000000000000000000000000000AF
:1071E000000000000000000000000000000000009F
:1071F000000000000000000000000000000000008F
:10720000DFF810D000F0A6FC0048004781F1020032
:10721000AFF3008028A6002030B450E8012F93B2CD
:10722000C48923448489A34228BF1B1B0489A34229
:1072300002BFBFF32F8F002007E0C3EA020340E83C
:107240000134002CE9D14FF001000A6030BC7047D6
:1072500050E8012FC2EA024240E801210029F7D19B
:10726000704730B450E8022F1FFAA2F3C488A3423B
:1072700002BFBFF32F8F00200DE0C489234484890F
:10728000A34228BF1B1BC2EA034340E80234002C80
:10729000E8D14FF001000A6030BC704750E8022F7F
:1072A000C2EA224240E802210029F7D17047034692
:1072B00053E8022FD988B2EB324F4FF0000017BFCE
:1072C00092B241EA014142EA014104E05A68B2EB5C
:1072D000324F08BF012043E80212002AE8D170476C
:1072E00030B4044654E8000F0D4644E80053002B28
:1072F000F8D1156030BC704730B4044654E8000F34
:1073000040EA010544E80053002BF7D1156030BC7A
:10731000704730B4044654E8000F00EA010544E821
:107320000053002BF7D1156030BC704730B40446D1
:1073300054E8000F80EA010544E80053002BF7D120
:10734000156030BC704730B4044654E8000F00EBC1
:10735000010544E80053002BF7D1156030BC70479D
:1073600030B4044654E8000FA0EB010544E8005394
:10737000002BF7D1156030BC704770B404464FF055
:10738000000054E8006F0D68AE4207BF44E80023D8
:10739000012044E800630E60002B1CBF0020F0E7D2
:1073A00070BC704730B4044654E8000F88422CBFCC
:1073B000451A054644E80053002BF5D1156030BC52
:1073C000704700000648804706480047FEE7FEE792
:1073D000FEE7FEE7FEE7FEE7FEE7FEE7FEE7FEE785
:1073E0002199020001720200202A04DB203A00FAEF
:1073F00002F1002070479140C2F1200320FA03F30C
:10740000194390407047202A04DB203A21FA02F009
:107410000021704721FA02F3D040C2F120029140CE
:10742000084319467047000000487047C4700300C5
:1074300010B50446FFF7F8FF0068005D00F001009A
:1074400010BD000038B5D0E90221491E01EB410111
:1074500002EBC1014268C1EB011102EB810102683C
:10746000C1EB011102EB8102D0E9043101EB4101D2
:1074700003EB81013023A1F5527191FBF3F4174D19
:107480006C4302EBC41291FBF3F403FB1411009262
:107490001A2902DB124B1A4400920C2291FBF2F3E0
:1074A000104C6343009C04EBC313009391FBF2F375
:1074B00002FB13110C4A08E0491E40F2A324535C5E
:1074C0006343009C04EBC31300930029F4DC0146E2
:1074D000684600F023FA009838BD00003F0C0F000A
:1074E0008051010067C20300C870030040EA010335
:1074F0009B0703D009E008C9121F08C0042AFAD26A
:1075000003E011F8013B00F8013B521EF9D270472D
:10751000D2B201E000F8012B491EFBD270470022D5
:10752000F6E710B513460A4604461946FFF7F0FF82
:10753000204610BD421C10F8011B0029FBD1801A07
:10754000704730B504460020034600E05B1C9342C0
:1075500003D2E05CCD5C401BF8D030BD034611F88F
:10756000012B00F8012B002AF9D1184670470000C2
:107570000FB400B58DB010A909900B9000914FF099
:10758000FF300A9000200C900548069005480790AF
:107590006A4609A80F9900F01BFA0DB05DF814FBBC
:1075A000ED7902000B7A02002DE9FF5F1D464FF0D6
:1075B000FF3BD5E9014691465F464FF00008A969B7
:1075C0007F1C01988847296A824688470028F6D19F
:1075D000BAF1FF3F0CD024F4C064002E19DD600620
:1075E00014D5BAF12B0F09D0BAF12D0F0ED103E04B
:1075F000584604B0BDE8F09F44F48064A9697F1C3C
:1076000001988847761E8246002E02DDBAF1300FBF
:1076100003D0B9F1000F26D032E0A969761E44F4F8
:1076200000747F1C019888478246002E05DDBAF160
:10763000780F06D0BAF1580F03D0B9F1000F10D06F
:107640001EE0B9F1000F02D0B9F1100F18D1A969ED
:10765000761E24F400747F1C01988847824610200F
:1076600002E0082000E00A20814609E008FB090842
:10767000A969761E44F400747F1C019888478246ED
:10768000002E05DD4946504600F08EF90028EDDA5F
:10769000E96901988847A00502D46FF00100A8E7C6
:1076A000E00725D1600613D5600502D5C8F10000BA
:1076B00000E0404629680A1D2A600968220501D5B4
:1076C000087015E0220701D5088011E008600FE07E
:1076D0002868011D29600068210502D580F8008016
:1076E00006E0210702D5A0F8008001E0C0F8008084
:1076F00038467EE72DE9FE4F81EA030404F000449A
:1077000021F0004100944FF0000B23F0004350EAB9
:1077100001045ED052EA03045BD0C3F30A54C1F300
:107720000A552C44A4F2F3340194A0FB0254C1F393
:10773000130141F48011C3F3130343F4801301FBDD
:10774000024400FB034E840A970A44EA815447EA44
:107750008357A4FB076802958D0A05FB07854FEA4E
:10776000932C04FB0C542705029D4FEA065847EA68
:107770001637B5EB08056EEB070C870E920E47EA3D
:10778000811742EA8312A7FB0201B6EB0B0164EBFF
:1077900000042B0D43EA0C335E1844EB1C50DA4610
:1077A0005146E7FB0201C5F313044FEA0B3343EAEA
:1077B00014534FEA0432019C43EA0603A4F10C047B
:1077C0000294009CCDE900B400F076F903B0BDE866
:1077D000F08F00200146F9E72DE9F04D81EA03041E
:1077E00004F0004B21F0004514464FF0000A23F04E
:1077F000004150EA050220D054EA01021DD0C5F331
:107800000A570246C5F31303C1F31300C1F30A5626
:1078100040F4801543F48013A7EB0608101BD646EE
:1078200008F2FD3873EB050002D308F1010801E00E
:1078300092185B41B8F1000F03DA00200146BDE861
:10784000F08D00204FF48011064684460EE0171B91
:1078500073EB050705D3121B63EB050306434CEAE4
:10786000010C49084FEA300092185B4150EA0107C9
:10787000EDD152EA030012D082EA040083EA050146
:10788000084305D0101BAB4106D20122002306E0BD
:1078900000224FF0004302E06FF0010253101AEB98
:1078A00006004CEB085110EB0A0041EB0B01BDE860
:1078B000F04D00F0F2B80EB5C10F80EAE070084458
:1078C000CA07002140F233438DE80E000A460B46FA
:1078D00000F0F2F803B000BD01F0004330B421F035
:1078E000004150EA010206D00A0DA2F56072C1F310
:1078F0001301002A02DC30BC00207047440F44EA28
:10790000C104C100E01830BC00EBC25000F08EB8DA
:10791000014900F003B80000F895002010B5006898
:107920003C22B0FBF2F302FB1303B0FBF2F00B605E
:10793000B0FBF2F302FB1303B0FBF2F018224B6032
:10794000B0FBF2F302FB1303B0FBF2F0021D8B60FD
:107950000723B2FBF3F403FB1422800040F2B5537B
:1079600000F66C308A61B0FBF3F2B0FBF3F403FB7A
:107970001400443280084A61C8613B2802D3920750
:1079800000D0401C0022074C13460A61E25C824290
:1079900003D8801A5B1C0B61F8E7401CC8600846DE
:1079A00010BD0000D47003003A2800D2303820F017
:1079B0002002412A01D3A2F13700884201D34FF0BF
:1079C000FF30704702681144137801601846704711
:1079D000D1600449516104491162002111611146CD
:1079E00000F0CAB8C579020031740200426842B1A1
:1079F000016811F8013B23B1521EC0E9001218467C
:107A000070470121C160881E704742685AB1C3683F
:107A1000016843B983688B4205D0491E521CC0E9F6
:107A20000012002070474FF0FF3070470029A8BFB8
:107A30007047401C490008BF20F00100704710B497
:107A4000B0FA80FC00FA0CF050EA010404BF10BC4C
:107A5000704749B1CCF1200421FA04F411FA0CF179
:107A600018BF012121430843A3EB0C01CB1D4FEAB2
:107A700000614FEA102042BF002010BC704700EBAD
:107A8000C35010440029A4BF10BC7047401C4900DB
:107A900008BF20F0010010BC704710B5141E73F130
:107AA000000408DA401C41F1000192185B411A43BE
:107AB00001D120F0010010BD2DE9F04D92469B460A
:107AC00011B1B1FA81F202E0B0FA80F220329046B0
:107AD000FFF78AFC04460F4640EA0A0041EA0B0120
:107AE00053465A46084313D0114653EA010019D0B1
:107AF000C8F140025046FFF786FC05460E46504648
:107B000059464246FFF770FC084305D0012004E0C7
:107B100020463946BDE8F08D0020054346EAE07670
:107B20002C4337430A986305E40AA0EB08000022BF
:107B3000FD0A44EA47540A3002D500200146E9E72D
:107B4000010510196941DDE9084500196941BDE8E1
:107B5000F04DA2E7064C074D06E0E06840F0010357
:107B600094E8070098471034AC42F6D3FFF74CFB7B
:107B70009C7C0300BC7C03002DE9F34F8BB04FF0DD
:107B8000000801F10C000C464FF0010B46460DF1C8
:107B9000080A01906269012101989047051E2DD0C5
:107BA000252D2CD0216A8847C0B162690121019836
:107BB0009047216A88470028F7D1411E62690198E1
:107BC000904700E0761CA1690B988847216A884796
:107BD0000028F7D1E1690B988847DBE7A1690B988A
:107BE00088470746A84201D1761CD3E7E1690B9884
:107BF00088477F1C02D1B8F1000F6FD047E1002702
:107C000062693D463946019890472A2804D1626945
:107C10000121019890470125DFF8889262690121CE
:107C200001989047A0F130010A290AD24F45E5DCBE
:107C300007EB870100EB4107303FDFD445F010052B
:107C4000ECE7E90601D46FF000476C280AD04C2815
:107C500014D0682815D06A280DD074281CD07A2832
:107C60001AD01DE062690121019890476C2802D06A
:107C700045F0040514E045F002050DE045F020054F
:107C80000AE06269012101989047682802D045F016
:107C9000080505E045F400656269012101989047F7
:107CA000C4E9015765283DD019DC58287AD00CDC8E
:107CB000452837D004DC252826D0412831D131E0B1
:107CC00046282FD047282CD12CE05B2877D061287C
:107CD00028D063287CD0642823D15AE0D1E06F28D3
:107CE00048D008DC66281DD067281BD0692821D021
:107CF0006E2816D127E0702845D0732868D07528E3
:107D000047D078280DD14DE0A1690B9888470546EA
:107D100025283FF469AFE1690B9888476D1C3FF453
:107D20006AAFB4E023466A466FF001000B99AFF3E7
:107D300000809FE045F040006060A80723464FF0B8
:107D4000000236D43EE0E8077FF447AF2068011D0B
:107D500021600068290501D506701BE7290701D5B8
:107D6000068017E7A90703D5F117C0E9006111E7FD
:107D700006600FE745F040006060A80723464FF01B
:107D8000080216D41EE040F60E0125EA01006060EC
:107D900016E045F040006060A80723464FF00A0255
:107DA00007D40FE045F040006060A80708D52346DF
:107DB00010226FF001000B99AFF300805AE007E04A
:107DC000234610226FF001000B99FFF7EDFB51E005
:107DD0004FF000094F464B46632802D05B2807D07E
:107DE00041E02079C00601D40120A06001273AE0DB
:107DF00062690121019890475E2805D14FF0010981
:107E00006269494601989047216939B900210A46BB
:107E1000534643F82120491C0829FADBB0B32169F5
:107E200069B9C11700EBD16253110AEB830122F04B
:107E30001F02821A01200B68904003430B606269A5
:107E40000121019890475D28E8D1B9F1000F09D0D0
:107E50000020514651F82020D24341F82020401CF8
:107E60000828F7DB02AB224600976FF001000B9960
:107E7000AFF3008000280CDA401C08D1BBF1000FE2
:107E800005D04FF0FF300DB0BDE8F08FFFE7404662
:107E9000F9E7E90701D108F1010806444FF0000BAA
:107EA00078E60000CCCCCC0C70B58C1810F8015BD7
:107EB00015F0070301D110F8013B2A1106D110F883
:107EC000012B03E010F8016B01F8016B5B1EF9D187
:107ED0002B0705D40023521E0DD401F8013BFAE70D
:107EE00010F8013BCB1A921C03E013F8015B01F878
:107EF000015B521EF9D5A142D8D3002070BD00000D
:107F00002CB5294800F00CF928480078002847D102
:107F100000BF274A0121274802F0F4FF0546D5B1EA
:107F200025482649264A891AC9080322CDE90005B1
:107F300042EA014040F2152322A228A108F0F4FCF5
:107F400008F0ACFA00BF00BF24B100BF204602F029
:107F5000E1FB00BF00BF00BF00BF284A0021284846
:107F600002F0D0FF0546D5B126481449144A891AB3
:107F7000C9080322CDE9000542EA014040F2162378
:107F800010A216A108F0D0FC08F088FA00BF00BFCC
:107F900024B100BF204602F0BDFB00BF00BF00BF00
:107FA0000120024908702CBD31A70200152C0020C9
:107FB000C18E0200306B0300E0700300647D03009B
:107FC000CC7C03007372635C6170705F626C655F90
:107FD000736572766963652E6300000025733A2528
:107FE00064205A4552524F525F434845434B28251F
:107FF0007329206661696C3A25640000458D020092
:10800000346B0300387103002CB51A491A4A891AD7
:10801000C908032242EA014018A108F04BFC1E489F
:10802000002101601D481C49086000BF1C480EF07B
:10803000FFFA0546002D1AD01AA00E490E4A891AD9
:10804000C9080322CDE9000542EA014040F2F313DA
:1080500020A226A108F068FC08F020FA00BF00BFAB
:1080600024B100BF204602F055FB00BF00BF00BF97
:108070002CBD0000647D0300CC7C0300696E697434
:10808000207A646174616368616E6E656C207365EB
:108090007276696365000000282C00208565030066
:1080A000A44D00207A646174616368616E6E656CD2
:1080B0005F696E697428266D5F7A6872732C20265A
:1080C0007A646174616368616E6E6C655F696E6924
:1080D000742900007372635C6170705F626C655F2D
:1080E000736572766963652E6300000025733A2517
:1080F00064205A4552524F525F434845434B28250E
:108100007329206661696C3A2564000010B5044645
:10811000024A3821204602F063FC10BDADA90200DE
:1081200004490A680968491C024B1960024941F870
:1081300022007047C02D00208869002010B5012062
:108140000EF09AFC0446204610BD000070B52DEDDF
:108150000C8BFFF7F3FF0546FFF7ADFB41EC1D0B62
:108160009FED2F0B53EC102BFFF736FB41EC1C0B54
:108170009FED2D0B53EC102BFFF7BCFA41EC1B0BC2
:108180009FED2B0B53EC102BFFF726FB41EC1A0B4A
:108190009FED290B53EC102BFFF7ACFA41EC190BB8
:1081A000FFF79AFB08EE100AB1EE000AB4EEC08A9F
:1081B000F1EE10FA03DDB1EE000AB0EE408A9FED59
:1081C000200AB4EEC08AF1EE10FA03D29FED1C0A29
:1081D000B0EE408A9FED1A0A38EE400A9FED191A58
:1081E000C0EE010A9FED181A9FED180AF0EE408AC2
:1081F00040EE818ABDEEE80A10EE100A04B20A2CA5
:1082000002DA0CB1032406E00A2094FBF0F000EB44
:108210008000400004B22046BDEC0C8B70BD000015
:10822000000000000000B0406666666666660A40B0
:1082300000000000000000400000000000000840B6
:10824000333353403433333F0000C842CDCCCC3DB0
:108250007047000070B586B02D4800680590022078
:108260008DF8140000BF05AD002605B9294D314633
:10827000284609F0A1FC044600BF002C19D026A016
:108280002E492F4A891AC9080322CDE9000442EA7F
:10829000014008232BA233A108F046FB08F0FEF8AA
:1082A00000BF00BF25B100BF284602F033FA00BF6F
:1082B00000BF00BF164A121D07CA02AB07C3042045
:1082C0008DF80C0000BF02A9012009F01FFC054633
:1082D000002D19D02BA01949194A891AC90803225F
:1082E000CDE9000542EA01400C2316A21DA108F0C9
:1082F0001BFB08F0D3F800BF00BF24B100BF20462D
:1083000002F008FA00BF00BF00BF06B070BD000059
:10831000606B03005C6B03006E72665F6472765F75
:1083200073616164635F696E697428266164636365
:1083300066672C204E554C4C29000000647D0300DC
:10834000CC7C03007372635C626F6172645C626F09
:108350006172645F626174746572795F7374617471
:10836000652E630025733A2564205A4552524F52B8
:108370005F434845434B28257329206661696C3A61
:10838000256400006E7266785F73616164635F6389
:1083900068616E6E656C5F696E6974284241545401
:1083A0004552595F4144435F4348414E4E454C2C32
:1083B00020266368616E6E656C5F636F6E666967C9
:1083C0002900000010B5034A0121034802F09AFD7C
:1083D00010BD000021B10200706B030010B500BF9A
:1083E00000220649064809F001FA044624B100BFFC
:1083F000204602F08FF900BF00BF10BD846B030060
:10840000E82D002010B504466CB10949088900EB3D
:10841000D0714910074A11800223012206490748FA
:1084200009F086FA03E00121044809F0C3FA10BDFF
:10843000846B0300F02D0020746B0300E82D0020F6
:1084400010B504460B4804700B48006802F0D3FDD9
:1084500000200A4908600748007818B90020FFF793
:10846000D1FF06E0002240F69A110348006802F0AE
:1084700093FD10BDF82D0020706B0300FC2D002033
:108480000149086070470000002E0020704700007E
:108490002CB5002109200EF025FB00BF114A012157
:1084A000114802F02FFD0546CDB110481049114A80
:1084B000891AC9080322CDE9000542EA01402B23AD
:1084C0000DA215A108F030FA07F0E8FF00BF00BFC9
:1084D00024B100BF204602F01DF900BF00BF00BF5D
:1084E0002CBD000039850200906B0300DC72030094
:1084F000647D0300CC7C03007372635C626F617205
:10850000645C626F6172645F6C696768745F6374F6
:10851000726C2E630000000025733A2564205A45D2
:1085200052524F525F434845434B282573292066DA
:1085300061696C3A2564000010B504462348007850
:1085400030B92348007808B3002000F071F836E015
:108550001E480078012806D11D480078B0B90120D6
:1085600000F066F82BE019480078022827D1194856
:108570000068022818DA1749086800EBD071491022
:10858000A0EB410119B9012000F052F817E01149A0
:10859000086800EBD0714910A0EB410101290ED110
:1085A000002000F045F80AE00A48006864214843CA
:1085B000B0F57A7F03DB00200649086010BD05484E
:1085C0000068401C0349086000BFF7E7102E002038
:1085D000112E0020142E00207047000010B5044614
:1085E0001148047024B1012C0AD0022C18D10FE0DC
:1085F0000E48006802F0FFFC002000F019F810E0BF
:108600000A48006802F0F7FC012000F011F808E0C9
:10861000002240F266610548006802F0BDFC00E0FF
:1086200000BF00BF10BD0000102E0020906B0300A3
:1086300038B504468CB109200090684607F07EFDED
:1086400005460121009A01FA02F0C5F8080500BFAD
:1086500000BF01200A49087010E009200090684618
:1086600007F06CFD05460121009A01FA02F0C5F8F9
:108670000C0500BF00BF00200149087038BD000094
:10868000112E002010B520480078022800D110BD1E
:1086900001221EA1002005F0EBFA002004F08AFF61
:1086A00000221146052007F0CAFC002211460B20CB
:1086B00007F0C5FC00221146112007F0C0FC002283
:1086C0001146042007F0BBFC01211E2007F0BDFD70
:1086D000642007F0BFF900211E2007F0B6FD00213D
:1086E000012007F0B2FD00211C2007F0AEFD1E2086
:1086F00007F0B0F901211C2007F0A7FD0220024974
:10870000087000BFC3E70000382E00200000000002
:108710002DE9F84357480078012801D1BDE8F883D6
:1087200001211E2007F091FD0121084607F08DFD73
:108730001E2007F08FF900211E2007F086FD01247E
:108740004FF00A0805E0002004F0D0FD0446A8F12F
:108750000108B8F1000F01D0002CF4D1002C25D075
:108760004549464A891AC908032242EA014022467D
:1087700043A108F0A9F800BF49A03F493F4A891A20
:10878000C9080322009042EA01409A2345A24DA164
:1087900008F0B6F807F082FE00BF4FF0000800BFF7
:1087A000002001F0B7FF00BF00BF00BF3249334ACD
:1087B000891AC908032242EA014048A108F07AF860
:1087C00001224EA14E4805F053FA0546002D24D053
:1087D00029492A4A891AC908032242EA014049A1C3
:1087E00008F068F800BF2EA02349244A891AC90856
:1087F0000322009042EA0140A1232AA231A108F0FD
:108800007FF807F04BFE00BF4FF0000800BF0020CC
:1088100001F080FF00BF00BF00BF3E480068416913
:108820003C48884740684FF48011B1FBF0F6394866
:1088300000684169374888470068B0FBF6F70E4981
:108840000E4A891AC908032242EA014032A108F0FF
:1088500031F80949094A891AC908032242EA014044
:108860003A4631A108F030F801200249087000BFF3
:1088700054E70000382E0020647D0300CC7C030008
:108880004469736B20696E697469616C697A61749B
:10889000696F6E206661696C65642E202564000036
:1088A000300000007372635C626F6172645C626FBF
:1088B0006172645F7364636172645F647269766538
:1088C000722E630025733A2564205A415353455252
:1088D0005428257329206661696C00004469736B14
:1088E00020696E697469616C697A6174696F6E2060
:1088F0007375636365656465642E000000000000A5
:10890000B06900204D6F756E74206661696C656496
:108910002E000000A06B03004D6F756E7420737500
:108920006363657373000000436170616369747908
:108930003A202564204D420001480078704700002D
:10894000382E002010B51E48007800B110BD00225E
:108950001146052007F073FB002211460B2007F09B
:108960006EFB00221146112007F069FB0022114620
:10897000042007F064FB03211C200EF0B3F8012152
:108980001C2007F062FC032101200EF0ABF800214F
:10899000012007F05AFC03211E200EF0A3F800214D
:1089A0001E2007F052FC00200649087001210648ED
:1089B00004F0EAFE01200249087000BFC6E700008B
:1089C000392E0020382E00203C2E002070B50446A1
:1089D000204605F07FF805460B48007805F07AF848
:1089E00006460A490A4A891AC908032242EA01408E
:1089F0002B46324607A107F073FF034804700DF0C1
:108A000045FF0B49086070BDA82D0020647D030060
:108A1000CC7C03006368616E676520737461746564
:108A20002066726F6D20257320746F2025730000FF
:108A3000AC2D00202CB5FFF7C5FCFFF729FD2E4813
:108A4000FFF71EFDFFF704FC00F0E0FD06F008F85C
:108A50002A48FFF765FB2A480DF014FD0AF056FA84
:108A600000BF284A0121284802F04CFA0546D5B13A
:108A700026482749274A891AC9080322CDE9000553
:108A800042EA01404FF4907323A22AA107F04CFF61
:108A900007F004FD00BF00BF24B100BF204601F075
:108AA00039FE00BF00BF00BF00BF002240F2666178
:108AB0001548006802F070FA0546D5B125481449FA
:108AC000144A891AC9080322CDE9000542EA014087
:108AD00040F2211310A217A107F026FF07F0DEFCD9
:108AE00000BF00BF24B100BF204601F013FE00BF4D
:108AF00000BF00BF2CBD000061C402008DA70200B2
:108B00001161030035540300586B030078720300B1
:108B1000647D0300CC7C03007372635C64657669DA
:108B200063655F6374726C5F736572766963652EEB
:108B30006300000025733A2564205A4552524F5273
:108B40005F434845434B28257329206661696C3A89
:108B5000256400003072030001480078704700006F
:108B6000A82D002010B50849084A891AC90803220F
:108B700042EA014006A107F09DFE06200849087060
:108B80000846FFF7C3FA10BD647D0300CC7C0300E8
:108B900073746172742073616D706C650000000005
:108BA0001869002010B50849084A891AC908032223
:108BB00042EA014006A107F07DFE07200749087040
:108BC0000846FFF7A3FA10BD647D0300CC7C0300C8
:108BD00073746F702073616D706C65005069002054
:108BE0002DE9FC4700260020009001904FF480778B
:108BF0000125002410E0384607F05CFB40B100BFBF
:108C000025480068284018B1384607F045FB2E4338
:108C10006D00381D87B2641C082CECD34FF4BE7075
:108C200007F048FB50B14FF4BE7007F035FB46F03B
:108C300000466A460221002007F03CFAF0B210B369
:108C4000012500241DE005EA0600C0B100BF13485D
:108C500050F82400C0F30520814600BF0F4850F8AB
:108C60002400C0F301408246204603F0EBFC80461E
:108C7000B8F1000F02D051464846C04700BF6D0012
:108C8000641C082CDFD306F0004010B168460AF0DF
:108C900001F8BDE8FC870000046300401065004057
:108CA00010B54FF4807006F0B9FE50B14FF48070EB
:108CB00006F0BDFE012006F0C3FE0A480168002050
:108CC00088474FF4827006F0A9FE50B14FF48270CD
:108CD00006F0ADFE022006F0B3FE02480168012056
:108CE000884710BD582E002010B50249024806F0F2
:108CF00075F810BD682E002000C0014010B5034A71
:108D00001068034A1168884710BD0000B82E002083
:108D1000B42E002010B504220021024806F0B0F85D
:108D200010BD00000040024010B50020034908704B
:108D30000348006802F05FF9002010BD142C0020E9
:108D4000306B030010B504460248006800F00AF8D2
:108D500010BD0000102C0020014800787047000072
:108D6000142C002070B50546074C07266A20A07019
:108D70000020607003202070C4F803503146204664
:108D80000DF04EFC70BD0000A44B00207CB50646E3
:108D900000F048FB0021304600F042FC1B4908600F
:108DA00008460068002801DC07207CBD00BF0022C7
:108DB00021211748006802F0EFF80546002D19D070
:108DC00014A02449244A891AC9080322CDE90005C0
:108DD00042EA0140FC2321A226A107F0A5FD07F0ED
:108DE0005DFB00BF00BF24B100BF204601F092FC34
:108DF00000BF00BF00BF012026490870002026499F
:108E000008602649086000BFCFE70000082C00205A
:108E1000306B03006170705F74696D65725F7374AD
:108E2000617274286D5F7265636F72645F75706CD8
:108E30006F61645F746D722C204150505F54494DD6
:108E400045525F5449434B532832292C204E554CF0
:108E50004C290000647D0300CC7C03007372635CCA
:108E60006170705F626C655F736572766963652EB1
:108E70006300000025733A2564205A4552524F5230
:108E80005F434845434B28257329206661696C3A46
:108E900025640000142C00200C2C0020102C002035
:108EA00010B500200449087000F09AFA03480068E1
:108EB00002F0A1F8002010BD142C0020306B03003C
:108EC0002DE9FC4E81466548007808B9BDE8FC8E66
:108ED0006348006800284AD14FF480716148FEF76A
:108EE0001EFB4FF480725F495F48006800F006FC8B
:108EF0008246BAF1000F36DC5C495D4A891AC9081E
:108F0000032242EA01405BA107F0D4FC00BF6048A5
:108F10004FF4F67102685F48006802F03DF883463E
:108F2000BBF1000F1BD05C485049514A891AC9084F
:108F30000322CDE9000B42EA0140C42357A25DA100
:108F400007F0F2FC07F0AAFA00BF00BFB8F1000F6B
:108F500004D000BF404601F0DDFB00BF00BF00BFF2
:108F6000FFF7E2FEB2E73E48C0F800A000BF3C4871
:108F7000006800B9AAE70DF0E3F80546802D01DA94
:108F8000284600E08020054635480068C0F580701E
:108F90003449461832480068A84201DD284601E0FD
:108FA0002F48006807463149314A891AC908032207
:108FB00042EA01402A4900953A460B6845A107F06C
:108FC0009FFC0DF0F9FB60B92849294A891AC908A4
:108FD000032242EA014043A107F06CFCFFF7A4FE24
:108FE00074E7B8B2019001A930460DF0A3FA044627
:108FF00000BF0CB3082C0CD11C491D4A891AC908A2
:10900000032242EA01403FA107F054FCFFF78CFE27
:109010005CE7112C01D0132C00D157E71349144AF7
:10902000891AC908032242EA014022463DA107F0FD
:109030004BFCFFF779FE49E7002006E0315C144A5B
:1090400012681144124A1160401CB842F6D3044819
:109050000068C01B0249086000BF37E7142C0020DD
:109060000C2C0020C84D0020082C0020647D03003B
:10907000CC7C0300726561642066696C6520656E56
:10908000642C73746F702075706C6F6164000000E5
:10909000102C0020346B0300BC7103007372635CFE
:1090A0006170705F626C655F736572766963652E6F
:1090B0006300000025733A2564205A4552524F52EE
:1090C0005F434845434B28257329206661696C3A04
:1090D0002564000075706C6F616420256420256430
:1090E00020256400626C6520697320646973636F76
:1090F0006E6E65637465642C73746F702075706C2C
:109100006F616400626C6520756E656E61626C658E
:10911000206E6F746966792C73746F702075706C33
:109120006F616400626C652073656E6420657272A5
:109130006F722C73746F702075706C6F6164202572
:1091400078000000FEB54FF4827007F0EFFE0028B3
:1091500037D04FF4827007F0F3FE6C4890F82E0081
:1091600018B16A4890F82F0058B300208DF800001D
:1091700066484068019065480189ADF80810C068EC
:1091800018B900206149087412E06048008B5F49FB
:1091900048830846C06848600846008B0881002064
:1091A000C860084690F82E0010B9002007F0E0FED5
:1091B00056480168684688470020544981F82F00C6
:1091C00000BF524890F82E00002852D04FF4807013
:1091D00007F0ACFE00284CD04FF4807007F0B0FED2
:1091E0004A48408B494991F82D10884216DD47487E
:1091F000408B464991F82D10401A444948830A464D
:1092000012890B465B8BD21A0B465B6803EB42005C
:109210000A4692F82D1007F075FE23E03B48408B7C
:109220003A4991F82D1088420FD13848C06860B192
:109230000120364981F82F00002048830A4692F821
:109240002D10D06807F05EFE0CE03048408B2F49AF
:1092500091F82D10884205D101202C4981F82F006A
:10926000002048834FF4827007F06AFE042007F064
:109270007FFE4FF4887007F059FE70B14FF488708C
:1092800007F05EFE00202149087402208DF80000DE
:10929000084601686846884700BF4FF48A7007F0A7
:1092A00045FE38B14FF48A7007F04AFE0020174996
:1092B00008742AE01548456924E0B5FA85F64FF0B0
:1092C0000040F0408543B00000F58C74204607F064
:1092D0002DFEB8B1204607F033FE01208DF80000C6
:1092E000A4F58C70C0F3C7008DF80400A4F58C7051
:1092F000012121EA90018DF80510044801686846B3
:10930000884700BF002DD8D100BFFEBD506D0020A2
:1093100010B500F023FC10BD2DE9F0470746884644
:109320001646C24607EB47011B4800EBC109D9F8B6
:10933000140020B1012811D0022826D11EE0484691
:1093400000F044FC0546B54201D2002405E0344655
:1093500032465146484600F080FC18E0484600F08E
:1093600035FC0546B54201D2284600E030460446A9
:1093700022465146484600F070FC08E0324651460D
:10938000484600F031FC044601E0002400BF00BF65
:109390002046BDE8F0870000C08C002010B50249CF
:1093A000024805F009FD10BD806D0020003000402E
:1093B00010B503494FF040200CF0C0FA10BD00007A
:1093C000E86D002010B50249024805F0F5FC10BD1B
:1093D000A46D00200030024010B507F0CDFF10BD95
:1093E00010B50949094A891AC908032242EA01400D
:1093F00007A107F05FFAFFF79FFA012801D10AF0F1
:1094000019F9FFF73FF910BD647D0300CC7C030020
:109410006368616E676520746F20657874206D6F76
:109420006465000010B50749074A891AC908032274
:1094300042EA014005A107F03DFAFFF769F90AF099
:10944000F9F810BD647D0300CC7C03006368616E95
:10945000676520746F206C6F63616C206D6F64654D
:1094600000000000F8B5064600BF2048007800283C
:1094700017D11FA02149224A891AC9080322009046
:1094800042EA014081231FA227A107F039FA07F021
:1094900005F800BF002500BF002001F03BF900BF28
:1094A00000BF00BF264804F0A9FB044600BF002C03
:1094B00017D024A01149124A891AC9080322009022
:1094C00042EA014083230FA217A107F019FA06F020
:1094D000E5FF00BF002500BF002001F01BF900BF21
:1094E00000BF00BF002001490870F8BD382C0020E3
:1094F0006D5F69735F6F70656E000000647D0300CF
:10950000CC7C03007372635C73616D706C655F6427
:109510006174615F6D616E616765725F73657276BC
:109520006963652E6300000025733A2564205A4163
:10953000535345525428257329206661696C0000F5
:10954000744F002066665F726573756C74203D3DD4
:109550002046525F4F4B00000148406870470000B2
:10956000302C002038B5054600BF10480078002890
:1095700017D10FA01149124A891AC9080322009075
:1095800042EA014096230FA217A107F0B9F906F0AD
:1095900085FF00BF002400BF002001F0BBF800BF22
:1095A00000BF00BF1648C06838BD0000382C00203E
:1095B0006D5F69735F6F70656E000000647D03000E
:1095C000CC7C03007372635C73616D706C655F6467
:1095D0006174615F6D616E616765725F73657276FC
:1095E0006963652E6300000025733A2564205A41A3
:1095F000535345525428257329206661696C000035
:10960000744F002000487047302C002010B5FFF741
:1096100099F9FFF707FFFFF7E3FE10BD7047000061
:10962000F8B507460C46012C25D10B2219A11B4881
:1096300004F04CFB054600BF002D17D018A01D49B3
:109640001D4A891AC9080322009042EA0140742386
:109650001AA223A107F054F906F020FF00BF00264C
:1096600000BF002001F056F800BF00BF00BF01207E
:1096700021490870F8BD012206A1084804F026FB24
:10968000054615B14FF0FF30F4E701201A49087084
:1096900000BFEFE7302E62696E000000744F0020BB
:1096A00066665F726573756C74203D3D2046525F3F
:1096B0004F4B0000647D0300CC7C03007372635C3D
:1096C00073616D706C655F646174615F6D616E6123
:1096D0006765725F736572766963652E630000006B
:1096E00025733A2564205A41535345525428257313
:1096F00029206661696C0000382C00202DE9FC41AE
:1097000080460D46164600BF21480078002817D134
:1097100020A02349234A891AC9080322009042EA5B
:1097200001408F2320A229A107F0EAF806F0B6FE37
:1097300000BF002700BF002000F0ECFF00BF00BF0B
:1097400000BF01AB32462946264804F0B6FB04466A
:1097500000BF002C17D024A01149124A891AC90849
:109760000322009042EA014092230FA217A107F0C2
:10977000C7F806F093FE00BF002700BF002000F0EE
:10978000C9FF00BF00BF00BF0198BDE8FC81000019
:10979000382C00206D5F69735F6F70656E0000008C
:1097A000647D0300CC7C03007372635C73616D7035
:1097B0006C655F646174615F6D616E616765725F46
:1097C000736572766963652E6300000025733A2520
:1097D00064205A4153534552542825732920666109
:1097E000696C0000744F002066665F726573756C6B
:1097F00074203D3D2046525F4F4B000003484068B7
:10980000012801DB012070470020FCE7302C0020FC
:109810002DE9FC4180460D46164600BF21480078E0
:10982000002817D120A02349234A891AC9080322F6
:10983000009042EA0140882320A229A107F060F8A5
:1098400006F02CFE00BF002700BF002000F062FFE2
:1098500000BF00BF00BF01AB32462946264804F0D6
:1098600069FC044600BF002C17D024A01149124AFD
:10987000891AC9080322009042EA01408B230FA2F3
:1098800017A107F03DF806F009FE00BF002700BF52
:10989000002000F03FFF00BF00BF00BF0198BDE8FF
:1098A000FC810000382C00206D5F69735F6F70656C
:1098B0006E000000647D0300CC7C03007372635C67
:1098C00073616D706C655F646174615F6D616E6121
:1098D0006765725F736572766963652E6300000069
:1098E00025733A2564205A41535345525428257311
:1098F00029206661696C0000744F002066665F7203
:109900006573756C74203D3D2046525F4F4B0000DF
:1099100001480249086070470090D003602F002082
:1099200010B505F035FE40B10020644908604FF0E5
:109930008041C1F810016249086005F043FE00282B
:1099400055D060480068604908605E48001D0068A6
:10995000091D08605B4808300068091D0860594807
:109960000C300068091D0860564810300068091D59
:109970000860544814300068091D086051481830C8
:1099800000685149203108604E481C300068091DAC
:1099900008604C4820300068091D086049482430A0
:1099A0000068091D0860474828300068091D0860E4
:1099B00044482C300068091D086042483030006877
:1099C0004149403108603F4834300068091D086053
:1099D0003C4838300068091D08603A483C3000684F
:1099E000091D0860374840300068091D086005F00F
:1099F0009BFD40B13548006800F0010018B16FF0E0
:109A00000100324908603248006840F47000304973
:109A1000086000BF00BF00BFBFF34F8F00BF00BF93
:109A200000BF00BF00BF00BFBFF36F8F00BF00BF0C
:109A300000BF00BF05F092FD20B126480068204914
:109A40002031086000BF2348001D006800F00100BD
:109A500080B3012008F01CFC1E48001D006820F0A7
:109A600001004FF01021C1F80C0208F01BFC00208F
:109A700008F00EFC00BF00BF00BF00BF00BFBFF377
:109A80004F8F00BF00BF00BF11487C38006800F452
:109A9000E06011490843001D0D497C39086000BF92
:109AA00000BF00BFBFF34F8F00BF00BF00BF00BFAC
:109AB00000BFFDE7FFE7FFF72BFF10BD0C010040E3
:109AC000380500400404001020C500400004004098
:109AD00088ED00E0081200100000FA0510B504221D
:109AE0000249034805F028FA10BD0000246E00204A
:109AF0000080004010B504220249034805F01CFA1A
:109B000010BD0000306E00200090004010B50249EA
:109B10000868804710BD0000602E002008B500BF17
:109B20004FF480700B49405808B1012000E000203C
:109B300078B109480068804700BF00204FF4807169
:109B4000044A8850084611464058009000BF00BFA4
:109B500000BF08BD00000140742E002010B5124C5B
:109B600002202061606111A0A0611349E1614FF4FE
:109B7000007121620021A1626162E1620BA0A06418
:109B80000E49E164102121650021A1656165E1654F
:109B90000BA1E01DFDF7E2FC0AA12046FDF7DEFC6B
:109BA0002020A07110BD0000A88C00205465726DAB
:109BB000696E616C00000000208D0020208F002065
:109BC00052545400534547474552000010B50146D2
:109BD0000A69CB689A4204D88C68641EE41AA018FB
:109BE00001E0D41A601E10BD2DE9F04704468946F5
:109BF00017464FF0000AE56800BFD4F81080A8456A
:109C000003D9A8EB0500461E04E0A5EB0800401CA4
:109C1000A1680E1AA068401BB04201D9304601E08D
:109C2000A068401B0646BE4201D2304600E03846DE
:109C300006466168481932464946FDF757FCB2446A
:109C4000B144BF1B3544A068A84200D10025E5609F
:109C5000002FD2D15046BDE8F0872DE9F0470446E9
:109C600089461546E668A068871BAF4208D9616837
:109C700088192A464946FDF739FC7019E06010E062
:109C8000B8466168881942464946FDF72FFCA5EBA6
:109C9000070809EB070142466068FDF727FCC4F896
:109CA0000C80BDE8F08702E008C8121F08C1002A36
:109CB000FAD170477047002001E001C1121F002A4D
:109CC000FBD170470146202908DA012088400A4A62
:109CD000104008B1012070470020FCE7402909DA54
:109CE000A1F12000012202FA00F008B10120F2E700
:109CF0000020F0E70120EEE7FC06FFBD00BFEFF318
:109D00001081084672B670470246002104E0505C9C
:109D100008B101207047491C0629F8D30020F9E753
:109D2000FEB5FF208F49C870142088700F2048703E
:109D300029200870C00788600320087300BF002333
:109D40001A46894805F0AAFF0546002D19D087A0BC
:109D50009249934A891AC9080322CDE9000542EACB
:109D60000140F6238FA297A106F0DEFD06F096FBD8
:109D700000BF00BF24B100BF204600F0CBFC00BFF5
:109D800000BF00BF002103200CF0ACFE00211D200D
:109D90000CF0A8FE032006F031FA1D2006F02EFA82
:109DA00090489149086000204860904890490860B8
:109DB000012048608B498C4800F0F8FA8B498C48A8
:109DC00000F0F4FA01208B4908704021864800F029
:109DD000EFFA06467149724A891AC908032242EA13
:109DE0000140324684A106F06FFD4021804800F01A
:109DF000DFFA064669496A4A891AC908032242EA13
:109E00000140324682A106F05FFD002211467648ED
:109E100000F018FB0020029002AB4122824983A08F
:109E20000BF01AFDBDF80800002837DD5B495C4ADD
:109E3000891AC908032242EA01407EA106F03AFDD0
:109E4000822282497848FDF77CFB50B15349544A3D
:109E5000891AC908032242EA01407DA106F02AFDC1
:109E600009E04E494E4A891AC908032242EA0140D4
:109E700080A106F01FFD00240BE06B4800EB4400BE
:109E80004278694810F81410574800F0EBFA601C4B
:109E900084B2BDF808008442EFDB0FE000240BE041
:109EA0006A4800EB44004278684810F814104E48A5
:109EB00000F0D8FA601C84B2412CF1D302AB4122ED
:109EC000734974A00BF0C8FCBDF80800002837DD0A
:109ED0003249334A891AC908032242EA01406FA174
:109EE00006F0E8FC822273496948FDF72AFB50B16D
:109EF0002A492B4A891AC908032242EA01406EA165
:109F000006F0D8FC09E02549254A891AC908032228
:109F100042EA014071A106F0CDFC00240BE05C4850
:109F200000EB440042785A4810F81410304800F012
:109F300099FA601C84B2BDF808008442EFDB0FE0A0
:109F400000240BE05B4800EB44004278594810F8CD
:109F50001410274800F086FA601C84B2412CF1D31B
:109F6000FEBD0000782D0020406B03006E72665F1E
:109F70006472765F7370695F696E697428267370A6
:109F8000692C20267370695F636F6E6669672C2089
:109F90004E554C4C2C204E554C4C2900647D0300F2
:109FA000CC7C03007372635C68656172745F776177
:109FB00076655F73616D706C655F736572766963FA
:109FC000652E630025733A2564205A4552524F523C
:109FD0005F434845434B28257329206661696C3AE5
:109FE00025640000D5A30200482D00200DA4020026
:109FF000502D0020582D0020616473313239335FB9
:10A00000302072657669643A2025640A00000000F9
:10A01000616473313239335F312072657669643A35
:10A020002025640A00000000AC510020302E636639
:10A03000670000006C6F616420302E6366672066E5
:10A04000726F6D2066617466730A0000442C0020F4
:10A05000302E636667206973206469666665726581
:10A060006E742066726F6D2064656661756C740A2B
:10A0700000000000302E6366672069732073616DF5
:10A08000652061732064656661756C740A00000068
:10A090002E520020312E6366670000006C6F6164F1
:10A0A00020312E6366672066726F6D20666174666C
:10A0B000730A0000C62C0020312E63666720697386
:10A0C00020646966666572656E742066726F6D20C5
:10A0D00064656661756C740A00000000312E636669
:10A0E000672069732073616D652061732064656604
:10A0F00061756C740A000000FEB505460C4600262A
:10A100003726002000900190029009236A463146CC
:10A11000284600F023F99DF8000000049DF8011086
:10A1200000EB01209DF80210084420609DF8030018
:10A1300000049DF8041000EB01209DF80510084470
:10A1400060609DF8060000049DF8071000EB0120F8
:10A150009DF808100844A060FEBD10B50446182103
:10A16000204600F025F910BD70B56C48007800B9A4
:10A1700070BD6B4800680A2805D269480068401C19
:10A1800067490860F4E767480068401C6549086053
:10A190006548006808B908F09DFE64496448FFF707
:10A1A000ABFF62490C316348FFF7A6FF6048FFF739
:10A1B000D4FF614908705F48FFF7CFFF5F4908701F
:10A1C0005F480078B0B95C48007810B9084600785C
:10A1D000C8B101205A490870574804785748057893
:10A1E000002058490870084604714571FDF78EFF3C
:10A1F00000BF08E05048007828B95048007810B9EE
:10A2000000204F490870494800784F490870474876
:10A210000088000A487045480068000C8870434870
:10A22000007BC87041488089000A08713F48C068B7
:10A23000000C48713D48007C88713C48008A000A47
:10A24000C8713A480069000C087200242CE000BF75
:10A250003E480068B0F5106F01DB012000E00020EF
:10A2600070B131484FF41066056802203849087013
:10A27000084645608660FDF749FF00BF08F02AFEEA
:10A280003149085D31490968B1F5106F00DB0AE01A
:10A29000254909682D4A126888542C490968491CC7
:10A2A0002A4A116000BF641C092CD0DB1F4B1868C0
:10A2B000D9681A69274B1B68042B00D31AE0254B79
:10A2C0001B6803EB4303244C44F82300214B1B6819
:10A2D00003EB430304EB830359601E4B1B6803EB42
:10A2E000430304EB83039A601A4B1B685B1C194CF5
:10A2F000236000BF00BF17480068042801D3012075
:10A3000000E0002038B108F019FE00BF002011491C
:10A31000086000BF00BF00BF2AE70000642D0020D6
:10A32000602D00205C2D0020682D0020B0670020EB
:10A33000482D0020502D0020742D0020752D002068
:10A34000762D002050650020C86700206C2D00206D
:10A35000E0640020702D0020B06400202DE9F04161
:10A3600005460E4617461C46FF2C01DDFF2000E087
:10A370002046044646F080080A4880F800802146BE
:10A38000401CFDF7CCF8601CC2B2074905482B6899
:10A39000984722460449491C3846FDF7A7F8BDE80E
:10A3A000F0810000642F00206430002001607047BD
:10A3B0007CB504460D4645F080008DF80400002071
:10A3C0008DF805000222694601A8236898479DF888
:10A3D00001007CBDF8B504460D46164609480078D4
:10A3E00000B9F8BD032005F07FFE2B46324621461A
:10A3F0000548009605F096FC032005F0FFFE00BF1F
:10A40000EFE70000582D0020406B0300F8B504462C
:10A410000D4616460948007800B9F8BD1D2005F024
:10A4200063FE2B46324621460548009605F07AFC2D
:10A430001D2005F0E3FE00BFEFE70000582D0020CF
:10A44000406B0300F8B504460D46164605F07F0044
:10A450008DF800008DF80160022200216846236813
:10A460009847F8BDFEB506460C46154600200290FA
:10A470000295182C02DB1E2C00DCFEBD302C02DB0A
:10A480003F2C00DCF9E7402C00D1F6E7502C00D13E
:10A49000F3E702AB2A462146304600F02FF89DF83C
:10A4A0000800A8420FD09DF80800CDE900500749E8
:10A4B000074BC91AC908012343EA0140234605A1F5
:10A4C000726806F031FA00BFD7E70000647D030030
:10A4D000CC7C03006164735F2564207772697465C6
:10A4E000202578206661696C65642C773A25782090
:10A4F0007265616462616B3A25780A002DE9F0416A
:10A5000005460E4617461C463A4631462846FFF792
:10A5100099FF31462846FFF74BFF2070BDE8F081D8
:10A5200070B50446002501252A4600212046FFF784
:10A5300089FF70BD70B50446002504252A46002118
:10A540002046FFF77FFF70BD10B504F06FFB0020C1
:10A5500003490870034C201D07F00EFD00BF10BD1D
:10A56000582D0020406B030070B504460D4604F2E0
:10A570002740FFF7C9FB0646012D06D0022D0DD05E
:10A58000032D11D0042D19D113E0A07928B194F82E
:10A59000240010B90EB1012070BD00BFE07910B1E8
:10A5A0000EB10220F8E700BF207A08B10320F3E7DC
:10A5B00000BF607A08B10420EEE700BF0020EBE79F
:10A5C0000146481C052290FBF2F302FB1300C0B2C7
:10A5D0007047014691F82420012A01D1EE2000E0C5
:10A5E0001F20704710B501220221002001F048FF12
:10A5F000044600BF1CB1072C01D0204610BD00BF8F
:10A6000007220221012001F03BFF044600BF1CB1DC
:10A61000072C01D02046F1E700BF0A22002108469E
:10A6200001F02EFF044600BF1CB1072C01D02046CC
:10A63000E4E700BF0020E1E710B504462C212046E6
:10A64000FCF76DFF012020714020206144F2506032
:10A65000606110BD10B572B600BF06F019FA00BFF8
:10A6600000BF05F01BFF0028FBD100BF00BF1E4943
:10A670001E4A891AC908012242EA01401CA106F0BB
:10A6800019F900BF1D48006800F0010000B100BECC
:10A6900000BF1549154A891AC908022242EA014039
:10A6A00017A106F007F900BF00BF00BF00BF00BF41
:10A6B000BFF34F8F00BF00BF00BF1048E4380068F1
:10A6C00000F4E06012490843001D0C49E4390860B9
:10A6D00000BF00BF00BFBFF34F8F00BF00BF00BF70
:10A6E00000BF00BFFDE70000647D0300CC7C0300D9
:10A6F000466174616C206572726F7200F0ED00E06B
:10A7000053797374656D2072657365740000000081
:10A710000000FA053EB5044600200090019002902A
:10A7200002946A46002144F20100FFF793FF3EBD08
:10A7300070B505460E462C46207820B961792079FF
:10A7400008F0BEFE1CE02078012807D10D48006803
:10A75000401C0C490860FEF7FFF911E02078092839
:10A7600002D108F09DFE0BE02078032808D10648AE
:10A77000007828B1042204F10801606808F00EFE98
:10A7800070BD00002C2C0020C12B00202DE9F843C7
:10A79000054689462C4620780A2804D10120FDF779
:10A7A0001DFFBDE8F88320780B2803D10220FDF7B8
:10A7B00015FFF6E74B480078002847D04948007855
:10A7C000012844D12078062840D14749474A891AB0
:10A7D000C908032242EA014045A106F06BF8FEF7E2
:10A7E00021FE04F0F5F902F00FFA06460121FEF70A
:10A7F00017FF4349086000BF08460068002817DCBF
:10A8000040A03949394A891AC9080322009042EA0E
:10A810000140BB2341A248A106F072F805F03EFEBC
:10A8200000BF002600BF0020FFF774FF00BF00BF7D
:10A8300000BF08F075FB04F0CFF908204449087008
:10A840000846FDF763FC0120FDF7FAFD48E02548C6
:10A850000078022844D12078022805D12848D4E97C
:10A8600001120068FEF7D4FF04F0EEF8074604F08A
:10A87000F1F88046002622480068FEF773FEB0F12A
:10A88000604F0BD91849194A891AC908032242EAAC
:10A89000014030A106F00EF801260DE020780728CF
:10A8A0000AD11149114A891AC908032242EA014012
:10A8B00033A105F0FFFF01268EB111480068FEF7B5
:10A8C000D1FDFEF78DFD04F0B1F904F0D3F908F0E5
:10A8D0001DFB0920344908700846FDF717FC00BF2E
:10A8E00000BF5EE7A82D0020647D0300CC7C030040
:10A8F00073746172742073616D706C650000000088
:10A90000B02D00206D5F73616D706C655F64617464
:10A91000615F6664203E2030000000007372635C5B
:10A920006465766963655F6374726C5F7365727684
:10A930006963652E6300000025733A2564205A413F
:10A94000535345525428257329206661696C0000D1
:10A95000A868002073746F702073616D706C65203F
:10A96000626563617573652066696C652073697AD9
:10A970006520697320746F6F206C617267650000D9
:10A9800073746F702073616D706C652062656361B4
:10A990007573652073746F702073616D706C6520C2
:10A9A0006576656E74000000E068002070B50546AD
:10A9B0000E4600240AE0084850F8240028B1064852
:10A9C00050F82420314628469047641C034800680C
:10A9D0008442F0DB70BD000088690020C02D00209B
:10A9E0002DE9F84307460C469046264800888442E5
:10A9F00044DC4FF6FF7500200090684600F01EFB17
:10AA000000BF214890F800902048007804F064FDD1
:10AA1000484501D1012000E0002030B91B480578ED
:10AA2000007804F059FD194908709DF8000000F005
:10AA30000BFB4FF6FF7085421ED01548006840F8AA
:10AA400035808FB1002C0FDD124909680D4A12883C
:10AA500005FB021022463946FCF748FD0C48006809
:10AA600000EBC500848005E000200949096801EB7E
:10AA7000C5018880002600E0042600E00926304653
:10AA8000BDE8F8838A2E0020882E0020892E002021
:10AA9000802E0020842E00202DE9F0411AE0164877
:10AAA0000478164800681649098804FB0105154812
:10AAB000006800EBC40086881248006850F83470C3
:10AAC00031462846B8470C48007804F005FD0A498D
:10AAD000087000BF00BF002058B900BF06490878C1
:10AAE00009490978814201D1012100E000210029B2
:10AAF000D5D0BDE8F0810000882E0020842E0020F3
:10AB00008A2E0020802E0020892E002030B503469A
:10AB1000481C4FF6FF7505EAC004104600F0030517
:10AB20000DB9012500E000250DB9072030BD08480A
:10AB300002601019074D28600020074D2870074D4E
:10AB4000287007480380074801800020EEE70000D6
:10AB5000802E0020842E0020892E0020882E0020A8
:10AB60008A2E00208C2E00202DE9F04707460E4645
:10AB700014461F4890F8220010B90820BDE8F0875D
:10AB80001B4890F82200032801D01120F6E70CB9E9
:10AB90000720F3E70421164880F82210807AC0F3DA
:10ABA000C00018B971021248016101E01048066145
:10ABB0000F48C7608482C48200218183012C01DD9B
:10ABC000522000E05120814609480122016948468F
:10ABD00009F02AF8054600BFA846B8F1000F04D0D6
:10ABE00000BF4046FFF796FD00BF00BF0020C5E74D
:10ABF0000C6F00202DE9F04107460E4615462D4802
:10AC000090F8220010B90820BDE8F081294890F89A
:10AC10002200032801D01120F6E70DB90720F3E741
:10AC20000521244880F82210807AC0F3C00018B9AA
:10AC300071022048016101E01E4806611D48C7609D
:10AC40008582C58200218183012D12D101220169F3
:10AC5000582008F0E9FF044600BFA046B8F1000FF5
:10AC600004D000BF4046FFF755FD00BF00BF0020E5
:10AC7000CAE71048807A00F00700012807D10D4884
:10AC800001220169592008F0CFFF044605E00122A6
:10AC90002946D72008F0C8FF044600BFA046B8F1F7
:10ACA000000F04D000BF4046FFF734FD00BF00BFD7
:10ACB0000020A9E70C6F0020064890F82200032826
:10ACC00005D0044890F8220008B101207047002008
:10ACD000FCE700000C6F0020044890F822000328D5
:10ACE00002DB0248001D70470020FCE70C6F0020CB
:10ACF000F0B587B004460E463A4890F8220010B1ED
:10AD0000082007B0F0BD5EB1E078FF2808D0607879
:10AD1000FF2805D02078FF2802D0A078FF2801D195
:10AD20000720EEE7E0782F4981F85800084690F8B0
:10AD300058700020009003460122114601903846C9
:10AD400005F057F900BF00BF264991F8580005F0FB
:10AD50006FFA00BF244B0FCB03AD0FC5A0788DF861
:10AD60000C0020788DF80D0060788DF80E0000231F
:10AD70001E4A03A91E4804F091FF054600BF2F4656
:10AD800027B100BF3846FFF7C5FC00BF00BF15481C
:10AD90000660012180F82210807A20F00701114816
:10ADA0008172807A20F008010E488172002180F8BB
:10ADB0002310FF200B4981F828000A2001F13803F5
:10ADC0000122283100900A4804F0C5FF054600BF63
:10ADD0002F4627B100BF3846FFF79CFC00BF00BFDD
:10ADE00000208EE70C6F0020286F0300C14F030086
:10ADF000186F03007CB5144890F8220008B90820A9
:10AE00007CBD114890F82200032801D01120F7E7FB
:10AE10000E4C201D07F0B0F800BF0B4890F85840CA
:10AE20000025002000902B46024601460190204656
:10AE300005F0DFF800BF0021034880F8231080F8F8
:10AE400022100020DCE700000C6F0020186F0300C8
:10AE500010B50446022C0AD10C490D4A891AC908BA
:10AE6000032242EA01400BA105F024FD01E001208C
:10AE700010BD00BF0549064A891AC908032242EAE3
:10AE8000014010A105F016FD0120F1E7647D0300EB
:10AE9000CC7C0300506F776572206D616E616765D1
:10AEA0006D656E742077616E747320746F207265A7
:10AEB00073657420746F20444655206D6F64652E51
:10AEC00000000000506F776572206D616E616765EC
:10AED0006D656E7420616C6C6F77656420746F2093
:10AEE000726573657420746F20444655206D6F64DD
:10AEF000652E000010B5024802F0A2FC10BD000053
:10AF0000902E002030B503460C460AB9072030BD0C
:10AF100019684FF0FF358D60CD604A61012C01D179
:10AF2000012000E0002008610020F0E738B5134858
:10AF3000006800900823A82211491248006804F014
:10AF40005BFB04460CB1204638BD0F4A69460F48EA
:10AF500002F07CFC04460CB12046F5E701210B48C9
:10AF600002F01AFD01230A4A1946084802F03AFC89
:10AF70000120084908702046E6E70000306D030014
:10AF80003C6E0020206D030091380300902E0020BD
:10AF9000FFFF7F009C2E00202DE9F84306460D465A
:10AFA0009046344600200090684600F047F84FF085
:10AFB000FF33D4E9021059405840014308D103F04F
:10AFC00025FD401941F10001C4E90201012700E01B
:10AFD00000279DF8000000F037F817B90020BDE801
:10AFE000F883C4F81880206900B12561214600204B
:10AFF0000AF010FCF3E7F8B504462546002000905F
:10B00000684600F01BF84FF0FF33D5E902105940B5
:10B010005840014301D1002604E04FF0FF31A96000
:10B02000E96001269DF8000000F00EF80EB900203E
:10B03000F8BD294601200AF0EDFBF9E710B50446FA
:10B04000204608F041FD10BD70B5044625460E4867
:10B050008068B0B1ADB9FEF751FE06460A480068F7
:10B060000A490860084840684FF0E021C1F804012F
:10B070000020054988601EB900BF62B600BF00BF4E
:10B0800000BF00BF70BD0000F46E002000E100E0D2
:10B09000F8B505460C4617462088001DB84201D970
:10B0A0000C20F8BD684679DF064600BF304600B187
:10B0B000F7E700BF0320218868542088401C2080C7
:10B0C0001920218868542088401C2080208841193C
:10B0D000BDF800000AF0A9FE218808442080002065
:10B0E000DFE70000002113E00C480269012308E0BB
:10B0F00000BFD0680079884201D1002303E0D06806
:10B100000268002AF4D100BF0BB108467047491C01
:10B110000A29E9DB4FF0FF30F8E70000888C0020B7
:10B1200010B504463948007818B90020FDF76AF9CF
:10B1300064E036480078012815D13548006818B910
:10B140000120FDF75FF959E031480068002855D02B
:10B150000020FDF757F92F480068FFF74CFF00204B
:10B160002A4908704AE029480078022820D1284856
:10B170000068062811D22648007800F0010018B9AE
:10B180000120FDF73FF939E02148007800F0010087
:10B1900038B30020FDF736F930E00020FDF732F932
:10B1A0001C480068FFF727FF00201849087025E0B9
:10B1B00016480078032821D115480068062811D2C6
:10B1C0001348007800F0010018B90120FDF71AF9C2
:10B1D00014E00F48007800F0010010B10020FDF7E6
:10B1E00011F90BE00A4800689621484342F21071B9
:10B1F000884203D300200649086010BD0448006857
:10B20000401C0349086000BFF7E70000F82D00204C
:10B21000FC2D0020706B03002DE9FC41054688469B
:10B220001646002437880020308095F82D0058B14C
:10B230003A463146404600F0A9FA044600BF20468F
:10B2400008B1BDE8FC8100BFA87850B13A4631464C
:10B250004046FFF71DFF044600BF204600B1F0E75F
:10B2600000BFE87860B1E97848B23B4632464146D3
:10B2700003F0F2F9044600BF204600B1E1E700BF49
:10B28000686868B1696891F900003B4632464146FA
:10B290000AF0AAFD044600BF204600B1D1E700BF76
:10B2A000288900280EDD43460622022105F1080008
:10B2B000CDE900670AF065FE044600BF204600B1F4
:10B2C000BFE700BF288A00280EDD4346072203217E
:10B2D00005F11000CDE900670AF053FE044600BFF7
:10B2E000204600B1ADE700BF288B00280EDD4346A5
:10B2F0001522142105F11800CDE900670AF041FE7E
:10B30000044600BF204600B19BE700BF286A58B141
:10B310003B4632464146286A01F0E5FB044600BF41
:10B32000204600B18DE700BF686A58B13B463246FF
:10B330004146686A03F06EFF044600BF204600B134
:10B340007FE700BF95F82C0000280BDD3B46324616
:10B350004146284609F036FC044600BF204600B1AD
:10B360006FE700BF287858B13B4632464146284631
:10B3700004F04EF8044600BF204600B161E700BF6C
:10B3800020465EE7F8B504460E46154600200090BC
:10B390002B466A463146204600F008F807460FB9AA
:10B3A0000020F8BDBDF800002044FAE7F0B50446DF
:10B3B0000D461E4604B10AB90020F0BD002103E08D
:10B3C000605C401C084481B2481CA84206DA108820
:10B3D0008842F5DC481C205CB042F1D1A94201DB77
:10B3E0000020EAE7881C87B2605C10B1605C401EF8
:10B3F00000E0002083B213B1F818A84201DD00205C
:10B40000DBE717801846D8E780F83010704770B532
:10B4100004460D4605B10CB90E2070BD05F178004B
:10B4200001F096FA08B90720F7E70020A0702C2257
:10B4300005F17801201DFCF759F8002084F8300050
:10B44000D5F8A4006063D5F8A800A0634FF6FF709C
:10B45000A4F8240404F58260C4F82004002140F21A
:10B460002C40C4F82614A4F82A140155207810B9E9
:10B47000FF2084F8540004F15500C4F8100420465D
:10B48000FFF7A7F840F21441085304F2144204F104
:10B4900055012846FFF7C0FE064600BF304600B102
:10B4A000BBE700BF04F231204FF48361085120460E
:10B4B000FFF78FF8A4F81C044FF48360015904F2DD
:10B4C0001C4205F13C00FFF7A7FE064600BF3046D0
:10B4D00000B1A2E700BF012151200155208B81B2AC
:10B4E00048200153012084F83C00002121645020B1
:10B4F00001556169616404F13C02002104F15400CA
:10B5000072DF064600BF304600B186E700BF01206B
:10B510002070304681E770B504460D462C2229463E
:10B52000201DFBF7E3FF70BD70B504460D462E46A7
:10B530002088102804D0112807D026280FD109E030
:10B540002146304606F084FF0AE02146304607F0E7
:10B550007BF905E02146304607F0FEFA00E000BF27
:10B5600000BF70BD70B504460E46207808B90820AB
:10B5700070BDA670002140F22C40C4F82614A4F837
:10B580002A140155A07910B1A078012809D0E079DA
:10B5900010B1A078012804D0E07970B1A078022819
:10B5A0000BD1606B30B1012084F82D040820616B51
:10B5B000884702E0002084F82D0431462046FEF73B
:10B5C000D3FFA070606BA0B1A078032802D0A07850
:10B5D00004280ED1607960B194F82E0448B9002097
:10B5E00084F83004012084F82F040720616B884719
:10B5F00002E0002084F82F04182104F13C00FBF73E
:10B600008EFF012084F83C0004F12C0007F033FB8E
:10B6100020B194F82C105120015502E00121512055
:10B62000015594F8240060B104F1280007F023FBD1
:10B6300020B194F828105220015502E00121522037
:10B640000155002150200155A078052824D2DFE8BB
:10B6500000F01F030A11180004F13C01204609F014
:10B6600014FB054619E004F13C01204609F0F5FA07
:10B67000054612E004F13C01204609F018FB05469E
:10B680000BE004F13C01204609F03FFB054604E0D5
:10B69000002084F8310000E000BF00BFA07898B11E
:10B6A00004F13C0204F15400D4F8201472DF054682
:10B6B0000DB128465CE794F8301094F8540073DF1D
:10B6C00005460DB1284653E7606B18B194F8310078
:10B6D000616B884700204BE72DE9F041044600BF2D
:10B6E00014B90E20BDE8F08100BF1C2221461C4881
:10B6F000FBF7FCFE1B481A490860206860B120680F
:10B700007ADF05460DB12846ECE7164821680A683D
:10B7100002604968416005E012487BDF05460DB1D3
:10B720002846DFE7002617E006EB86000E4901EB0E
:10B73000800700BF4FF6FF70388000BF0B4800EB5A
:10B74000461078600A4A0021381DFFF7DBFB0546EA
:10B750000DB10320C6E7761C002EE5D00020C1E71E
:10B760003C6C0020502E0020286C0020086C00202B
:10B77000F15E030070B504460D46034988682A4609
:10B78000214602F0EBFF70BD586C00202DE9FC4112
:10B7900005460C46174620880930B84202D90C20CD
:10B7A000BDE8FC8168466DDF064600BF304600B14B
:10B7B000F6E700BF0820218868542088401C2080BC
:10B7C0001B20218868542088401C20802088284421
:10B7D000DDF801100160BDF8051081802088801D12
:10B7E00020809DF80000400818B900202188685486
:10B7F00002E00120218868542088401C208000201D
:10B80000CEE7000070B504F03DF9044600BF2046C5
:10B8100000B170BD00BF00BF084D28464FF0030CBB
:10B8200000DF00BF044600BF204600B1F1E700BFC3
:10B8300004F0A2F904462046EBE70000D095002072
:10B84000014600BF09B90E20704700BF01480160E2
:10B850000020F9E75C2F002010B51349134A891A1C
:10B86000C908042242EA014011A105F023F84FF073
:10B87000FF3100203DDF044600BF204600B110BD6F
:10B8800000BFB12100203CDF044600BF204600B1CC
:10B89000F5E700BF1348416901208847022005F001
:10B8A000ADFA0020EBE70000647D0300CC7C0300D0
:10B8B000496E20626C655F6466755F627574746F53
:10B8C0006E6C6573735F626F6F746C6F61646572C9
:10B8D0005F73746172745F66696E616C697A650D1D
:10B8E0000A000000B495002010B5054800684169C1
:10B8F00000208847FFF7B0FF0446204610BD000037
:10B900005C2F002010B588B0044620216846FBF764
:10B9100006FE0320ADF8000020788DF802009DF8A7
:10B920000D0020F0200020308DF80D009DF80D0056
:10B9300020F0080008308DF80D0001208DF810006F
:10B940008DF80C001720ADF8040001208DF81300CD
:10B950008DF812008DF811006088A21D694600F074
:10B960007FFE08B010BD000030B585B00546244B01
:10B970000FCB8DE80F0000BF15B90E2005B030BD0C
:10B9800000BF4FF6FF701F4988802868486100207B
:10B9900008760846406908B91B4848611948FFF70E
:10B9A0004FFF044600BF204600B1E7E700BF00BFDD
:10B9B00001208DF812004FF65960ADF8100000BF5D
:10B9C000104A921C04A90120A8DF044600BF2046AB
:10B9D00000B1D3E700BF0B49684662DF044600BFF1
:10B9E000204600B1CAE700BF0648FFF78BFF0446B8
:10B9F00000BF204600B1C1E700BF0020BEE7000045
:10BA000030700300B495002019DB020070B50446C5
:10BA10000D4600BF04B970BD00BF2088102806D0B5
:10BA2000112808D051280AD0532810D10BE0204605
:10BA300006F008FD0CE0204606F0F8FE08E020467F
:10BA400007F068F804E0204607F040F800E000BF87
:10BA500000BF00BFDFE7000070B504460426207B6E
:10BA6000012802D0022822D109E002F07BF8054625
:10BA70000DB9012602E0112D00D1062619E0607BE8
:10BA8000142801DC607B08B905260FE0627B04F115
:10BA90000E011248FBF72AFD607B1049091F8861DF
:10BAA000084609F061F9054605B9012601E00226BC
:10BAB00000BF00BF012E0FD0207B314600F058F8A8
:10BAC000054625B1064800684169032088470448B7
:10BAD000006841690220884770BD0000E0950020A1
:10BAE0005C2F002070B505460E4600BF1E4800685A
:10BAF00020B11D48406808B1012000E0002000B9D5
:10BB000070BD00BF184800F1080142682846904700
:10BB1000044600BF082C24D07CB9002013490968D2
:10BB200048760121022000F023F80446CCB10F48EA
:10BB3000006841690320884713E000200B49096829
:10BB400048760621022000F013F8044624B1074885
:10BB50000068416903208847044800684169022061
:10BB6000884700BFCCE70000D09500205C2F002064
:10BB7000F0B587B004460D460327002001900290DF
:10BB8000039004900320069020208DF814008DF877
:10BB900015408DF816500E48C088ADF804000220FC
:10BBA0008DF806000020ADF8080006A8039005A84F
:10BBB00004900749888801A9AEDF064626B9BDF87A
:10BBC0001800032800D00C26304607B0F0BD000056
:10BBD000B495002030B58BB0044634B1012C29D087
:10BBE000022C32D0032C49D13AE02B492B4A891A36
:10BBF000C908032242EA014029A104F05BFE68461D
:10BC0000FEF71AFD01208DF8000069463048FFF765
:10BC100082FC00212F48FFF7ADFD05461E491F4A53
:10BC2000891AC908032242EA01402A462AA104F0DF
:10BC30004BFE2EE01849194A891AC908032242EA24
:10BC400001402BA104F036FE23E01349134A891A60
:10BC5000C908012242EA01402EA104F02BFE18E09F
:10BC60000D490E4A891AC908012242EA014038A149
:10BC700004F020FE00BF002000BF0AE00649074A8A
:10BC8000891AC908012242EA01403DA104F012FECE
:10BC900000BF00BF0BB030BD647D0300CC7C03004F
:10BCA000446576696365206973207072657061729E
:10BCB000696E6720746F20656E74657220626F6FA5
:10BCC000746C6F61646572206D6F64652E00000096
:10BCD0005C91002079D20200446973636F6E6E65D7
:10BCE00063746564202564206C696E6B732E00009C
:10BCF0004465766963652077696C6C20656E746550
:10BD00007220626F6F746C6F61646572206D6F6416
:10BD1000652E00005265717565737420746F20651F
:10BD20006E74657220626F6F746C6F6164657220EF
:10BD30006D6F6465206661696C6564206173796EFE
:10BD40006368726F6E656F75736C792E000000000A
:10BD50005265717565737420746F2073656E64200D
:10BD60006120726573706F6E736520746F20636CF1
:10BD700069656E74206661696C65642E0000000060
:10BD8000556E6B6E6F776E206576656E7420667289
:10BD90006F6D20626C655F6466755F627574746F49
:10BDA0006E6C6573732E000070B505460E462888CC
:10BDB000102802D011282CD115E01748006860B96E
:10BDC00000F0F8FE044600BF34B11448006818B112
:10BDD000204612490968884700BF0F480068401C88
:10BDE0000D49086016E00C480068401E0A490860CA
:10BDF0000846006860B9FEF7F5FB044600BF34B1A1
:10BE00000648006818B1204604490968884700BF01
:10BE100000E000BF00BF70BD4C2E0020482E002067
:10BE200070B504460D462088102806D0112808D089
:10BE300012280ED0502810D107E0204606F0CAFA8A
:10BE40000CE0204606F0D8FC08E0204606F0A4FEF0
:10BE500004E0204606F0A6FA00E000BF00BF70BD77
:10BE60002DE9F04104460F46A6882088102806D008
:10BE7000112817D019283DD01A2848D116E007F00C
:10BE800081FC304607F05AFC20B900BF0420FEF7C1
:10BE900041FC06E0E07B022803D131461D4803F057
:10BEA00015FC34E0304607F091FC30E0207A0509BB
:10BEB000042D01DB012000E0002002463146154838
:10BEC0000C3002F0BAFB032D01DB012000E0002062
:10BED000024631460F48083002F0AFFB022D01DB6D
:10BEE000012000E00020024631460A48001D02F011
:10BEF000A4FB0CE0207A48B9607AC0F3C0052A465A
:10BF0000314604480C3002F098FB00BF00BF00BF70
:10BF1000BDE8F081646C00202DE9BE4105460F4666
:10BF2000288821282BD006DC10280BD0112817D008
:10BF300013287DD154E03B287BD052287BD0562853
:10BF4000F7D1C5E0A88877490880012076490870B4
:10BF50007648006818B10846744909688847DDE0EA
:10BF60004FF6FF706F49088002206F4908706F48D4
:10BF7000006818B108466D4909688847CEE06C49E9
:10BF80006C4A891AC908042242EA01406AA104F0F5
:10BF900091FC00200290A88802A98FDF044600BF10
:10BFA000A046B8F1000F19D068A06149614A891A0A
:10BFB000C9080322CDE9000842EA0140462366A2EF
:10BFC0006DA104F0B1FC04F069FA00BF00BF26B116
:10BFD00000BF3046FEF79EFB00BF00BF00BF9DE0E4
:10BFE00000231A4685214F4800887FDF044600BFA2
:10BFF000A046B8F1000F19D054A04D494D4A891AF6
:10C00000C9080322CDE9000842EA01404C2352A2AC
:10C0100059A104F089FC04F041FA00BF00BF26B129
:10C0200000BF3046FEF776FB00BF00BF00BF75E0E3
:10C0300073E028E0FFE700231A46194639480088D4
:10C04000B1DF044600BFA046B8F1000F19D03FA0F1
:10C050003749384A891AC9080322CDE9000842EA5B
:10C06000014052233CA244A104F05EFC04F016FA05
:10C0700000BF00BF26B100BF3046FEF74BFB00BF3C
:10C0800000BF00BF4AE0A888132176DF044600BF46
:10C09000A046B8F1000F19D02CA02549254A891ACD
:10C0A000C9080322CDE9000842EA014058232AA228
:10C0B00031A104F039FC04F0F1F900BF00BF26B152
:10C0C00000BF3046FEF726FB00BF00BF00BF25E0E3
:10C0D000A888132176DF044600BFA046B8F1000F00
:10C0E00019D01AA01249134A891AC9080322CDE9A6
:10C0F000000842EA01405E2317A21FA104F014FCCD
:10C1000004F0CCF900BF00BF26B100BF3046FEF7F7
:10C1100001FB00BF00BF00BF00E000BF00BFBDE8E3
:10C12000BE8100003C2F0020442F0020402F002023
:10C13000647D0300CC7C0300504859207570646115
:10C14000746520726571756573742E006572725F17
:10C15000636F6465000000002E2E5C6C69627A6E6D
:10C160006F726469635C7372635C7A626C655F6D45
:10C170006F64756C652E630025733A2564205A45FB
:10C1800052524F525F434845434B2825732920663E
:10C1900061696C3A2564000070B50446204609F0D8
:10C1A0003EFE0546C5F3400070BD70B5044620460E
:10C1B00009F035FE054605F0010070BD0120024979
:10C1C0000870002070470000C12B002000200149AA
:10C1D00008707047C12B002030B50246087A0B78F2
:10C1E00033B1012B05D0022B05D0032B14D101E074
:10C1F00000BF00BF00BF4B7800EB4004084D2D6826
:10C2000005EB84042372002300EB4004044D2D68E9
:10C2100005EB8404A37200E000BF00BF30BD000046
:10C220004C2F002001460A46906970472DE9FE43D5
:10C2300080460C4691464546AE692869B0F5007FB8
:10C2400002D00620BDE8FE831648006808B1112020
:10C25000F8E7C6F81890B460124805600027124944
:10C2600005F11400FEF744FD07464FB944B908F044
:10C27000D9FB0E48007808B9002000E00D200746E1
:10C2800077B100200749086054B1094A07CA8DE810
:10C290000700B069029069464046B268904700BF07
:10C2A0003846CFE7D02E0020213D0300CC2E0020C1
:10C2B000E86E030030B503461D4611B101290ED1C9
:10C2C00005E014460CB100202070002030BD0AB9F2
:10C2D0000720FBE71446281D20600020F6E700BF7A
:10C2E00000BF0620F2E700002DE9FE4307460D4699
:10C2F000B846D8F8184000261B480068404502D0D0
:10C300001120BDE8FE83FEF7D7FC08B11120F8E745
:10C3100095E80700C4E90412E060AB889AB2296886
:10C32000A868FEF721FC064656B9A06840B908F097
:10C3300079FB0E48007808B9002000E00D20064681
:10C34000A06870B16EB10A4A07CA8DE8070004F10F
:10C350000C000190A069029069463846A268904797
:10C3600000BF3046CDE70000D02E0020CC2E0020AC
:10C37000006F0300FEB506463746BD6913480068E6
:10C38000B84201D01120FEBDFEF796FC08B1112085
:10C39000F9E7FEF72FFD044614B900200B490860A9
:10C3A000A86880B10A4A07CA8DE807000CB10120CD
:10C3B00000E000208DF80100A8690290694630462F
:10C3C000AA68904700BF2046DDE70000D02E00207D
:10C3D000F46E03002DE9FE4307460D46B846D8F833
:10C3E000184000261B480068404502D01120BDE8D7
:10C3F000FE83FEF761FC08B11120F8E795E807001D
:10C40000C4E90412E060AB889AB22968A868FEF714
:10C41000F1FB064656B9A06840B908F003FB0E4888
:10C42000007808B9002000E00D200646A06870B131
:10C430006EB10A4A07CA8DE8070004F10C000190AA
:10C44000A069029069463846A268904700BF30460E
:10C45000CDE70000D02E0020CC2E00200C6F030072
:10C4600070B505460C46012C01D1042000E00520E2
:10C47000024908700846FBF749FE70BD0C680020B1
:10C4800030B503460020042B23D2012A07D101290D
:10C4900003D103F10E04E4B200E00024224679B196
:10C4A000012902D0022911D104E003EB43040A4D13
:10C4B0002A550DE003EB4304074D2C44627007E05E
:10C4C00003EB4304044D2C44A27001E0072000BF9D
:10C4D00000E0072030BD0000FC6B00202DE9FC4788
:10C4E00004460D461646A71C4FF001080020019097
:10C4F00001A8FEF7A3FD3048406828602E48406838
:10C500002D498968411A2D480068401CA0EB01099B
:10C5100015E001212A4803F0F6F802F0CBFD82462F
:10C520005146274803F0EFF82348406822498968BC
:10C53000411A22480068401CA0EB010900BF4F458A
:10C54000E7D8B8F1000F30D00021009176B1009902
:10C5500021F00301491C0091009921F00401091DFB
:10C560000091009964F3891100910DE0009921F088
:10C570000301891C0091009921F00401091D00911B
:10C58000009964F39F5100910B4949680B4A126866
:10C590001140094A0C3202EB810000990160064902
:10C5A000496839440C3A516000BF9DF80400FEF719
:10C5B0004BFD4046BDE8FC87887C0020E82E00202B
:10C5C000A48C002070B504460D460A2D03D10D2120
:10C5D0002046FFF7F7FFA168481CA060206845547B
:10C5E000D4E90110884202D3204603F0E2FB70BD7B
:10C5F0000448806803494968884201D10120704796
:10C600000020FCE7887C002070B505460C460448F5
:10C61000006820B121460020014A1268904770BD91
:10C62000002E002070B504460D46032C06D1A9202B
:10C630000349086000BF002004F0E0FB70BD00006B
:10C64000200500400146024850F8210070470000D4
:10C65000E86C00200146014840567047186D0020E4
:10C6600070B590B006460C461546A07818B9012062
:10C670008DF80E0002E0A0788DF80E002088ADF84D
:10C680000C0000200290607C02A908F09DFBA07CB9
:10C690000DF1090108F098FBE07B08B1012000E0F2
:10C6A00000209DF80A1060F3C3018DF80A10207C69
:10C6B00008B1012000E000209DF80A1060F3041189
:10C6C0008DF80A10207B08B1012000E000209DF8C1
:10C6D0000A1060F300018DF80A10207D08B10220D5
:10C6E00000E001209DF80A1060F342018DF80A1065
:10C6F0001C2109A8FAF713FF607BC0F3001018B9DA
:10C70000607BC0F34010F8B100200090E07C0DF198
:10C71000010108F059FB00BF9DF8000020F00F0058
:10C72000401C8DF800009DF8000020F0F000103053
:10C730008DF8000000BF9DF8020020F00600801C6C
:10C740008DF80200CDF838D0607B8DF82400A07BF6
:10C750008DF82500142104A8FAF7E1FE03A804903F
:10C7600002A80590A088ADF81C00A06820B1E08860
:10C77000ADF81800A0680890A069002849D00020F2
:10C780000190A0690088ADF82C00A0694088ADF840
:10C790002E00A06940680A9001A80D90A169087B4D
:10C7A00001A908F011FBA169487B0DF1050108F012
:10C7B0000BFBA069807A08B1012000E000209DF801
:10C7C000061060F3C3018DF80610A069C07A08B1A5
:10C7D000012000E000209DF8061060F304118DF8A0
:10C7E0000610A069007A08B1012000E000209DF841
:10C7F000061060F300018DF80610A069807B08B177
:10C80000022000E001209DF8061060F342018DF83F
:10C810000610E06908B1E0690C902B4604AA09A94A
:10C820003046AADF10B070BD70B504460D4600203A
:10C83000E070401EE0622946204602F0CFFD08B1BC
:10C84000042070BD04F22E2002F015FC4AF655219A
:10C85000884201D00320F4E794F83000E92807D09B
:10C8600094F83000EB2817D13220005D902813D1C6
:10C8700004F1660002F0F3FB20F07F400749884294
:10C8800001D10020DDE704F1820002F0E8FB044959
:10C89000884201D10020D4E70220D2E7464154006B
:10C8A00046415433024600E0521C107810B1107813
:10C8B0008842F9D11078704770B505460DB9094C1A
:10C8C00001E0084C083409E0204602F09CFB0646D3
:10C8D00006B904E028467168884700BFF4E700BF46
:10C8E00070BD0000DC6C002010B504462CB901209E
:10C8F000064948700020FFF7DFFF012C04D101201A
:10C9000002498870FFF7D8FF10BD0000D46C0020EA
:10C910000246891E5069801E884201D80020704757
:10C920005389906A01FB0300F9E72DE9F0470246BD
:10C9300013468C46D3E90245DCE90267B6EB0408EE
:10C9400077EB050002D30120BDE8F0870020FBE76C
:10C9500001468878012805D191F82000012801D1ED
:10C96000002070470120FCE72DE9F04F89B0064612
:10C970000F46002458E03D5DFF2D4ED0C5F3C0109A
:10C98000049025F0800005A941F82400049880B1A6
:10C9900005A850F82400039003A803F00FFC80467C
:10C9A0000121039A01FA02F0C8F8080500BF00BF90
:10C9B00010E005A850F82400039003A803F0FEFB44
:10C9C00080460121039A01FA02F0C8F80C0500BF65
:10C9D00000BF00BF05A850F824804FF00109CA46E7
:10C9E0004FF0000BCDE9018BCDF80CB001A803F09E
:10C9F000E5FB009049EA4A0040EA8B01029841EACF
:10CA00000021039841EA0041009800F5E060019A96
:10CA100040F8221000BF00BF04E04FF0FF3005A92E
:10CA200041F82400601CC4B2042CA4DB05AA3168C0
:10CA3000002007E052F8205001F5AC6343F8205085
:10CA4000431CD8B20428F5DB00BF09B0BDE8F08F65
:10CA500033B58BB00546002000900C9878B10024C7
:10CA60000BE021460CA802F022FE28B1009A501CCF
:10CA7000009001A820F81240641C142CF1D32C2241
:10CA800069462846FAF732FD0DB030BD01460888E8
:10CA9000062808DB0888B0F5486F06DD08884FF6E1
:10CAA000FF72904201D0072070474888062808DBB3
:10CAB0004888B0F5486F06DD48884FF6FF7290420F
:10CAC00001D00720F0E708884FF6FF72904208D0A7
:10CAD0004888904205D008884A88904201DD0720A6
:10CAE000E2E70020E0E72DE9F04107460D46144655
:10CAF00098462088801D404502D90C20BDE8F08171
:10CB00003846FFF7C3FF064600BF304600B1F5E7E1
:10CB100000BF0520218868542088401C20801220F6
:10CB2000218868542088401C208022885119388828
:10CB300009F07BF9218808442080228851197888DF
:10CB400009F073F92188084420800020D6E710B549
:10CB5000044600BF2046FDF7DDFD00BF10BD00000C
:10CB6000F8B505460C46607A88B9207A10B91048A5
:10CB7000476801E00E4887682A4639466068FEF734
:10CB80000BFA064616B1304607F08EFF0EE0002085
:10CB900020720748406948B101208DF80000ADF8C7
:10CBA0000250034841696846884700BFF8BD00004D
:10CBB0003C6C002010B5012200210846FFF760FC04
:10CBC000044600BF1CB1072C01D0204610BD00BF99
:10CBD000072202210120FFF753FC044600BF1CB1CD
:10CBE000072C01D02046F1E700BF042202210020DB
:10CBF000FFF746FC044600BF1CB1072C01D02046BD
:10CC0000E4E700BF0020E1E710B50F480021016014
:10CC100041600E4809F0E0FE0C48007D64380A4986
:10CC200008700A48007C401C48700848007B8870E7
:10CC30000648007AC87005480079087103480078F2
:10CC40004871084610BD0000B52D00207C6800200A
:10CC50002DE9F04782468946DAF80040B9F1000F25
:10CC600006D1E76817B16069B84215D8012713E00B
:10CC70004946504601F0CEFD0646022E02D2012062
:10CC8000BDE8F087701C08B93046F9E76069B0422A
:10CC900001D93046F4E74F463D4600BF6D1C606940
:10CCA000A84204D80225BD4201D90020E8E7294660
:10CCB000504601F0AFFD064606B909E0012E01D04D
:10CCC000701C08B93046DBE7BD42E7D10020D7E74A
:10CCD00000BF00BF4FF0FF322946204606F006FC99
:10CCE0008046B8F1000F08D1B9F1000F05D02A46EF
:10CCF0004946204606F0FAFB8046B8F1000F0DD1F8
:10CD0000E560D4E90410801E814202D22069401EF1
:10CD10002061207940F00100207107E0B8F1010F97
:10CD200002D14FF0FF3000E0012005462846A7E77A
:10CD30002DE9F35F8A46DAF80090009800F12005AB
:10CD40000B222021284602F0BFFA00208046074629
:10CD50004FF0080B00BF38467F1C19F80040202C0C
:10CD600000DC55E02F2C01D05C2C0AD100E07F1CA8
:10CD700019F807002F28FAD019F807005C28F6D018
:10CD800046E02E2C01D0D8450CD3BBF10B0F01D0BF
:10CD90002E2C02D00620BDE8FC9F4FF008084FF073
:10CDA0000B0BD8E7812C01DB9F2C03DDE02C1CDB77
:10CDB000FC2C1ADC38467F1C19F80060402E01DB81
:10CDC0007E2E03DD802E05DBFC2E03DCABF10100A3
:10CDD000404501D80620DEE7404608F101082C5402
:10CDE000404608F101082E5411E0214614A0FFF737
:10CDF00059FD08B10620CEE7612C04DB7A2C02DC59
:10CE0000A4F12000C4B2404608F101082C54A2E766
:10CE100000BF09EB0700CAF80000B8F1000F01D10C
:10CE20000620B8E72878E52801D105202870202CB5
:10CE300001DC042000E00020E8720020ABE70000E5
:10CE4000222A2B2C3A3B3C3D3E3F5B5D7C7F000021
:10CE50002DE9FF4105460C4629492A4A891AC90885
:10CE6000042242EA01402B46224627A103F038FD66
:10CE7000002002900390ADF80840ADF80A40009001
:10CE800001906A4602A9284690DF0646002E32D05D
:10CE9000304604F05FFB074619491A4A891AC90847
:10CEA000012242EA01403B462A46234903F018FD8D
:10CEB000BDF8000010B9BDF8020068B1BDF802303D
:10CEC000BDF800200E490F4FC91BC908012747EACA
:10CED00001401AA103F004FDBDF8040058B1BDF8EB
:10CEE00004200749074BC91AC908012343EA014036
:10CEF000224903F0E9FC304604B0BDE8F0810000AF
:10CF0000CC7C0300CC7C03005570646174696E674F
:10CF10002064617461206C656E67746820746F2092
:10CF20002575206F6E20636F6E6E656374696F6E1A
:10CF300020307825782E00009C730300546865200B
:10CF40007265717565737465642054582F5258204A
:10CF50007061636B6574206C656E677468206973BB
:10CF600020746F6F206C6F6E672062792025752F9B
:10CF70002575206F63746574732E0000E8730300D9
:10CF800020BF704701207047012070470120704783
:10CF90000120704770B5044603A50E22294620469D
:10CFA000FAF7A4FA70BD00004D3130303130303026
:10CFB000303030303032000010B50248FFF7EAFF61
:10CFC000004810BDA49500202DE9F04104460E460E
:10CFD000D4F800800021204600F000F90546EDB9A4
:10CFE000002700BF4046A16902F0F8F9054605B1E7
:10CFF00013E0E0690078E52802D0E069007820B904
:10D00000781C0746B04201D107E0002701212046E5
:10D0100000F040F80546002DE4D000BF042D00D1FB
:10D0200007252846BDE8F0812DE9F0410446276830
:10D030000021204600F0D2F8054615B12846BDE88B
:10D04000F08100BF3846A16902F0C8F9054605B174
:10D050001DE0E06906780EB9042518E0E069C07AA1
:10D0600000F03F00A071E069C07A00F0080038B914
:10D070000B2204F12001E06902F007F900B906E093
:10D080000021204600F006F80546002DDAD000BF4A
:10D090002846D4E72DE9F0470446894625682069EB
:10D0A00000F12007A06910B1B7F5001F02D30420DA
:10D0B000BDE8F087C7F30800002868D1A069401CCC
:10D0C000A061606938B92889B0EB571F5FD800208C
:10D0D000A0610420ECE76889401E00EA5720002880
:10D0E00055D12046616901F095FB0646012E01D815
:10D0F0000220DDE7701C08B90120D9E76869B04259
:10D100003FD8B9F1000F03D10020A0610420CFE780
:10D1100020466169FFF79CFD06460EB90720C7E768
:10D12000012E01D10220C3E7701C08B90120BFE71E
:10D13000284608F083FA08B10120B9E74FF40072DD
:10D14000002105F1300002F0BFF84FF00008314631
:10D150002846FFF7DDFBE8620CE00120E870284676
:10D1600008F06CFA08B10120A2E708F10108E86AAA
:10D17000401CE86268894045EFD8E86AA0EB0800E7
:10D18000E862666131462846FFF7C2FBA06127616D
:10D19000C7F3080105F130000844E061002087E78B
:10D1A00070B50446266801212046FFF70DFF0546AD
:10D1B00095B93046A16902F011F9054665B92022FA
:10D1C0000021E06902F080F80B2204F12001E069FF
:10D1D00002F06DF80120F070284670BD2DE9F04195
:10D1E00004460D462668B5F5001F02D205F01F0063
:10D1F00010B10220BDE8F0812561A7681FB9307821
:10D20000032800DB776A47B93089B0EB551F01D896
:10D210000220EFE7706AA0611CE070894FEA4028A5
:10D2200011E03946204601F0F5FA0746781C08B9A6
:10D230000120DFE7022F02D37069B84201D8022033
:10D24000D8E7A5EB08054545EBD239463046FFF750
:10D250005FFBA0616761A06908B90220CAE7A06905
:10D2600000EB5520A061C5F3080106F13000084429
:10D27000E0610020BEE7000070B504460E461321B1
:10D28000204676DF054665B10C490D4A891AC90862
:10D29000022242EA01402B4622460A4903F020FBC3
:10D2A0000AE00649064A891AC908042242EA0140EE
:10D2B000224605A103F008FB70BD0000647D030059
:10D2C000CC7C0300B87A0300446973636F6E6E65AB
:10D2D0006374656420636F6E6E656374696F6E203E
:10D2E00068616E646C652025640000002DE9F041E2
:10D2F00004463E480078844202DB0320BDE8F0810A
:10D3000004EB44003A49096851F8200008B90320A9
:10D31000F4E704EB44003649096801EB8000407AE9
:10D3200000F0010038B904EB44003149096801EB11
:10D330008000407AE2E704EB44002D49096801EBE4
:10D340008000406838B92B4804EB4401284A126831
:10D3500002EB81014860012004EB4401244A126879
:10D3600002EB8101887204EB44002149096851F8FD
:10D370002060214F3068224639460368304698477E
:10D38000054600BF4DBB07E004EB4401184A126894
:10D3900002EB81014868804704EB440014490968A6
:10D3A00001EB8000807A0028EED104EB44001049A4
:10D3B000096801EB8000007A78B904EB44000C495D
:10D3C000096801EB8000407A20F0010004EB440181
:10D3D000074A126802EB8101487204EB44000449D9
:10D3E000096801EB8000407A88E70000502F002098
:10D3F0004C2F002081CF0200D9C10200F8B50446AD
:10D400000E4615462A480078844201DB0420F8BD08
:10D4100026B1012E1BD0022E45D12EE00120009016
:10D4200000BF04EB4401234A126852F821006A4607
:10D43000002102F0E8FA074617B1112F00D003E0EF
:10D440009DF800000028ECD100BF0020DFE704EBCE
:10D4500044001849096851F8200008B90320D6E7AC
:10D460002F4604EB4401134A126852F8210002F0DF
:10D47000C3FA006838600020C9E704EB44000D4996
:10D48000096851F8200008B90320C0E72F4604EBD3
:10D490004401084A126852F8210002F0ADFA80886F
:10D4A00038800020B3E700BF00BF0120AFE70000D5
:10D4B000502F00204C2F00202DE9FE4F04468846B7
:10D4C00091461E462F480078844200DA16B904209F
:10D4D000BDE8FE8F04EB44002B49096851F8200099
:10D4E00048B104EB44002849096801EB8000407A08
:10D4F00000F0010008B10320EAE7CDF800900196A2
:10D50000CDF80880012004EB44011F4A126802EBA9
:10D510008101887204EB44001B49096851F82050CE
:10D520006F462868416928468847006839688842FC
:10D5300001D8072004E028683946826828469047C9
:10D540008246BAF1000F1BD107E004EB44010E4AFA
:10D55000126802EB81014868804704EB44000A49E5
:10D56000096801EB8000807A0028EED104EB4400CA
:10D570000549096801EB8000007A08B90020A7E797
:10D580000120A5E7502F00204C2F0020014607481E
:10D590000078814201DB0120704701EB4100044A21
:10D5A000126802EB8000407AF6E70000502F00205E
:10D5B0004C2F002070B5044636480078844201DBC9
:10D5C000032070BD04EB44003349096851F8200082
:10D5D00008B90320F5E704EB44002F49096801EB83
:10D5E0008000407A00F0010038B104EB44002A4981
:10D5F000096801EB8000407AE3E704EB4401264A26
:10D60000126852F821000022114602F0FCF900BF16
:10D6100004EB44002049096851F8206030684168F3
:10D6200030468847054600BF112DF1D08DB907E07F
:10D6300004EB4401184A126802EB810148688047F4
:10D6400004EB44001449096801EB8000807A00284B
:10D65000EED104EB44001049096801EB8000007A28
:10D6600078B904EB44000C49096801EB8000407A6A
:10D6700040F0010004EB4401074A126802EB81010B
:10D68000487204EB44000449096801EB8000407AC9
:10D6900097E70000502F00204C2F00202DE9FE4F6F
:10D6A0000446884691461E4635480078844200DA92
:10D6B00016B90420BDE8FE8F04EB44003149096827
:10D6C00051F8200048B104EB44002E49096801EBF1
:10D6D0008000407A00F0010008B10320EAE704EB83
:10D6E00044002849096801EB8000407A00F00400FA
:10D6F00008B10220DEE7CDF800900196CDF8088051
:10D70000012104EB44001F4A126802EB8000817281
:10D7100004EB44001B49096851F820506F46286803
:10D7200041692846884700683968884201D807203F
:10D7300004E028683946C268284690478246BAF114
:10D74000000F1BD107E004EB44010E4A126802EB04
:10D7500081014868804704EB44000A49096801EBED
:10D760008000807A0028EED104EB44000549096866
:10D7700001EB8000007A08B900209BE7012099E7BF
:10D78000502F00204C2F0020024A1060024B1970CD
:10D79000704700004C2F0020502F002010B50021B2
:10D7A000034801F0D1FF044684F3100010BD0000CF
:10D7B000A48C002070B505460C464FF4803000FA6A
:10D7C00004F1284600F0F2F970BD70B505460C462C
:10D7D0004FF4A07000EB840086B23146284600F07A
:10D7E000FFF970BD2DE9F04704460D4616461F4669
:10D7F0004FF4803000FA05F84FF4A07000EB85007C
:10D800001FFA80F926F07F464146206803F065FB49
:10D810004146206803F052FB4946206803F044FB70
:10D8200032462946206803F02FFB4146206803F06A
:10D830004BFB1FB14146206803F055FBBDE8F08764
:10D8400010B50446206803F024FB10BD2DE9F04715
:10D8500004460D4617466079324941F820706079D8
:10D86000314901EBC000007968B108262F49304AE0
:10D87000891AC908022242EA01402EA103F01AF8CF
:10D880003046BDE8F08729882068C0F8081500BF39
:10D8900094F90420AB7810461946002808DB4FEABB
:10D8A000417C4FEA1C68DFF8B0C00CF800800BE048
:10D8B0004FEA417C4FEA1C69DFF8A0C000F00F0876
:10D8C000A8F104080CF8089000BF00BF94F90410F8
:10D8D000084600280DDB00BF00BF00F01F03012237
:10D8E0009A4043099B0003F1E023C3F8002100BFE5
:10D8F00000BF00BF00BF012061790B4A02EBC101EC
:10D9000008716079114641F8304000260749084AFD
:10D91000891AC908032242EA014011A102F0CAFF94
:10D920003046AEE7B42E0020B82E00204C7D030018
:10D93000CC7C030052544320696E7374616E63653E
:10D9400020616C726561647920696E697469616CCB
:10D95000697A65642E00000000E400E018ED00E044
:10D960005254433A20696E697469616C697A6564DE
:10D970002E00000010B5014691F90400002807DBD5
:10D9800000F01F0301229A40024B440943F824206F
:10D9900000BF10BD00E200E070B505460C4622460F
:10D9A0000221284600F00EF970BD10B504464FF470
:10D9B0008271204600F014F910BD10B50446002114
:10D9C000206803F09BFA10BD10B5044604212068BE
:10D9D00003F094FA10BD2DE9F84F04468846154629
:10D9E00099464FF4803000FA08FA4FF4A07000EB2B
:10D9F00088001FFA80FB25F07F455146204600F045
:10DA0000D5F8206803F045FA06464146206803F041
:10DA100035FA009032464146206803F035FA5946FF
:10DA2000206803F041FA3146009807F030FE0128E3
:10DA300006D1102003F02AFE5946206803F034FA7C
:10DA4000206803F026FA06463146284607F01FFEF6
:10DA500007465146206803F037FA012F0FD16A1CA0
:10DA60004146206803F010FA102003F00FFE2068F2
:10DA700003F00FFAB04225D00D20BDE8F88F2A46FA
:10DA80004146206803F000FA206803F002FA0646D7
:10DA9000681E314607F0FBFD07466FF07F40A0EBA4
:10DAA0000900B84201D20D20E7E75FB96A1C414680
:10DAB000206803F0E9F9206803F0EBF9B04201D0E7
:10DAC0000D20DAE701225146204600F07BF80020C5
:10DAD000D3E70000014621B1012904D0022906D173
:10DAE00003E004A0704705A0FCE706A0FAE708A041
:10DAF000F8E700007374616E6462790072656164B6
:10DB00007900000073616D706C696E670000000041
:10DB1000756E6B6E6F776E0010B504460549064A48
:10DB2000891AC908042242EA0140224603A102F0F0
:10DB3000CBFE10BD647D0300CC7C030044756D6D8D
:10DB400079206576656E742068616E646C657220FC
:10DB50007265636569766564206576656E742030EC
:10DB60007825780010B510480068407E60B1062125
:10DB70000120FDF7FDFF044624B10B480068416910
:10DB800003208847002010BD012007490968087656
:10DB900001210846FDF7ECFF04461CB100200249B4
:10DBA000096808762046EEE75C2F002070B5044631
:10DBB0000D462946206803F081F92946206803F0C4
:10DBC0008CF970BD70B504460E4615463146206886
:10DBD00003F07AF91DB13146206803F084F970BD75
:10DBE00070B505460C462868015929B121462868B8
:10DBF00003F05AF9012070BD0020FCE738B5054656
:10DC0000284600F047FA04463CB96946284608F021
:10DC10004AFA04460CB900202860204638BD2DE998
:10DC2000FC4707468846914600243E4613E06B4673
:10DC3000012201A9484600F040F90098012800D0CF
:10DC40000DE09DF8045000BF06F8015B641C0A2D2E
:10DC500000D104E000BFA8F10100A042E7DC00BF52
:10DC60000020307014B13846BDE8FC870020FBE787
:10DC7000F7B582B016460398019001A800F0A2FE05
:10DC80000546002D02DA0B2005B0F0BD0E4850F815
:10DC900025400CB100202070029810B1002002999C
:10DCA00008700949029841F82500029808B1012E30
:10DCB00001D00020E8E7002202A903A800F02AFB17
:10DCC00007463846E0E70000542F00202DE9F74FC3
:10DCD0008EB0044616461CB9092011B0BDE8F08F7D
:10DCE00006F03F06324602A90FA800F013FB0546D6
:10DCF000002D70D10298039003A80F9900F0DDFC6D
:10DD000005462DB99DF8370000F0800000B10625CA
:10DD100006F01C00002856D045B1042D03D103A8FD
:10DD2000FFF73EFA054646F008060AE09DF81200A5
:10DD300000F0110008B1072503E006F0040000B16F
:10DD40000825002D51D106F0080000284DD000F024
:10DD5000D1FD01900A9901F10E00019907F022FB13
:10DD60000A9901F11600019907F01CFB20200A997D
:10DD7000C8720A99029801F05FF9814600220A9957
:10DD8000029807F0FDFA0A9901F11C00002107F042
:10DD900009FB01200299C870B9F1000F25D0029843
:10DDA000C06A01900022494603A805F019FD054606
:10DDB000DDB9DDE9011001F011FB0546A9F1010013
:10DDC0000299C86011E085B99DF8120000F01000BA
:10DDD00010B1042509E05DE006F0020028B19DF8CD
:10DDE000120000F0010000B107254DB906F008004F
:10DDF00008B146F040060298C06A20620A98606244
:10DE0000002D55D10A99029801F016F9A0600A99DF
:10DE100001F11C0001F023F9E060029820600298F3
:10DE2000C088A080267400206074E06160614FF4B7
:10DE30000072002104F1280001F046FA06F02000EB
:10DE400040B3E06830B3E0686061029840894FEA0F
:10DE5000402AA768D4F80C800CE03946204600F030
:10DE6000D9FC0746012F00D80225781C00B90125EE
:10DE7000A8EB0A080DB9D045EFD8A76155B9C8F38A
:10DE8000080038B139460298FEF742FDB0F1000BA8
:10DE900001D102250CE00BEB5820E061E269029908
:10DEA0004878012304F12801FFF706FB00B10125A2
:10DEB0000DB10020206028460FE72DE9FF4F85B007
:10DEC000044615469A46DDF818B00020CAF800004E
:10DED00003A9204608F0E7F80490049810B9607C84
:10DEE000049018B1049809B0BDE8F08F207C00F0D0
:10DEF000010008B90720F6E76169E068401A01905F
:10DF00000198854200D9019DA0E0A08AC0F30800D5
:10DF100000287ED103984089401E616900EA51299A
:10DF2000B9F1000F17D1606910B9A068029004E040
:10DF30002046A16900F06EFC02900298022802D2ED
:10DF400002206074CFE70298401C10B90120607471
:10DF5000C9E70298A061A1690398FEF7D9FC0646BB
:10DF600016B902206074BEE74E444FEA5528B8F156
:10DF7000000F29D009EB080003994989884203D989
:10DF800003984089A0EB0908039948784346324634
:10DF90005946FFF791FA10B101206074A3E7207C85
:10DFA00000F0800068B1E069801B404509D2E1695A
:10DFB000891B0BEB41204FF4007204F1280101F0A2
:10DFC00076F94FEA482737E0E069B04220D0207C5C
:10DFD00000F0800078B1E26903994878012304F1E8
:10DFE0002801FFF75BFB10B1012060747BE7207C08
:10DFF00000F07F002074039948780123324604F131
:10E000002801FFF759FA18B1012060746BE700E0AE
:10E01000E661A08AC0F30800C0F50077AF4200D9DE
:10E020002F46A08AC0F3080204F1280011183A46CE
:10E03000584601F03CF900BFBB4460693844606158
:10E04000DAF800003844CAF80000ED1B002D7FF418
:10E050005CAF002047E733B58BB00D460022694620
:10E060000BA800F057F904468CB968460B9900F0EC
:10E0700024FB04465CB99DF82B0000F0800008B139
:10E08000062404E01DB12946684600F055FC2046F0
:10E090000DB030BDF8B504466946204608F003F8D7
:10E0A0000646002E44D1207C00F0400000283FD0DE
:10E0B000207C00F0800070B1E2690099487801236B
:10E0C00004F12801FFF7EAFA08B10120F8BD207C2D
:10E0D00000F07F00207400F00DFC0746216A0098D4
:10E0E00001F07CF906461EBB656AE87A40F0200024
:10E0F000E8722946A268206807F042F905F11C0081
:10E10000E16807F04FF9394605F1160007F04AF9C2
:10E11000002105F1120007F051F901200099C870A3
:10E12000009807F043FA0646207C00F0BF002074F8
:10E130003046CBE72DE9FF4F83B0044615469B469A
:10E14000049800900020CBF8000001A9204607F0B9
:10E15000AAFF0290029810B9607C029018B1029850
:10E1600007B0BDE8F08F207C00F0020008B907205E
:10E17000F6E700BF606928446169884202D260699D
:10E18000C0F1FF35BBE0A08AC0F30800002875D1BC
:10E1900001984089401E616900EA512ABAF1000FD6
:10E1A0001ED1606938B9A76857B900212046FEF72B
:10E1B0004FFD074604E02046A169FEF749FD0746EA
:10E1C00007B99FE0012F02D102206074C8E7781CD4
:10E1D00010B901206074C3E7A761A06800B9A76007
:10E1E000207C00F0800078B1E26901994878012331
:10E1F00004F12801FFF752FA10B101206074AFE773
:10E20000207C00F07F002074A1690198FEF780FB5C
:10E21000064616B902206074A2E756444FEA552913
:10E22000B9F1000F2BD00AEB090001994989884206
:10E2300003D901984089A0EB0A09019948784B4617
:10E2400032460099FFF72AFA10B10120607487E77F
:10E25000E069801B48450ED2E069801B009A02EB02
:10E2600040214FF4007204F1280001F020F8207CD6
:10E2700000F07F0020744FEA49282BE013E0E069AA
:10E28000B0420FD0E168606988420BD201994878AA
:10E290000123324604F12801FFF70EF910B10120E5
:10E2A00060745DE7E661A08AC0F30800C0F50078FD
:10E2B000A84500D9A846A18AC1F3080204F12801A3
:10E2C00050184246009900F0F2FF207C40F0800098
:10E2D000207400BF00984044009060694044606131
:10E2E000E1686069884201D9606900E0E068E06047
:10E2F000DBF800004044CBF80000A5EB0805002D3A
:10E300007FF441AF00BF207C40F04000207400202B
:10E3100026E700002DE9F74F8AB000210B98016035
:10E320000A9800F04FFB08900898002803DA0B20A9
:10E330000DB0BDE8F08FB149089851F820400CB9F4
:10E340000C20F5E70B9804600C9800F0FE000C9090
:10E35000207878B16078FFF719F9814609F001005B
:10E3600040B90C9820B109F0040008B10A20DFE799
:10E370000020DDE700202070089860706078FEF7CC
:10E38000B5FF814609F0010008B10320D0E70C98E1
:10E3900020B109F0040008B10A20C9E70027394676
:10E3A0002046FEF741FA0546022D01D02EDA2DE077
:10E3B000002614E04FF4DF7000EB061104F130008A
:10E3C000084409900998007920B10998083000F0B4
:10E3D00046FE00E0002002A941F82600761C042E2B
:10E3E000E8D3002606B1761E00BF02A850F82670BA
:10E3F00027B139462046FEF717FA00E0032005460C
:10E40000022D03DB701C06460428EED3042D01D137
:10E4100001208DE7022D01DB0D2089E704F13B008F
:10E4200000F029FEB0F5007F01D00D2080E704F157
:10E43000460000F020FE8046B8F1000F04D104F140
:10E44000540000F00CFE8046C4F818804020005DA7
:10E45000A070A078012804D0A078022801D00D2057
:10E4600066E7A07808FB00F83D20005D60816089C8
:10E4700018B16089411E084008B10D2058E704F129
:10E48000410000F0F8FD2081207A00F00F0008B173
:10E490000D204DE704F1430000F0EDFD8246BAF196
:10E4A000000F04D104F1500000F0D9FD824604F1C0
:10E4B0003E0000F0E0FD0190019808B90D2037E71B
:10E4C00001984044218900EB11100790079882457C
:10E4D00001D20D202CE70798AAEB00006189B0FB60
:10E4E000F1FBBBF1000F01D10D2021E703254FF611
:10E4F000F570834500D8022540F6F570834500D8B5
:10E5000001250BF102006061E76101983844206247
:10E5100007983844A062032D13D104F15A0000F08B
:10E52000AAFD08B10D2003E7208908B10D20FFE600
:10E5300004F15C0000F093FD606260698000069069
:10E5400014E0208908B90D20F2E6206A4044606298
:10E55000022D02D16069400007E0207D00F001003B
:10E56000616901EB410100EB51000690A169069839
:10E5700000F2FF10B1EB502F01D20D20D8E64FF082
:10E58000FF302061E06080202071032D2CD104F148
:10E59000600000F070FD012826D1791C204600F0B3
:10E5A0001DFF08BB0020207104F22E2000F063FD47
:10E5B0004AF65521884217D104F1300000F04FFD92
:10E5C0000F49884210D104F5057000F048FD0D494F
:10E5D000884209D104F5067000F041FD206104F580
:10E5E000077000F03CFDE060257007480088401C83
:10E5F00080B205490880E080002099E6542F002071
:10E600005252614172724161582F002010B5044688
:10E61000E07FFF2808D0A07F18B1E07F01F071FDF6
:10E6200002E0E07F01F0F7FD00206077207204F146
:10E630000800D4E90021904710BD70B505460E468C
:10E64000144624B13146284601F040F803E0314633
:10E65000284601F01DF870BD30B504461088C01C76
:10E66000984201D90C2030BD0220158848551088E9
:10E67000401C10800120158848551088401C1080CF
:10E6800015884C551088401C10800020EBE770B5B1
:10E6900004460D4640F21442115B0122D4F81004E6
:10E6A000FCF770FE064606B1357004F13C0204F535
:10E6B000826104F1540072DF70BD2DE9F34104461C
:10E6C0002646D6F8008002E00198401C019001988F
:10E6D00000782F28F8D0019800785C28F4D000202A
:10E6E000B06001980078202808D280212B200155A5
:10E6F00000212046FEF772FD05462CE000BF01A96F
:10E700002046FEF715FB054605B123E02046FEF73F
:10E710008BFC05462B20075D3DB1042D04D100BFC5
:10E7200007F0040000B9052514E007F0040000B16B
:10E7300010E0B07900F0100008B905250AE0208A41
:10E74000C0F3080208F130001118404600F074FCD4
:10E75000B060D4E700BF2846BDE8FC81F7B50D46A0
:10E7600017460DB90020FEBD0026009868B10024B0
:10E7700009E02146684600F09AFF18B1A0B2394678
:10E78000A847761C641C142CF3D33046EBE700003A
:10E7900070B505460C4660880C490988884214D13A
:10E7A000208840F6772188420FD1A088C01E0849F2
:10E7B00008802B886A880749074E891BC9080426E8
:10E7C00046EA014005A102F08BF870BD3C2F002005
:10E7D0003E2F0020647D0300CC7C03004154542074
:10E7E0004D54552065786368616E676520636F6D71
:10E7F000706C657465642E2063656E7472616C2044
:10E800002564207065726970686572616C2025648A
:10E81000000000002DE9F04781460C46D9F8005071
:10E82000022C02D36869A04202D84FF001085EE0D2
:10E830004FF0FF382878012804D002282CD0032874
:10E8400051D13CE0264606EB5606286A00EB5621DD
:10E85000284600F0C3FD00B148E03046761CC0F306
:10E86000080105F13000475C286A00EB5621284674
:10E8700000F0B4FD00B139E0C6F3080105F1300045
:10E88000405C47EA002704F0010008B1380901E0C4
:10E89000C7F30B00804629E0286A00EB14212846C4
:10E8A00000F09CFD00B121E040F2FF1101EA4402BA
:10E8B00005F13001501800F0DEFB804616E0286AB2
:10E8C00000EBD411284600F089FD00B10EE040F2C3
:10E8D000FF1101EA840205F13001501800F0BFFB7E
:10E8E00020F0704802E04FF0010800BF00BF404632
:10E8F000BDE8F0871CB51F201D2117231A46CDE95E
:10E90000001001214FF4FD6000F001F81CBDF0B5CE
:10E910000446DDE905560020A4F2BC7740EA4760D2
:10E920004F1C40EA475040EA024040EAC32040EA18
:10E93000451040EA5600F0BD2DE9F04705460C466B
:10E9400000206072A86908B9BDE8F0870026374644
:10E950001CE03046761CEA6912F80090B9F1200FED
:10E9600000D113E0B9F1050F01D14FF0E509092EEF
:10E9700005D12E2238467F1C04F109010A5438467D
:10E980007F1C04F1090101F8009000BF0B2EE0D3B9
:10E99000002104F10900C155E869C07A2072E969D3
:10E9A00001F11C0000F05BFB2060E96901F1160039
:10E9B00000F055FB8046A4F806804FEA1840A0807E
:10E9C00000BFC1E770B502464FF0FF301568DDB1FA
:10E9D000116800E0491C0D78212D02D30D783A2DE5
:10E9E000F8D10D783A2D0ED1146814F8015BA5F119
:10E9F00030030A2B06D28C4204D11BB918464D1C99
:10EA00002946156070BD002000BFFBE770B50B48BC
:10EA1000FEF716FF0A4B0CCB841843F10005094999
:10EA200003C9201A75EB010004D24FF08073E4187B
:10EA300045F100052046294670BD0000902E0020BB
:10EA4000A02E0020A82E002001480078704700006A
:10EA5000742D00200148007870470000752D0020BB
:10EA60002DE9FE4F314903C9CDE90101304A01A921
:10EA7000304803F08FFB8346BBF1000F0AD02E49CC
:10EA80002E4A891AC908012242EA01405A462CA19D
:10EA900001F01AFF00BF00BF052526490868D0F81D
:10EAA0001015CEB200BF00964FF47A50A5FB009A25
:10EAB00048465146009AF8F7A6FC07463C4600BF78
:10EAC00000BF1D491D4A891AC908032242EA0140B4
:10EAD000224624A101F0F8FE00BF04F00100002846
:10EAE00018D024A01449154A891AC9080322009095
:10EAF00042EA014040F2A51324A22CA101F000FF3C
:10EB000001F0CCFC00BF002500BF0020FBF702FE97
:10EB100000BF00BF00BF6408012003462246002159
:10EB20000090044803F014FBBDE8FE8F506B030017
:10EB300045210300386B0300647D0300CC7C030097
:10EB40006E7266785F74696D65725F696E69742054
:10EB50006661696C656420776974683A2025640A87
:10EB60000000000074696D65725F7469636B733ACD
:10EB700025640A0074696D65725F7469636B732044
:10EB8000252032203D3D2030000000007372635C80
:10EB900068656172745F776176655F73616D706CD3
:10EBA000655F736572766963652E630025733A2528
:10EBB00064205A41535345525428257329206661D5
:10EBC000696C00000148007870470000642D002047
:10EBD00010B5FBF7A5F810BD10B500200B49087063
:10EBE00001200B49087000200A4908600A490860A2
:10EBF00000BF0A49086000BF0948FBF791FC0948BB
:10EC0000FBF78EFC084803F08BFA10BD762D002030
:10EC1000642D00205C2D0020602D0020702D002030
:10EC2000482D0020502D0020386B030010B50A48F5
:10EC300003F064FA0020094908700949086009498D
:10EC4000086000BF0849086000BF0848FBF772FC75
:10EC50000748FBF76FFC10BD386B0300642D0020E4
:10EC60005C2D0020602D0020702D0020482D0020FC
:10EC7000502D002010B5034803F040FAFBF764FC68
:10EC800010BD0000386B0300024600210CE001EBD0
:10EC90008100074B33F82000904204D101EB810042
:10ECA00003EB80007047491C0029F0D00020F9E7F1
:10ECB000286C00202DE9FC5F83460E4691461F46D6
:10ECC000DDE90C45002E01DA704200E03046824654
:10ECD0004FF0010803E09AFBF9FA08F10108CA4570
:10ECE000F9DA474500D9B84634B1002E03DB05F008
:10ECF0000400042800D1641E05F0020000B167B1D1
:10ED000005F0010048B944B104E0641E20215846D2
:10ED1000FDF758FC0CB1A045F7D3002E05DA76427A
:10ED20002D215846FDF74EFC07E005F004000428AD
:10ED300003D12B215846FDF745FC05F002000228BF
:10ED40000DD105F0010050B94FB944B104E0641E83
:10ED500030215846FDF736FC0CB1A045F7D33B46B1
:10ED60004A4631465846CDE9004507F065F8BDE80A
:10ED7000FC9F30B5024600201378C3F38003D3B163
:10ED8000137803F00303012B02D0022B10D107E00C
:10ED90001388C3F383139B1C0C6823440B6008E0A7
:10EDA0000B680225146805EB945423440B6000E0C3
:10EDB00000BF00BF012030BD70B505460C464FF4C2
:10EDC0008C71284602F092FB38B14FF48C712846C2
:10EDD00002F093FB2046FFF719FC70BD70B50546A5
:10EDE0000C464FF48871284601F079FF68B14FF462
:10EDF0008871284601F07AFF607900F0040020B1A4
:10EE0000206810B10120216888474FF48A71284694
:10EE100001F065FF68B14FF48A71284601F066FF82
:10EE2000607900F0080020B1206810B1022021684C
:10EE300088474FF48E71284601F051FF68B14FF4B6
:10EE40008E71284601F052FF607900F0100020B961
:10EE5000206810B10020216888474FF4827128464D
:10EE600001F03DFF58B14FF48271284601F03EFF9A
:10EE700001202071206810B103202168884770BDEF
:10EE80002DE9F04781460C4616464FF480374FF483
:10EE9000A078002520E03946484602F027F8A8B1BE
:10EEA0004146484602F013F880B13946484602F020
:10EEB00002F83946484602F00DF84146484601F04E
:10EEC000ECFFE8B21B4A52F8241088477F0008F193
:10EED00004001FFA80F86D1CB542DCD34FF4807833
:10EEE0000121484602F002F868B14146484601F067
:10EEF000EEFF40B14146484601F0CFFF0D4850F8C3
:10EF00002410042088474FF482780221484601F0FB
:10EF1000EDFF68B14146484601F0D9FF40B1414696
:10EF2000484601F0BAFF034850F8241005208847EE
:10EF3000BDE8F087782E00202DE9F04704460E4604
:10EF40009046002722E0384602F012FB054638467C
:10EF500002F015FB81462046294642580AB101229B
:10EF600000E0002282B14846D4F80413014009B100
:10EF7000012100E0002139B12946204602F004FBBE
:10EF80002846D6E900219047781CC7B24745DADB0E
:10EF9000BDE8F0872DE9F0410446A08800EB020CA3
:10EFA000B4F80480904501DD104600E0A088A8EB8D
:10EFB0000005E088C618B4F80680984501DD1846BB
:10EFC00000E0E088A8EB00074888B4F800804045DE
:10EFD00004DB4888B4F80280404502DD0020BDE82B
:10EFE000F0818888A84202D38888604501D9002032
:10EFF000F5E7C888B84202D3C888B04201D90020DA
:10F00000EDE70120EBE70146086808B102680A60F5
:10F01000704710B5044622460221002001F04AF84C
:10F02000002105E054F8210008B1012010BD491C61
:10F030000229F7D30020F9E770B505460C4604F124
:10F040001A0000F018F806462878032805D104F1C4
:10F05000140000F010F846EA0046304670BD014644
:10F06000C8788A7842EA00204A7842EA00200A7882
:10F0700042EA00207047014648780A7842EA0020B8
:10F080007047000010B502F0BBFA20B902F0DCFABC
:10F0900000200149887010BDD46C0020F721018048
:10F0A000172141800021017141711B218171C171C2
:10F0B000704770472DE9FF4100272E4800F01CFBE8
:10F0C0002C48001F00F018FB2B48806803902B4849
:10F0D00005680398284028490C3101EB800800BFDF
:10F0E00003A94046FFF745FE30B103982840224966
:10F0F0000C3101EB800800E000E0F1E700BF0024E4
:10F100000AE00398411C284003911B490C3151F837
:10F1100020004DF82400641C022CF2D3009800F06B
:10F12000030001280DD0022814D1BDF80670042177
:10F13000009801EB9050401E039901EB9000039062
:10F1400009E0BDF806700098C0F3831003990844E5
:10F15000039000E000BF00BF0648001F00F0C5FAA2
:10F16000064616B1044903988860384604B0BDE8E5
:10F17000F0810000A08C0020887C0020E82E002078
:10F1800070B500BF164A64213820FBF7BFFC044667
:10F1900000BF254625B100BF2846FBF7BBFA00BFDC
:10F1A00000BF00BF07F08AFB0E490F4A891AC90841
:10F1B000032242EA01400DA20FA101F085FBFDF7F9
:10F1C000FBFE1249086012484860084606F0BEFF80
:10F1D000F8F796FEF9F72EFC07F0F4FB002070BD5F
:10F1E00064310020647D0300CC7C030031323A306E
:10F1F000383A333400000000636F6D70696C65202D
:10F2000074696D65203A257300000000B82B00205A
:10F21000098002002DE9F04105460E461446984645
:10F22000A888871C2088801C3844404502D90C20BF
:10F23000BDE8F081FE2F01D90C20F9E7781C218868
:10F2400070542088401C2080FF2021887054208822
:10F25000401C208022889119288806F0E6FD21882C
:10F2600008442080A88800280DDDA86808B9072078
:10F27000DEE7AA8823889819A968F8F737F9208863
:10F28000A988084420800020D2E7F0B503461D4637
:10F290000C46002000BF15F8017B14F801CBA7EB4A
:10F2A0000C00561E321E01D00028F4D0F0BD30B53F
:10F2B00003460C463AB100BF14F8015B03F8015B4A
:10F2C000551E2A1EF8D130BD10B5034600BF03F805
:10F2D000011B541E221EFAD110BD2DE9FF4F87B02D
:10F2E000044691461E46A2462546BAF806009AF8FC
:10F2F00005104843001F0690BAF806B0301DB0FB59
:10F30000FBF00590301DB0FBFBF10BFB11000490EE
:10F31000D9F8000081190698814202D90698801B0D
:10F3200001E0D9F800000746C9F8007003E02D6835
:10F330000598401E059005980028F8D10390049880
:10F34000ABEB0008B84501D9384600E0404680469E
:10F3500023E00399089808440290281D0499084462
:10F360000190149828B14246DDE90110F8F7BEF883
:10F3700004E04246DDE90101F8F7B8F80020049006
:10F380002D68A7EB0807039840440390BB4501D9BB
:10F39000384600E05846804600BF002FD9D10BB058
:10F3A000BDE8F08F70B503460C469CB101F054FBEC
:10F3B000054600220AE0084800EB820108881E6822
:10F3C000B04202D11A60002070BD521CAA42F2D392
:10F3D0000520F9E70020F7E70000000070B50446BB
:10F3E0000D460026E06AA84210D0204606F026F915
:10F3F00006465EB9607801232A4604F13001FEF723
:10F400005BF810B14FF0FF350126E562304670BD64
:10F410002DE9F84F05460F461446984628780128EE
:10F4200004D1687810B90720BDE8F88F2088801CC7
:10F43000404508D82878012807D12088801C6978A1
:10F440000844404501D90C20EEE72088A8EB0000D5
:10F45000801E86B200962188891CC81969467DDF06
:10F46000814600BF484600B1DEE700BF2878022889
:10F4700004D06878BDF80010884206DBBDF80000B3
:10F48000B04202DC4FF0090A0BE04FF0080A28787E
:10F49000012805D16878B04202DC6878009000E06D
:10F4A0000096BDF80000FE2801D90C20BCE7BDF88D
:10F4B0000000401C218878542088401C208020882F
:10F4C00007F800A02088401C20802088BDF800108C
:10F4D000084420800020A7E70146044800888142B4
:10F4E00001DA481C00E00020C0B270478C2E0020DA
:10F4F000FEB504460D46002001900290CDF808D0DC
:10F500000220ADF804000020ADF8060001AA29464B
:10F510002046ADDF06462EB90298FCF746FE08B13C
:10F520000120FEBD0020FCE70B4802684FF0805030
:10F53000D0F834110D2A0DD121B1012904D00229AE
:10F5400006D103E0012070470120FCE70120FAE723
:10F550000120F8E70020F6E7300100100B480268B0
:10F560004FF08050D0F834110D2A0DD121B101296E
:10F5700004D0022906D103E0002070470020FCE7F8
:10F580000120FAE70120F8E70020F6E7300100103B
:10F590000B4802684FF08050D0F834110D2A0DD17D
:10F5A00021B1012904D0022906D103E001207047CE
:10F5B0000120FCE70120FAE70120F8E70020F6E748
:10F5C000300100100B4802684FF08050D0F8341121
:10F5D0000D2A0DD121B1012904D0022906D103E061
:10F5E000012070470120FCE70120FAE70120F8E73D
:10F5F0000020F6E73001001010B5044609B90E20CE
:10F6000010BD92FBF3F003FB102008B10920F7E7CF
:10F61000216000206060A060A281E38100BFEFE76D
:10F6200070B504460D4629462046F7F7F5FD18B19A
:10F630002A882168881870BD0020FCE770B505464F
:10F640000C4620886188884204D12846F7F726FEB8
:10F65000012070BD0020FCE770B504460D46294628
:10F660002046F7F7FEFD18B16A882168881870BD3A
:10F670000020FCE770B505460C462088618888426A
:10F6800004D12846F7F7E4FD012070BD0020FCE717
:10F6900070B505460C4604F01F0301229A40D14381
:10F6A000620905EB820000F039F8064670BD10B51E
:10F6B0000246480952F8200001F01F040123A3402C
:10F6C000184008B1012010BD0020FCE770B50546C8
:10F6D0000C4604F01F03012202FA03F1620905EB54
:10F6E000820000F03CF8064670BD10B504460021CB
:10F6F000204600F01EF810BD10B50446012120463A
:10F7000000F02DF810BDF8B504460D466A462946AE
:10F710002046F7F718FE06460098F8BDF8B50446EF
:10F720000D466A4629462046F7F7F3FD064600983F
:10F73000F8BDF8B504460D466A4629462046F7F757
:10F74000E8FD06463046F8BDF8B504460D466A4663
:10F7500029462046F7F7C4FD06463046F8BDF8B501
:10F7600004460D466A4629462046F7F7C5FD06467B
:10F770000098F8BDF8B504460D466A46294620466D
:10F78000F7F7EEFD06460098F8BDF8B504460026EA
:10F79000002000906846FBF751FC20680068616813
:10F7A000884215D920680068401E226810600178E0
:10F7B000204600F033F80646207A21680978401A7E
:10F7C000C5B220680079A84201DA2068057100BF3F
:10F7D0009DF80000FBF738FC3046F8BD0246D068C3
:10F7E000081A138AB0FBF3F0C0B27047F8B50446AC
:10F7F0000D462E46002000906846FBF71FFC314660
:10F800002046FFF7EBFF21680A68511C2368196046
:10F8100010709DF80000FBF717FCF8BD0246138A34
:10F82000D06801FB0300704710B5014600BF09B95D
:10F830000E2010BD00BF087A0B79C01AC2B2D1E900
:10F840000030186005E008680368581C0C682060E8
:10F850001A70101EA2F10103DAB2F4D10B6818710C
:10F8600000BFE6E730B502460B46D40802F00702B7
:10F87000012090401D5D284030BD024600BF0AB9FE
:10F880000E20704700BF172901DBF72901DD072093
:10F89000F7E711800020F4E770B504460E4600BF7C
:10F8A0000CB90E2070BD00BF2661F720208060805B
:10F8B0001B202071002505E0A11D01EBC500FFF70D
:10F8C000EDFB6D1C002DF7D00020EBE72DE9F04794
:10F8D000064688464546B488012C01DBBDE8F08722
:10F8E0003088242820D006DC102809D011280CD01C
:10F8F000232823D11DE03A280CD055281ED10EE034
:10F900003146284602F0ACFD19E03146284602F0A7
:10F91000B4FF14E03146284603F078F80FE0314692
:10F92000284602F0B5FF0AE03146284602F074FE90
:10F9300005E03146284602F017FF00E000BF00BF97
:10F94000A81D00EBC400007970B3A81D30F8341076
:10F950002046A5DF0746C7B90021A81D00EBC4005B
:10F9600001710121A81D00EBC4004171A91D31F8EE
:10F9700034201149114BC91AC908042343EA014034
:10F9800023460F4900F0ACFF12E0112F10D038468B
:10F9900001F0E0FD81460849084A891AC908012298
:10F9A00042EA01404A4600E003E006A100F08CFF75
:10F9B00000BF00BF92E70000CC7C0300CC7C0300BA
:10F9C0005473030073645F626C655F676174746392
:10F9D0005F65786368616E67655F6D74755F72659A
:10F9E000717565737428292072657475726E65640B
:10F9F0002025732E0000000010B5044620684169E0
:10FA00002046884710BD70B504460D46164620684E
:10FA10003246294603692046984770BD01464FF09B
:10FA20008040405808B1012070470020FCE708B52D
:10FA300000224FF080410A500958009100BF08BDD4
:10FA40000149086070470000080300400122910747
:10FA50000A5070472DE9F04104460CB9BDE8F08129
:10FA600000BF4FF47A7505B904E0054FAE0130468A
:10FA7000B84700BF601E041EF3D100BFEEE70000D0
:10FA8000C16B030070B540F6F8700068401C18B9EF
:10FA90004FF01020406902E040F6F870006805461B
:10FAA000681C00281CD01449144A891AC90803226A
:10FAB00042EA01402A4612A100F006FF284613DF61
:10FAC00004465CB10C490D4A891AC908012242EA70
:10FAD000014016A100F0EEFE204670BD0020FCE7BC
:10FAE0000549064A891AC908012242EA01401CA1B7
:10FAF00000F0E0FE0420F0E7647D0300CC7C03000E
:10FB000053657474696E6720766563746F722074D0
:10FB100061626C6520746F20626F6F746C6F6164DA
:10FB200065723A2030782530387800004661696C7B
:10FB300065642072756E6E696E672073645F736FA3
:10FB400066746465766963655F766563746F725F1A
:10FB50007461626C655F626173655F7365740000F8
:10FB60004E6F20626F6F746C6F6164657220776195
:10FB70007320666F756E640010B50E490E4A891ABF
:10FB8000C908032242EA01400C4A0DA100F09CFE84
:10FB90000A4813DF04465CB10649074A891AC908B6
:10FBA000012242EA014011A100F084FE204610BD6E
:10FBB0000020FCE7647D0300CC7C030000700200A1
:10FBC00053657474696E6720766563746F72207410
:10FBD00061626C6520746F206D61696E2061707068
:10FBE0003A20307825303878000000004661696C92
:10FBF00065642072756E6E696E672073645F736FE3
:10FC000066746465766963655F766563746F725F59
:10FC10007461626C655F626173655F736574000037
:10FC200010B500240F48007808B1852411E00020A9
:10FC30000C49886048600861C8600B4801F0F4FC1A
:10FC4000044601F0B1FB08B901F0E4FC01200549CC
:10FC5000087001F0D5FC10B10120024988702046DF
:10FC600010BD0000D46C0020E9C8020008B50020D7
:10FC700000906846FBF7E2F90748C068401E064955
:10FC8000C8600846C06808B9FFF7FCF99DF8000095
:10FC9000FBF7DAF908BD0000D46C00202DE9FF471E
:10FCA00005460C46164698462F781A4840F82760B5
:10FCB000194840F827804FF00009184B0FCB8DE80A
:10FCC0000F0020788DF8000060788DF80100A07892
:10FCD0008DF80200E0788DF8030020798DF805009A
:10FCE00060798DF80600A0680290207B8DF80C00EA
:10FCF000607B8DF80D000EB1094800E0002002463F
:10FD00003B466946281D02F051F88146484604B03A
:10FD1000BDE8F087C86D0020D86D0020106D03008D
:10FD2000315203002DE9FF4704460D4616461F4693
:10FD3000DDF830804FF00009009501960297CDF86C
:10FD40000C8000226946201D02F07EF9814648465B
:10FD500004B0BDE8F0872DE9FF4704460D4616467E
:10FD60001F46DDF830804FF000090095019602979C
:10FD7000CDF80C8000226946201D02F065F981460D
:10FD8000484604B0BDE8F0870FB438B5044605987E
:10FD900010B938BC5DF814FB0020009006A8009054
:10FDA0006A462046059900F012F80020009000BF36
:10FDB000EFE770B50446A06800B970BDD4E904034C
:10FDC000A268216898470020A06000BFF5E72DE9F0
:10FDD000FC5F82460D4614460DB9BDE8FC9F00BF8E
:10FDE0002E786D1C06B9E1E0252E70D100274FF06A
:10FDF000010900BF2E782B2E0CD02D2E02D0302ED4
:10FE00000CD103E047F001076D1C0AE047F0020740
:10FE10006D1C06E047F004076D1C02E04FF000097E
:10FE200000BF00BFB9F1000FE4D14FF0000800BFE0
:10FE30002A2E06D12168081D2060086880446D1CA8
:10FE40000DE02E78302E01DB392E00DD07E06D1C31
:10FE5000A6F1300008EB880100EB4108E8E700BF9D
:10FE60004FF0000B2E782E2E10D16D1C00BF2E7877
:10FE7000302E01DB392E00DD07E06D1CA6F13000CD
:10FE80000BEB8B0100EB410BF1E700BF2E7800BFBD
:10FE90006C2E01D0682E02D16D1C2E7800E000E09F
:10FEA000F6E700BF692E21D008DC252E6DD0582E34
:10FEB00039D0632E0CD0642E6CD116E0702E4CD04D
:10FEC000732E3ED0752E1FD0782E63D12AE065E0C8
:10FED0002168081D2060D1F8009009F0FF00019012
:10FEE00050460199FCF76EFB55E000BF2168081DE4
:10FEF0002060D1F800905B460A2249465046CDE981
:10FF00000087FEF7D7FE46E02168081D2060D1F883
:10FF100000905B460A2249465046CDE9008705F02D
:10FF20008BFF38E000BF2168081D2060D1F80090E9
:10FF30005B46102249465046CDE9008705F07CFF1C
:10FF400029E02168081D2060086801903B46424670
:10FF50005046019905F0F0FA1DE02168081D206067
:10FF6000D1F8009030215046FCF72CFB7821504608
:10FF7000FCF728FB002008210B461022CDE90010D9
:10FF80004946504605F058FF05E025215046FCF74C
:10FF900019FB00E000BF00BF6D1C03E03146504676
:10FFA000FCF710FB287800287FF41AAF00BF9AF8FE
:10FFB0000C0010B15046FFF7FCFE00BF0DE72DE925
:10FFC000FF470C4615461E46DDE90C78684600F0F2
:10FFD000E5F8814644EA450040EA860040EA072009
:10FFE00040EA084109F5E060009A40F82210BDE8B7
:10FFF000FF872DE9FF470C4615461E46DDE90C78C4
:020000040003F7
:10000000684600F0EBF8814644EA450040EA860085
:1000100040EA072040EA084109F5E060009A40F80C
:100020002210BDE8FF871CB504460020009003465F
:100030000122114601902046FFF7C1FF1CBD2DE9AA
:10004000F84F06460D4614460027B846B9460096B6
:10005000684600F083F8824647EA480040EA850097
:1000600040EA092040EA04410AF5E060009A40F8BD
:10007000221000BFBDE8F88F73B50D46684600F04A
:100080007DF8044604F5E060009950F8210020F462
:10009000403104F5E060009A40F82210009950F8D1
:1000A000210040EA054104F5E060009A40F8221082
:1000B0007CBD00003CB503460A4D30CDCDE900457E
:1000C00018460BE05DF82040D4F8204514605DF838
:1000D00020501468C5F82045121D401C5C1884424D
:1000E000F0D83CBDE06B030031B5684600F016F86F
:1000F00004460121009A01FA02F0C4F80C0500BF81
:1001000038BD31B5684600F049F804460121009A2F
:1001100001FA02F0C4F80C0500BF38BD01460868BA
:10012000202802D24FF0A0407047087800F01F004E
:1001300008600148F8E70000000300500146086825
:10014000202802D24FF0A0407047087800F01F002E
:1001500008600148F8E70000000300500146086805
:10016000202802D24FF0A0407047087800F01F000E
:1001700008600148F8E700000003005001460868E5
:10018000202802D24FF0A0407047087800F01F00EE
:1001900008600148F8E700000003005001460868C5
:1001A000202802D24FF0A0407047087800F01F00CE
:1001B00008600148F8E700000003005001460868A5
:1001C000202802D24FF0A0407047087800F01F00AE
:1001D00008600148F8E70000000300500146086885
:1001E000202802D24FF0A0407047087800F01F008E
:1001F00008600148F8E700000003005031B5684688
:10020000FFF78CFF04460121009A01FA02F0C4F8BE
:10021000080500BF38BD31B56846FFF7BFFF04468B
:100220000121009A01FA02F0C4F8080500BF38BDA8
:1002300031B56846FFF7D2FF04460121009A01FA62
:1002400002F0C4F8080500BF38BDF8B504460D46F5
:100250006DB900946846FFF781FF06460121009AB8
:1002600001FA02F0C6F80C0500BF00BF0DE00094D3
:100270006846FFF773FF06460121009A01FA02F073
:10028000C6F8080500BF00BF00BFF8BD0146014821
:10029000084470470060004038B504462046FFF728
:1002A000F5FF002101602046FFF7F0FF0068009095
:1002B00000BF38BD10B504462046FFF7E7FF0068D1
:1002C000012800D110BD0020FCE7000070B50446F5
:1002D0000E46FAF707FF0546681C08B9284670BDA8
:1002E000E8B2E168087100BF0A48006928B9094806
:1002F00004610020E168086009E006480069C06800
:100300000068E168086003480069C0680460284626
:10031000E5E70000888C0020704710B5F8F7F8FF7B
:1003200010BD704738B504460D4605484FF480634C
:10033000044A29460090204600F006F838BD000027
:10034000414B0300686F00202DE9F04F93B08246C7
:100350000E4617469846DDF87090304600F075FC62
:1003600018210DA8F7F7DBF80D97CDF83880CDF8F8
:10037000489000252B46082207A9304600F082FC51
:10038000082509980A90BDF82000ADF82C00BDF8AA
:100390002200ADF82E0000208DF83100079800F003
:1003A000030001281BD107984FEA902B0798C0F350
:1003B000C2008DF830000798C0F38314A2002B46CA
:1003C00001A9304600F05EFC05EB84050DA80AABE0
:1003D000224601A90090584600F076FB27E00798D6
:1003E00000F00300022822D107984FEA905B07989B
:1003F000C0F3C2008DF8300000BFBBF1080F01D27E
:10040000584600E0082004462B46224605A93046FF
:1004100000F038FC2544ABEB040B0DAB0AAA2146D7
:1004200005A800F097FABBF1000FE6D100BF3046F7
:1004300000F019FC13B0BDE8F08F000010B50246C3
:100440000B4C04EBC203012906D0022906D0032974
:1004500006D0042908D105E0022007E0042005E0C9
:10046000187903E0587901E0002000BF00BF10BDFB
:10047000CC7C030010B54FF0FF34FFF74EFF042192
:100480000548FFF723FF044600BF01200249C96861
:10049000487100BF10BD0000BC7C03002DE9F04F87
:1004A0008BB0FCF7A5F818B100200BB0BDE8F08FB9
:1004B0000021B548816100BF00BF00BFBFF34F8F6F
:1004C00000BF00BF00BFA0F5805080680A90AF4811
:1004D00004680A982040AE4901EB800A00250026F6
:1004E0000020069000BF0AA95046FEF742FCB0B1BA
:1004F000A548806998B9A6480C3840680A9988428E
:1005000007D8A3480C384068A1490C3988600020FE
:10051000CBE70A9820409E4901EB800A00E000E00A
:10052000E1E700BF00270AE00A98411C20400A9139
:10053000974951F8200007A941F827007F1C022F96
:10054000F2D3079800F0030002287AD10798800DB3
:1005500005904FF448710798B1EB905F02DD079862
:10056000800D01E04FF448708146079869F39F5071
:10057000079009F1080004900798C0F3C2000690A4
:100580008448049900F004FB0546002D57D0284606
:1005900000F05BFB3346082207A9284600F083FBE6
:1005A00008360A982040611C081A4FEA8008C145A5
:1005B00032D9B8F1000F05D00A982040744901EBF8
:1005C000800000E072480390B8F1000F01D040466F
:1005D00000E0484600F0FF0BB8F1000F01D06C4876
:1005E00000E000200290B8F1000F02D0A9EB080053
:1005F00000E00020C0B2019033465A4628460399D5
:1006000000F051FB5E44029828B133462846DDE9EC
:10061000012100F048FB0BE00A9820405C4901EB07
:10062000800B33464A465946284600F03CFB00BF43
:100630000598C01C0A9901EB90000A9000BF43E0A6
:10064000FFE7079800F0030001283DD10798C0F3A9
:100650008310062803DA0798C0F3831000E0062011
:10066000079960F3891107910798C0F3831000F18F
:1006700002080798C0F3C20006904FEA8801454877
:1006800000F086FA0546F5B1284600F0DEFA33465A
:10069000082207A9284600F006FB083600270DE0CF
:1006A0000A98421C20400A92394A02EB80013346E4
:1006B0000422284600F0F7FA361D7F1C0798C0F385
:1006C0008310B842ECD800BFDDB32F48D0F81080BB
:1006D000806918B1284600F0C6FA31E019E04FF001
:1006E000000900BFD8F80C004079012800D18146EC
:1006F000B9F1000F08D000BFD8F800002946026801
:100700004046904700BF00BFD8F80C00D0F80080EA
:1007100000BFB8F1000FE2D1284600F0A4FA002093
:10072000059005A8FAF78AFC1748806918B9184996
:100730000C390A9888609DF81400FAF785FC00BF10
:100740001DE0FFE71048D0F810800AE0C146D9F854
:10075000000081684846884700BFD8F80C00D0F8F0
:100760000080B8F1000FF1D10B490C4A891AC90871
:10077000022242EA01400AA100F09CF800BFFBF708
:1007800037FF80F0010090E6888C0020E82E0020E2
:10079000947C0020847D0300647D0300CC7C0300F6
:1007A0004261636B656E647320666C757368656423
:1007B000000000002DE9F74F82B0074615463B4880
:1007C0000668E91C8808002201A9FBF787FE0028BB
:1007D00051D0DDF804A00198801C019001983040B0
:1007E00032490968491C081A4FEA8008454509D86A
:1007F000019931402E4A02EB81002A460399F6F70F
:1008000075FE10E001993140294A02EB8100424611
:100810000399F6F76BFEA5EB0802039800EB0801BD
:100820002348F6F763FE4FEA174BFCF7B7FF814604
:100830004BEA09420AF1010030401D4941F82020ED
:100840000AEA060001EB8004206867F3C500206017
:100850000021206861F38F102060206865F39F50AD
:100860002060206820F00300801C2060206820F0B9
:100870000400206000BF0E480C38007880B10020D2
:1008800000906846FAF7DAFB00BF00BFFFF706FEEC
:100890000028FBD100BF9DF80000FAF7D5FB00BF90
:1008A000FEF707FC05B0BDE8F08F0000E82E002041
:1008B000947C002070B504460D4600231A46294654
:1008C000204604F0F5FD70BDF8B505460E46144609
:1008D000009401236A463146284604F0E9FDF8BD3C
:1008E0002DE9FC4106460F4614461D46009401952D
:1008F00002236A463946304604F0DAFDBDE8FC8141
:100900002DE9FE4306460F4614461D46DDF82880B5
:1009100000940195CDF8088003236A463946304695
:1009200004F0C6FDBDE8FE832DE9FF4706460F46ED
:1009300014461D46DDE90C8900940195CDF8088028
:10094000CDF80C9004236A463946304604F0B0FDD9
:10095000BDE8FF872DE9F05F07460E4690461D462D
:10096000082E01D9BDE8F09F95F80C90002028735F
:100970002946404602F042FA00240CE0B44205D277
:100980003A5D1DA12846FFF7FFF903E01CA12846A8
:10099000FFF7FAF9641C082CF0D31AA12846FFF7D8
:1009A000F3F900241DE0B44216D217F804A0BAF1FE
:1009B0007E0F09DCF6F738FD006810F80A0000F039
:1009C0003E0008B1504600E02E2083465A460EA154
:1009D0002846FFF7D9F903E00CA12846FFF7D4F920
:1009E000641C082CDFD301222946404602F0C4F9DA
:1009F00085F80C9000BFB5E7202530327800000064
:100A0000202020007C000000256300002000000062
:100A10002DE9F04106460F4600BF00200949087045
:100A2000094800F01AF9044614B12046BDE8F081E7
:100A3000064800F015FA06480649401AC508002085
:100A4000F4E70000887C0020847D0300586F0300D9
:100A5000847D0300CC7C030002480349401AC0088F
:100A600070470000847D0300CC7C030013B50C4666
:100A700021466846FEF796FC28B90448009A00EB28
:100A8000C20108681CBD0020FCE70000CC7C03000C
:100A900070B50B48046901200A4908700CE000BFDA
:100AA0000120E168487100BF254628684168284652
:100AB000884700BFE0680468002CF0D170BD0000DA
:100AC000888C0020887C00202DE9FF4707460C46D3
:100AD000164698460C9D95F80C90002028732946E0
:100AE000404602F08BF9072E47D2DFE806F00409F2
:100AF0000F161F2A370039462846FFF745F93DE013
:100B0000394628462268FFF73FF937E0394628463C
:100B1000D4E90023FFF738F930E0A06800903946A7
:100B20002846D4E90023FFF72FF927E0D4E9020192
:100B3000CDE9000139462846D4E90023FFF724F91E
:100B40001CE0D4E902122069CDE900120290394676
:100B50002846D4E90023FFF717F90FE0D4E9022370
:100B6000D4E90410CDE90023CDE902103946284626
:100B7000D4E90023FFF708F900E000BF00BF00221E
:100B80002946404602F0F8F885F80C90BDE8FF874A
:100B90002DE9F84F07468A46388AA0F104080AF181
:100BA00004004044401EB0FBF8F0C0B2009038464C
:100BB000FEF7EBFD044614B90020BDE8F88F0020D5
:100BC000207101216171A4F8068025460098A0F1EA
:100BD000010B2C462F604FF0000912E03846FEF75B
:100BE000D4FD064636B16079401C60712E603760D6
:100BF000354604E0204600F008F80020DDE709F162
:100C00000109D945EAD32046D7E72DE9F05F04462C
:100C1000274697F805802646A8F1010B002501E03C
:100C200036686D1C5D45FBD3D6F800A0264600252E
:100C300007E0D6F8009031465046FEF7D7FD4E4605
:100C40006D1C4545F5D3BDE8F09F70B504462546BB
:100C50000121281DFEF757FD70BD10B50446204642
:100C6000FEF7E2FD10BDF8B5044626460121301D11
:100C7000FEF780FD00906D46287810B92046FFF7FA
:100C8000C4FFF8BD2DE9FC4105460E4614461F463B
:100C9000019401203B4601AA314600902846FEF708
:100CA0001CFBBDE8FC812DE9FC4105460E461446BF
:100CB0001F46019400203B4601AA31460090284679
:100CC000FEF70BFBBDE8FC8100BF00BF00BFBFF318
:100CD0005F8F00BF00BF00BF002101607047024668
:100CE000505808B1012070470020FCE708B50022E9
:100CF00042504258009200BF08BDC0F80013704730
:100D0000C0F81415704710B5136800F5A46404EB1F
:100D10004114236000BF938800F5A46404EB4114E0
:100D2000636000BF936800F5A46404EB4114A36002
:100D300000BFD36800F5A46404EB4114E36000BF76
:100D400010BDC0F8001270470122425070470000E9
:100D500010B500200A49087000BF0A49086000BFAA
:100D600000BF00BF00BFBFF35F8F00BF00BF00BF69
:100D700000BF0549054800F04AFB002010BD0000F7
:100D8000C82E0020C42E0020706D0300006F0020CC
:100D900038B500BF002000906846FAF74FF900BF51
:100DA000F1EE100A044624F09F00E1EE100A00BFA5
:100DB00000BF00BF00BF00BFBFF35F8F00BF00BF19
:100DC00000BF2620002807DB00F01F020121914010
:100DD000094A430942F8231000BF9DF80000FAF7C2
:100DE00033F900BF00F0E0FA10B141DF044602E041
:100DF00020BF40BF20BF38BD80E200E070B5044690
:100E0000144D01212846FEF79FFC064600BF00BF97
:100E100000BF00BFBFF35F8F00BF00BF00BF0EB9B0
:100E2000012000E0002000B970BD042C0BD00A485E
:100E3000007818B10748FFF747FFF5E70748047047
:100E400001200549087004F01FF80248FFF73CFF35
:100E500000BFE9E7C42E0020C82E0020C02E0020CD
:100E600000218268916082681161826851618268A4
:100E7000D16082685160826811607047024602F555
:100E8000A86050F82100704700F5A86343F82120BE
:100E900070470146D1F80405704708B5002242505A
:100EA0004258009200BF08BD08B500224250425887
:100EB000009200BF08BDC0F848137047C0F848133F
:100EC0007047C0F844137047C0F844137047024697
:100ED00050587047C0F808137047C0F8081370479F
:100EE000C0F804137047C0F8041370470246D2F8E4
:100EF00004030840704701224250704701224250CB
:100F000070470000024A1060121D11607047000017
:100F10002C760040044B03EB00135A60024B03EBAA
:100F20000013196070470000107500400146034827
:100F3000085808B1012070470020FCE7007000400D
:100F400008B50021034A815011464158009100BF65
:100F500008BD0000007000400149086070470000B3
:100F600008730040014908607047000004730040A6
:100F70000121014A8150704700700040014609B9C3
:100F80000E2070470248006808600020F9E7000062
:100F9000E86F0300FEB506460C462046FFF7EEFF5D
:100FA00005460DB12846FEBD00200090019002903C
:100FB0008DF8006001208DF802000621ADF80410C4
:100FC00069462020226869DF054675B1284600F091
:100FD000C1FA07464F49504A891AC908012242EA14
:100FE00001403A464D49FFF76FFC00200090019008
:100FF000029001208DF8010000208DF802008DF88C
:10100000030069464020226869DF054675B128461D
:1010100000F0A0FA07463F493F4A891AC908012251
:1010200042EA01403A463E49FFF74EFC002000905C
:10103000019002908DF80060F720ADF8020069463B
:101040002320226869DF054675B1284600F082FA40
:1010500007463049304A891AC908012242EA01404C
:101060003A463049FFF730FC002000900190029092
:1010700002208DF8000069460120226869DF0546DC
:1010800075B1284600F066FA07462249224A891AB5
:10109000C908012242EA01403A462349FFF714FCFD
:1010A00000200090019002904FF4C86000906946C3
:1010B000A120226869DF054675B1284600F04AFA8A
:1010C00007461449144A891AC908012242EA014014
:1010D0003A461649FFF7F8FB002000900190029075
:1010E0008DF800006946A020226869DF054675B1C9
:1010F000284600F02FFA07460649074A891AC90808
:10110000012242EA01403A460949FFF7DDFB00208F
:1011100049E70000747D0300CC7C0300DC79030008
:10112000247A0300707A03003C7903008879030075
:10113000E87803002DE9F04104462568204660DF89
:1011400006462068A84225D91E491F4A891AC9089F
:10115000022242EA01401DA1FFF7ACFB19491A4ADD
:10116000891AC908022242EA01402A4623A12368BB
:10117000FFF7B6FB02F056FA2168471A1149124AE6
:10118000891AC908022242EA01403A4628A1FFF71B
:101190009BFB00E000BF1EB90120304908700EE043
:1011A000304600F0D7F907460649074A891AC908A8
:1011B000012242EA01403A4629A1FFF785FB304669
:1011C000BDE8F081747D0300CC7C0300496E73752B
:1011D0006666696369656E742052414D20616C6C6E
:1011E0006F636174656420666F7220746865205354
:1011F0006F66744465766963652E00004368616EAE
:101200006765207468652052414D20737461727463
:10121000206C6F636174696F6E2066726F6D203031
:1012200078257820746F20307825782E0000000013
:101230004D6178696D756D2052414D2073697A65F5
:1012400020666F72206170706C69636174696F6E83
:1012500020697320307825782E0000002F2F002081
:1012600073645F626C655F656E61626C65282920DE
:1012700072657475726E65642025732E000000001F
:101280002DE9F041ADF5027D80461848007818B987
:101290000DF5027DBDE8F0811DE04FF4FA70049079
:1012A00004A905A861DF044604B115E005AD1049A5
:1012B00001A800F0ACF809E000BF039806463768C3
:1012C00028467168B84701A800F0C2F800BF03982B
:1012D0000028F1D100BFE0E700BF052C04D000BF1B
:1012E0002046F9F717FA00BF00BFD1E72F2F0020E3
:1012F000DC6F03001CB51B48007808B108201CBD3A
:10130000012019490870002003F096FB112801D133
:101310000020F4E7002003F0ADFB144800680190C2
:10132000002000906846F9F789FE114901A810DFF6
:1013300004460CB9012000E000200A4908709DF81D
:101340000000F9F781FE0CB12046D8E700200649DD
:1013500008700849087003F00BFE012003F08AFBB7
:101360000020CCE72C2F00202E2F0020B86F030088
:1013700055A602002D2F00203EB50A49684600F010
:1013800046F809E0684600F03FF8044625686068C2
:10139000A847684600F05CF8684600F035F8002879
:1013A000F0D13EBDAC6F03000148007870470000EB
:1013B0002C2F00202DE9FF41074618E003A84BDF42
:1013C000044604B114E00F49684600F020F809E033
:1013D00000BF029805462E6869680398B0476846C2
:1013E00000F036F800BF02980028F1D100BFE5E711
:1013F00000BF052C04D000BF2046F9F78BF900BFD1
:10140000BDE8FF81FC6F030001468868704770B536
:1014100004460D46256028686060204600F001F80B
:1014200070BD14E0D0E900215268914202D1002140
:10143000816070474168096842685268914203D0F0
:10144000416809688160F4E7416808314160E9E773
:1014500010B50446A06800B910BD2168A06889686D
:101460000844A060D4E901104968884205D1606849
:10147000083060602046FFF7D4FF00BFECE770B58E
:1014800005460E466C6806E020683146AA6890471B
:1014900000B903E0246820680028F5D100BF206867
:1014A0003060266070BD014648680068704701469C
:1014B0004A6810684A68126822B14A68126812685D
:1014C0004B681A60704710B503460A4600205968F9
:1014D00007E00C68944203D114680C60012003E01B
:1014E00009680C68002CF4D100BF10BD02465058AA
:1014F00008B1012070470020FCE708B500224250E7
:101500004258009200BF08BDC0F80813704701227E
:101510004250704770B502460D4B03F5947413E0CA
:10152000E61AF01000EBD076761003EBC6010D68DA
:10153000954201D90C4606E0954202D201F108031A
:1015400001E0486870BD00BFA342E9D30020F9E77D
:10155000906D030030B504462046FFF7DBFF0546DB
:101560000DB9024830BD2846FCE700007C6D030041
:1015700001464FF4A07000EB810080B27047014635
:101580004FF480308840704708B5002242504258DE
:10159000009200BF08BDC0F808137047C0F80413DC
:1015A0007047D0F800228A43C0F800227047012219
:1015B000425070470021C0F8001570470521C0F85F
:1015C000001570470146D1F8C404C1F8C40470473F
:1015D0000246505808B1012070470020FCE708B5CA
:1015E000002242504258009200BF08BDC0F80413C8
:1015F0007047C0F800127047012242507047000047
:101600000348006808B1012070470020FCE7000093
:101610000004014010B500F05FF8012001490860A6
:1016200000BF10BD1805004001460020054A127990
:101630000AB1852004E0034A11600122014B1A71AE
:1016400070470000582E002010B50220FEF7F8F970
:101650004FF48270FEF7EBF90C20FEF7F7F900BFAC
:1016600000BF03480068C0F300400028F8D110BD57
:101670001804004070B5044604B970BD024EA501BF
:101680002846B04700BFF8E7316C030070B5044648
:1016900004B970BD024EA5012846B04700BFF8E767
:1016A000416D03000146080B40B270470146080B2C
:1016B00040B270470146080B40B270470146080B24
:1016C00040B27047014601F06040B0F1005F01D1C7
:1016D000012070470020FCE72DE9F04106254FF07E
:1016E0008040FFF7DFFF04462046E21704EBD2629A
:1016F0005211920002F1E022D2F800212146E317B4
:1017000004EBD3635B11A4EB43160123B3401A40EF
:101710000AB1012200E0002282BB4FF08040FFF7B7
:10172000C1FF04462E4620463146002804DB4A0706
:10173000130E134A135406E04A07170E114A00F01D
:101740000F031B1FD75400BF00BF4FF08040FFF7AF
:10175000A9FF0446204600280DDB00BF00BF00F0B3
:101760001F02012191404209920002F1E022C2F8D9
:10177000001100BF00BF00BF00BF00BFBDE8F08187
:1017800000E400E018ED00E02DE9F84307460E46BE
:10179000384601F093FB0446D4B14FF00008002016
:1017A00000906846F9F74AFC207910B14FF0010823
:1017B00002E02660012020719DF80000F9F744FC4A
:1017C000B8F1000F03D011252846BDE8F88300BF0B
:1017D00000252846F9E770B50546284601F06EFB5E
:1017E000044614B100202060207170BD2DE9F0473F
:1017F00004460D46914620793E4901EBC0063079FA
:1018000020B14FF008084046BDE8F087C6F80090C8
:1018100029462046FBF7A8F820680121C0F80015EA
:1018200000BF6979AA792B892068C0F80C15C0F827
:101830000425C0F8083500BFA97AEA7A206841EA91
:101840000223C0F8103500BF00212068FFF779FAA5
:1018500000212068FFF751FA4FF48E712068FFF7DE
:1018600045FA4FF488712068FFF740FA4FF48A7107
:101870002068FFF73BFA4FF482712068FFF736FAD1
:10188000306888B32068FFF715FF074695F804A075
:1018900038465146002804DB4A07130E164A1354F3
:1018A00008E04A074FEA126C144A00F00F031B1FAE
:1018B00002F803C000BF00BF2068FFF7FBFE074629
:1018C000384600280DDB00BF00BF00F01F020121D9
:1018D00091404209920002F1E022C2F8001100BFDB
:1018E00000BF00BF00BF00BF012030714FF00008F3
:1018F000404689E7682E002000E400E018ED00E093
:1019000070B504462079094901EBC0050026287905
:10191000022800D001264FF482712068FFF7DFF91A
:1019200010B1012028710126304670BD682E0020BC
:101930002DE9F05F0446894615461E4620791C496C
:1019400001EBC00A4A4600212068FFF7DCF94A464D
:1019500001212068FFF7D7F905F00107AB4605EB39
:10196000DB7207EB620291B22068FFF7C9F906F05B
:10197000010010B14FF010080AE006F0020028B193
:101980000FB1082000E00420804601E04FF000087D
:1019900041462068FFF7D5F90FB10C2000E0082080
:1019A0000346F2B25146204603F00EFDBDE8F09F1B
:1019B000682E002070B504460D46002600212068E0
:1019C000FFF7BFF904212068FFF7BEF92046FFF7B3
:1019D00097FF08B1012609E000BF2046FFF790FFFE
:1019E00008B1012601E0002DF7D100BF304670BDDF
:1019F00010B5044600212068FFF77DFA02206179C6
:101A000001EB4101014A505410BD00007C2E002022
:101A10002DE9F0430346164658792D4A42F82060D6
:101A2000587900EB40002B4A105C18B1082420467E
:101A3000BDE8F08393F904508F7828463A46002891
:101A400008DB4FEA427C4FEA1C68DFF88CC00CF8D8
:101A500000800BE04FEA427C4FEA1C69DFF87CC053
:101A600000F00F08A8F104080CF8089000BF00BFB0
:101A700093F90420104600280DDB00BF00BF00F0E2
:101A80001F070125BD404709BF0007F1E027C7F840
:101A9000005100BF00BF00BF00BF0A881868C0F82F
:101AA000082500BF08795A7902EB4202094D2A4401
:101AB0005070C8785A7902EB42022A449070012093
:101AC0005A7902EB4202A85400242046B0E70000F5
:101AD000782E00207C2E002000E400E018ED00E0CD
:101AE0002DE9F04104460D464FF48076012731463A
:101AF0002068FFF7D2F939462068FFF7E2F91DB1F7
:101B000039462068FFF7ECF9BDE8F08170B505466D
:101B10000C462748007C10B11126304670BD244881
:101B20001C3010F8150030B9214890F82D00401CE9
:101B30001F4981F82D00E1791D481C3000F815106F
:101B4000217A00EB4500417000BF207800F00300CF
:101B50006178302202EA01110843A1784FF4E06273
:101B600002EA01210843E1784FF4805202EA013190
:101B7000084321794FF4E02202EA014108436179E8
:101B80004FF4801202EA01510843A179120102EADE
:101B900001610843074901EB05118860227AE17968
:101BA0002846FFF7B7F900BF00263046B6E7000029
:101BB000506D0020107500402DE9F04104460E469E
:101BC000374890F82C0018B108252846BDE8F08168
:101BD0003348066020783349086000BF6078091DEB
:101BE000086000BFE0782E4981F82E00012081F8BE
:101BF0002C000020087481F82D00486181F82F0026
:101C00006FF00040FFF7A8F94FF48270FFF798F9E2
:101C10004FF48070FFF794F94FF48A70FFF790F952
:101C20000722A37810461946002806DB4F074FEA23
:101C3000176C1D4F07F800C009E04F074FEA1768FF
:101C40001A4F00F00F0CACF1040C07F80C8000BF29
:101C500000BF0721084600280DDB00BF00BF00F0D1
:101C60001F0301229A4043099B0003F1E023C3F8BC
:101C7000002100BF00BF00BF00BF0220FFF772F9C4
:101C8000074890F82E0010B10120FFF76BF900BF54
:101C900001200449F039086000BF0025284695E777
:101CA000506D0020F075004000E400E018ED00E009
:101CB0002DE9F04105460F463B48007C18B111263E
:101CC0003046BDE8F0810120374908740320FFF752
:101CD00043F901213846FFF715F9334890F82D00F4
:101CE000012809DD002405E0E0B200221146FFF7DB
:101CF00011F9641C082CF7D32B481C3000EB45006D
:101D0000427829481C3010F815102846FFF702F9D0
:101D10000020FFF72DF90420FFF72AF900BF4FF04C
:101D2000000842F2107400BF4FF48270FFF7FEF813
:101D300010B14FF0010805E00020FFF79BFC601E8A
:101D4000041EF1D100BF00BF4FF48070FFF7F8F818
:101D50004FF48270FFF7F4F8134890F82D00012833
:101D600010DD00240CE0104B1C3303EB44035A78C5
:101D70000D4B1C3313F81410E0B2FFF7CBF8641CC2
:101D8000082CF0D3084890F82E0018B10320FFF774
:101D9000E9F802E00220FFF7E5F8002002490874A4
:101DA000002630468DE70000506D00202DE9FF4FE2
:101DB00083B007460C46387900EBC0006A4901EB56
:101DC0008006307F28B14FF0080A504607B0BDE8C2
:101DD000F08F3D683A79654B53F822103868FFF769
:101DE000D3FC18B14FF0110A5046EFE70598306068
:101DF00006987060207B012803DC2078FEF781F9CB
:101E000002E02078FEF707FA002000900190207889
:101E100000231A460121FEF7D2F86078FF2808D087
:101E200094F801904846FEF76CF94846FEF7FBF837
:101E300001E04FF0FF39A078FF280ED094F802801F
:101E40004FF0010B002000905B46024601460190D6
:101E50004046FEF7B4F800BF01E04FF0FF38A0782D
:101E600086F82000E078F077E078FF280DD0207920
:101E700018B1E078FEF745F902E0E078FEF7CBF91B
:101E8000E078FEF7D0F82079B0772078C5F808051B
:101E9000C5F80C95C5F8108500BFA068C5F82405E5
:101EA00000BF217B627B0AB1012300E000231846BA
:101EB00031B1012906D0022907D0032908D000BF7B
:101EC00000BF08E040F0020005E040F0040002E03E
:101ED00040F0060000BF00BFC5F8540500BFA07960
:101EE000C5F8C00500BF00BF0720C5F8000500BF4A
:101EF000306888B33868FFF7D9FB8346617902916F
:101F000058460299002804DB4A07130E184A135456
:101F100008E04A074FEA126C164A00F00F031B1F35
:101F200002F803C000BF00BF3868FFF7BFFB83465D
:101F3000584600280DDB00BF00BF00F01F02012142
:101F400091404209920002F1E022C2F8001100BF64
:101F500000BF00BF00BF00BF0020707701203077B6
:101F60004FF0000A504631E7806D0020EC6C030012
:101F700000E400E018ED00E02DE9FC410546287979
:101F800000EBC0002D4901EB8004206808B32868ED
:101F9000FFF78CFB06463046002817DB00F01F02D7
:101FA00001219140264A430942F8231000BF00BF97
:101FB00000BFBFF34F8F00BF00BF00BF00BF00BF17
:101FC00000BFBFF36F8F00BF00BF00BF00BF00BFE7
:101FD00000BF2F68206898B11A493846FFF794FA75
:101FE000607F68B114213846FFF791FA00BF4FF4C3
:101FF00082713846FFF77AFA0028F8D0002060771F
:1020000094F82000FF280CD094F820600020009065
:1020100003460122014601903046FDF7D0FF00BF84
:1020200000BF00BF0020C7F8000500BF2868FFF709
:10203000D2FB00202077BDE8FC810000806D0020ED
:1020400080E100E0520108002DE9F04105460E460E
:102050001746287900EBC000154901EB80044FF0CA
:102060000008607F20B14FF011084046BDE8F081C4
:10207000206820B107F0140008B90120607796E8C5
:102080000E10C4E9053CC4E90312E07FFF2808D024
:10209000A07F18B1E07FFEF7BEF802E0E07FFEF718
:1020A00030F83B4632462146286803F0E1F8DDE788
:1020B000806D00202DE9F04704460D4616461F4668
:1020C0002846FFF75CFA804667B12846FFF750FACA
:1020D000814649462068FFF757FA41462068FFF7D6
:1020E0005DFA03E041462068FFF755FA206800F5E5
:1020F000A86141F8256000BFBDE8F08710B504462F
:1021000010212068FFF753FA0120217901EB4101EA
:10211000024A02EB8101087210BD0000246E00200B
:1021200010B5044600212068FFF741FA022021790A
:1021300001EB4101024A02EB8101087210BD00006F
:10214000246E002070B504460D46F8F70DF870BDFA
:102150002DE9F04105460E4617461C46DDF818806D
:102160004FF48072B2400123B34042EA0301286871
:10217000FFF717FA2868D0F800122143C0F80012C0
:1021800000BF43463A4631462846FFF793FFBDE875
:10219000F08100002DE9F05F04460D46924620795B
:1021A00000EB4000374901EB8006307A20B14FF058
:1021B00008094846BDE8F09FC6F800A0686870604E
:1021C000002709E03846FFF7D3F9804641462068EA
:1021D000FFF7DAF9781CC7B26079B842F2DC206800
:1021E000FFF76CFA804695F803B040465946002840
:1021F00004DB4A07130E244A135408E04A074FEA47
:10220000126C224A00F00F031B1F02F803C000BF2C
:1022100000BF2068FFF752FA8046404600280DDBD9
:1022200000BF00BF00F01F0201219140420992004F
:1022300002F1E022C2F8001100BF00BF00BF00BFE2
:1022400069782068D0F8042561F30102C0F80425FC
:1022500000BFA9782068D0F8082561F30102C0F812
:10226000082500BF29782068D0F8102561F3030203
:10227000C0F8102500BF012030724FF00009484619
:1022800098E70000246E002000E400E018ED00E074
:1022900000B501460248016000F004F800BD0000EE
:1022A00004E5014000BF024800680028FBD07047E9
:1022B00000E4014010B1032801D101E000E000BFBB
:1022C00000BF704710B50446FCF7A0FB014A03C2EB
:1022D00010BD0000A82E002010B504460548006877
:1022E00030B10448006803F0D7F9002001490860C4
:1022F00010BD0000982E0020DCB50646307800287E
:1023000023D13B211148008876DF044600BF2746D1
:10231000002F19D00EA01149114A891AC9080322A9
:10232000CDE9000742EA014073230EA215A1FEF792
:10233000FBFAFEF7B3F800BF00BF25B100BF284687
:10234000F8F7E8F900BF00BF00BFDCBD3C2F00205C
:102350006572725F636F646500000000647D030056
:10236000CC7C03002E2E5C6C69627A6E6F7264699D
:10237000635C7372635C7A626C655F6D6F64756CCD
:10238000652E630025733A2564205A4552524F52F8
:102390005F434845434B28257329206661696C3AA1
:1023A0002564000070B50546AE883046FCF76CFC2D
:1023B000044674B14FF6FF7340F2F31205F10801C1
:1023C00004F10A00FCF7E6FD607221463046FAF798
:1023D000C7FB70BD2DE9F0410546EF7BAE88012FAC
:1023E00001D0BDE8F0814FF6FF70FCF74DFC0446CC
:1023F0001CB9042002F058FBF3E700BF2680002040
:1024000020720E480168C4F80A104068C4F80E0033
:1024100000BF4FF6FF7340F2F31205F1100104F113
:102420000A00FCF7B7FD60720548C08918B921465B
:102430003046FAF795FB00BFD3E70000502E00208E
:102440003C6C00208188014A91807047B49500203F
:10245000CA7B012A02D18A88A0F824247047000090
:102460002DE9F04705460F46BE88A81D00EBC604BF
:102470002879A071F87B012802D0022806D102E059
:102480002888208003E06888208000E000BF00BF2B
:1024900020886188884236DD22882049204BC91A6D
:1024A000C908042343EA014033461EA1FEF718FA87
:1024B00021883046A5DF8046B8F1000F02D1012007
:1024C00060711FE0B8F1110F0DD101202071134987
:1024D000134A891AC908042242EA014032462149B6
:1024E000FEF7F2F90EE04046FFF734F881460B495B
:1024F0000B4A891AC908012242EA01404A461AA138
:10250000FEF7E2F900BFA079E179884203DDA17905
:102510003046FAF79DFCBDE8F0870000CC7C030054
:10252000CC7C030052657175657374696E672074A5
:102530006F2075706461746520415454204D54556A
:1025400020746F202575206279746573206F6E206A
:10255000636F6E6E656374696F6E20307825782EB8
:10256000000000004074030073645F626C655F6785
:10257000617474635F65786368616E67655F6D74CD
:10258000755F72657175657374282920726574753D
:10259000726E65642025732E0000000030B587B090
:1025A00005460020039004900590069002208DF8C7
:1025B0000C00174903C9CDE9000102A80190154A92
:1025C000518990886A46ADDF044654B902A8F9F7EC
:1025D000E3FD30B101218DF812100020ADF810009C
:1025E00003E040F2FD10ADF8100000BF09498888F3
:1025F00003A9B0DF0446112CF8D0BDF8100008B1D3
:1026000007B030BD2846F9F727FA00BFF8E7000009
:1026100028700300B495002070B58EB004460E46B5
:102620002C22311D03A8F4F761FFBDF80C50BDF852
:102630001000C1B2A01D00EBC500C171A11D01EBCE
:10264000C501CA792749284BC91AC908042343EA96
:1026500001402B4625A1FEF743F9BDF81220214980
:10266000214BC91AC908042343EA01402BA1FEF7F4
:102670002BF9BDF810201B491B4BC91AC9080423AC
:1026800043EA01402AA1FEF71FF9BDF816201549BB
:10269000154BC91AC908042343EA014029A1FEF7D2
:1026A00013F9BDF814200F490F4BC91AC9080423A8
:1026B00043EA014027A1FEF707F9206980B12949C3
:1026C00003C9CDE90101ADF80650A01D00EBC5001E
:1026D000C0798DF8080001A920462269904700BF03
:1026E0000EB070BDCC7C0300CC7C030044617461EF
:1026F000206C656E67746820757064617465642011
:10270000746F202575206F6E20636F6E6E65637425
:10271000696F6E2030782530782E00006D61785F0B
:1027200072785F6F63746574733A202575000000DA
:102730006D61785F74785F6F63746574733A202598
:10274000750000006D61785F72785F74696D653A3D
:10275000202575006D61785F74785F74696D653AE6
:1027600020257500D86B03002DE9F04705460E467D
:10277000341D2188A81D00EBC10794F8048022882D
:102780000B490C4BC91AC908042343EA01404346CC
:1027900009A1FEF7A5F8B879404501DAB87900E05B
:1027A0004046814620884946FAF752FBBDE8F0874B
:1027B000CC7C0300CC7C030050656572206F6E20DA
:1027C000636F6E6E656374696F6E20307825782054
:1027D00072657175657374656420612064617461EC
:1027E000206C656E677468206F662025752062799D
:1027F0007465732E000000002DE9F0410646B7888D
:102800003846FCF741FA05466DB16868F8F7F3FB06
:10281000044614B1204602F047F900BF4FF6FF709E
:10282000288000BF00BFBDE8F0810000054989880D
:102830008288914200D070474FF6FF71014A918023
:1028400000BFF8E7B495002070B504460E4600209E
:1028500084F82E04B088B4F8241488420CD120796E
:1028600050B901212046F8F77DFE054625B1A06B41
:1028700010B12846A16B884770BD70B504460D465F
:10288000AA88A11D01EBC200FCF708FC70BD000086
:102890002DE9FC4706460F46BD88B7F80690B01DE7
:1028A00000EBC5042B492C4A891AC908042242EAC4
:1028B00001404B462A4629A1FEF712F8B9F1170F3D
:1028C00001DA172000E0484681462088484501DDAE
:1028D000484600E020886080002020710095238811
:1028E00062881C49DFF870C0A1EB0C01C9084FF0E9
:1028F000040C4CEA014028A1FEF702F82188284682
:10290000B5DF8046B8F1000F0ED04046FEF722FE3C
:1029100082461049104A891AC908012242EA014038
:1029200052462DA1FDF7D0FF607908B1BDE8FC87C4
:10293000306968B1344903C9CDE90001ADF80250EE
:102940006088ADF80400694630463269904700BFA0
:1029500000BFEBE7CC7C0300CC7C030050656572C4
:10296000206F6E20636F6E6E656374696F6E2030CA
:102970007825782072657175657374656420616E61
:1029800020415454204D5455206F662025752062F7
:10299000797465732E0000005570646174696E6708
:1029A00020415454204D545520746F2025752062C9
:1029B000797465732028646573697265643A2025AB
:1029C0007529206F6E20636F6E6E656374696F6E1C
:1029D00020307825782E000073645F626C655F6735
:1029E000617474735F65786368616E67655F6D7449
:1029F000755F7265706C7928292072657475726EC6
:102A000065642025732E0000D06B03002DE9FC4186
:102A100005460E46B788B6F80A80A81D00EBC70425
:102A20002088404501DD404600E0208860806088C5
:102A3000172801DA172000E0608860806288114959
:102A4000114BC91AC908042343EA01403B460FA1B0
:102A5000FDF746FF286978B1607968B11A4903C962
:102A6000CDE90001ADF802706088ADF80400694658
:102A700028462A69904700BF002060712071BDE898
:102A8000FC810000CC7C0300CC7C0300415454202A
:102A90004D5455207570646174656420746F2025F1
:102AA00075206279746573206F6E20636F6E6E653A
:102AB0006374696F6E203078257820287265737092
:102AC0006F6E7365292E0000C86B030070B5054654
:102AD000AE1D30880749C98888420AD10548007E62
:102AE00038B1F8F701FF04461CB1024841690220E1
:102AF000884770BDB49500200548D0E900304FF0FC
:102B000080729A1840F100000149C1E90020704725
:102B1000A02E002070B50546A8880E4989888842F5
:102B200000D070BDAC1D2078022810D16088094902
:102B3000C98888420BD1207A042808D0207A062838
:102B400005D0207A052802D0A01CFFF727FD00BF82
:102B5000E7E70000B49500202DE9F04104460D465A
:102B60002888262801D0BDE8F081287A012802D0E3
:102B7000287A02280ED1A078F7F722FD07463946B9
:102B80002046F8F7EFFC064626B1A06B10B13046A0
:102B9000A16B884700BFE6E72DE9F0410446A51D7B
:102BA00028881249C98988421DD1688902281AD10A
:102BB000B4F804804046FCF767F8064696B105F184
:102BC0000C00F9F7F2FA20B131464046F9F7C8FF98
:102BD00008E07068F8F70FFA074617B1384601F0B9
:102BE00063FF00BF00BFBDE8F08100003C6C002027
:102BF000FEB504460E46B51D0020009001900290DF
:102C00002988208981420FD1688902280CD105F1D9
:102C10000C00F9F7CAFA18B1012084F8220029E063
:102C2000002084F8220025E02988208B81420FD1E2
:102C3000688902280CD105F10C00F9F7B6FA18B131
:102C4000012084F8230015E0002084F8230011E01F
:102C50002888A18988420DD1E06958B100208DF8FB
:102C6000000005F10C0001906989ADF80810684674
:102C7000E1698847FEBD01460868012805D008685B
:102C8000022802D00868042801D1012070470020E2
:102C9000FCE700002DE9F84F814600BF00244FE01B
:102CA0002C480057401C00B949E0204600F054F879
:102CB000054649462846FCF7D5FD00283ED020466B
:102CC00000F052F8064600956846FDF757FA83462D
:102CD0000BF5E060009950F82100C0F301408046F8
:102CE000B8F1020F01D1032000E0022082465146D4
:102CF0002846FDF7C1F900956846FDF73FFA83467F
:102D0000012000998840CBF8200500BF2846F9F73C
:102D1000A1FC8346F9F796FC074677B1032E09D04C
:102D2000B8F1020F01D1012E04D0B8F1030F04D184
:102D3000022E02D131462846B84700BF00BF641CAE
:102D4000042CADD34846FCF764F90028A6D1BDE8B1
:102D5000F88F0000426D002001460248425C22F0DC
:102D6000C0007047426D002001460248425C900955
:102D700070470000426D002070B504460D461646AF
:102D8000207A05280CD0607A28B10A480AA1026886
:102D90002846FCF7F9FF09A12846FCF7F5FF04E0F7
:102DA0001EB106A12846FCF7EFFF2846FDF701F803
:102DB00070BD0000002F0020257300000D0A0000E8
:102DC00010B50D48007800B110BDF5F707FBF5F719
:102DD00003FCF5F73FFAF5F759FBF6F71FFC012066
:102DE000F5F7F4FD03F054FB0220F5F7F7FB0120A3
:102DF0000149087000BFE7E7B42D0020F8B504468C
:102E00000D46E08838B116A00090E38816A218A1FC
:102E10002846FCF7B9FF207A05281FD0607A58B100
:102E2000217AA088FDF70AFB174951F82060324645
:102E300016A12846FCF7A8FF2846216802F00AFDE3
:102E4000A0880021FDF712FE0646207A104951F8AD
:102E5000202033460FA12846FCF796FFF8BD00005E
:102E60001B5B306D000000001B5B313B33316D009C
:102E700025734C6F67732064726F707065642028CF
:102E800025642925730D0A00002F002025730000FA
:102E9000EC2E00203C25733E2025733A20000000D4
:102EA00070B504460D462946204600F085F80020FE
:102EB0000149087070BD0000C02B00200146034886
:102EC000814201D1024870470020FCE70020004009
:102ED000602E0020094800680949884206D1094847
:102EE0000649086000200849086005E004480349D5
:102EF000086000200449086070470000682D002029
:102F0000B0520020B05B00206C2D002010B5FFF700
:102F100057FF0120F5F75AFD0120F5F791FA10BD92
:102F200010B505480078022800D110BD0220F5F741
:102F30004DFD00BFF9E70000A82D002010B50320CB
:102F40001A490870002025E000EB4001184A52F8A9
:102F5000212000EB40031549083141F8232000EB04
:102F60004001134A02EB810100EB40034A680F491C
:102F7000083101EB83014A6000EB40010C4A02EB8F
:102F8000810100EB40038A680849083101EB8301A5
:102F90008A60401C0428D7D306480068001F0349F4
:102FA00048600846F5F7B2F810BD0000186500202B
:102FB000B06400205C2D00202DE9FE4F804689463C
:102FC0004646DD4FB4784FF480713846F4F7A7FADF
:102FD000A9F1030000907378D849D94A891AC90821
:102FE000032242EA01402246D6A1FDF789FCD349DB
:102FF000D34A891AC908032242EA01404A46414697
:10300000FDF7D8FBB078B87070787870022038700F
:10301000012C13D1FD1C4FF00D0AF9F7B3FF6880A6
:10302000F9F7B2FFA880F9F7B1FFE880F9F7B0FF30
:1030300028815146384603F0F3FA7BE1022C13D184
:10304000FD1C4FF0090A0320287018206870282002
:10305000A8700220E8700420287108206871514689
:10306000B54803F0DDFA65E1032C39D1FD1C4FF0C2
:10307000090AFBF7E9FC2870FBF7ECFC68700020FC
:103080006870F5F769FD022801D1012000E00020F9
:10309000A97860F30001A970B2480178A87861F3BB
:1030A0004100A870F5F752F8142801DA012000E079
:1030B0000020A97860F38201A970F6F79FFBA97838
:1030C00060F3C301A9700020E870F5F73FF828719C
:1030D000F6F742FA68715146974803F0A1FA29E1E0
:1030E000042C1ED1FD1C4FF0090A9F4803F074FC0C
:1030F0009D48007D643828709B48007C401C6870A7
:103100009948007BA8709848007AE8709648007942
:1031100028719548007868715146874803F080FA15
:1031200008E1052C14D1F51C4FF0030A68792979C0
:10313000CDE90010EB78AA78697895F800C00CF515
:10314000FA6003F067FC51467B4803F069FAF1E04E
:10315000062C17D1F5F700FE68B17849784A891A2C
:10316000C908032242EA014080A1FDF7A3FB042124
:10317000304601F0A5FCF5F7F5FC0021304601F0E2
:10318000B7FCD7E0072C06D1F5F70CFD002130463F
:1031900001F0AEFCCEE0082C0DD1F9F70FF8054692
:1031A00025B90821304601F0A3FC03E0294630464A
:1031B00001F086FCBEE0092C0DD1F9F707F80546B1
:1031C00025B90021304601F093FC03E02946304642
:1031D00001F076FCAEE00A2C3ED1F01C0290FD1C02
:1031E00015200190029800780090FBF7EBFC28B1C5
:1031F0000421304601F064FCBDE8FE8FF6F702FAC8
:103200008246DAF804100098814204DC0721304637
:1032100001F056FCF0E700985AF820B0DBF8000007
:103220002860BBF80400A8800921DBF80C0090FBA3
:10323000F1F0C5F80600DBF80C00C5F80A00032021
:10324000A8732820E87318202874002068743A486E
:10325000019903F0E5F96DE00B2C0DD1F51C4B48FD
:1032600000210160416029680160A98881800221F4
:10327000304601F025FC5DE00C2C1AD1F51C4448C9
:1032800000210160416029680160A9888180F5F70B
:1032900063FC012804D00421304601F011FCABE7A7
:1032A0003B48F5F773FD82460021304601F020FCD3
:1032B00040E0102C06D1F5F7F3FD0021304601F077
:1032C00017FC37E00D2C04D10221304601F0F8FB49
:1032D00030E00E2C0AD1FD1C4FF0110A2846F9F7F8
:1032E00059FE5146144803F09BF923E00F2C1DD1E1
:1032F00000BF00BF00BF00BF00BFBFF34F8F00BFC4
:1033000000BF00BF2348006800F4E0602249084382
:10331000001D2049086000BF00BF00BFBFF34F8FF2
:1033200000BF00BF00BF00BF00BFFDE70221304665
:1033300001F0C6FB00BF5FE7A44B0020647D0300E3
:10334000CC7C0300727820636D643A256420696E3A
:103350006465783A256420646174616C656E3A2511
:1033600064000000C12B0020C84E002075706C6FF7
:103370006164696E672C63616E206E6F7420737474
:10338000617274206361707475726500162C002080
:103390001E2C00200CED00E00000FA052DE9F041A4
:1033A00007460D4616463C48007808B9BDE8F0814E
:1033B0003A4C6520A0700020607003202070C4F893
:1033C000037000205AE000EB400115F8213000EBBB
:1033D000C001E21D535400EB400135F82110C1F348
:1033E000072300EBC001491C535400EB400155F882
:1033F0002110C1F3074300EBC001891C535400EBBB
:10340000400105EB81010B7900EBC001C91C53544D
:1034100000EB400105EB81018988C1F3072300EB34
:10342000C001091D535400EB400105EB81014968BF
:10343000C1F3074300EBC001491D535400EB4001A9
:1034400005EB81010B7A00EBC001891D535400EBA1
:10345000400105EB81010989C1F3072300EBC0019D
:10346000C91D535400EB400105EB81018968C1F38C
:10347000074300EBC00108315354401CB042A2DBAB
:1034800006EBC600C01D1FFA80F84146034803F052
:10349000C7F800BF8AE70000C12B0020A44C002021
:1034A00070B5064C6820A07000206070032020706A
:1034B00003252946204603F0B3F870BDA44C002034
:1034C0002DE9F04105460E46074C6920A07000200A
:1034D000607003202070E57026710527394620466C
:1034E00003F09EF8BDE8F081A44C00202DE9F047E0
:1034F00004460D4616464FF00209022D74D360694A
:10350000A84271D92078012804D0022849D0032884
:103510000DD15EE02F4607EB5707206A00EB5721DD
:103520002046FBF75BFF8146B9F1000F00D075E044
:1035300038467F1CC0F3080104F1300001EB00089D
:1035400005F0010028B1F1B298F8000061F31F10F6
:1035500000E0304688F800000120E070206A00EBAF
:1035600057212046FBF73AFF8146B9F1000F00D002
:1035700054E0C7F3080104F1300001EB000805F046
:10358000010010B1C6F3071006E098F8000000F043
:10359000F000C6F30321084388F800000120E07022
:1035A0003CE0206A00EB15212046FBF717FF81461F
:1035B000B9F1000F00D031E0B1B240F2FF1202EADF
:1035C000450304F13002981801F0F8FE0120E07084
:1035D00024E0206A00EBD5112046FBF7FFFE814670
:1035E000B9F1000F01D019E019E040F2FF1101EA32
:1035F000850204F130015018FBF731FD66F31B0022
:10360000064640F2FF1101EA850204F1300150182C
:10361000314601F0C7FE0120E07000BF00BF484600
:10362000BDE8F08702480068810201F10050704750
:103630000C01001010B586B0694630A0FAF70BFDFA
:103640000446304830490860002C4ED1BDF80400D3
:10365000BC2101EB6020A0F5FA602C490870BDF890
:103660000400C0F343104870BDF8040000F01F00D0
:103670008870BDF80600C012C870BDF80600C0F31F
:1036800045100871BDF80600C006800E48711E483E
:1036900000680A680260496841601B49009809682F
:1036A000C86001201849486019491A4A891AC9088E
:1036B000032242EA014018A1FDF7FCF81449154A1B
:1036C000891AC908032242EA01400CA215A1FDF79C
:1036D000FBF80F490F4BC91AC908032343EA0140FD
:1036E00013A1009AFDF7F0F805E0002006490968EB
:1036F000C8600549486006B010BD0000302E626900
:103700006E0000009C510020302C0020392C00203D
:10371000647D0300CC7C030066696C656C6973741E
:103720003A000000206E616D653A257300000000CC
:103730002073697A653A25640000000010B50446DC
:10374000142C01DB002010BD21460548FBF7BEFF0D
:1037500021460348001FFBF7B9FF0120F3E70000F3
:10376000606C002070B50546002406E0044901EBBA
:1037700084002946FBF78CFF641C1E2CF6D370BD19
:103780005C6C002010B598B00F488068C04317905B
:103790000D48416817A8FBF7C1FF179901A8F9F771
:1037A00057F92C2201A90CA8F3F7A0FE002405E08C
:1037B0000DA931F81400FFF7D5FF641C0C98A04246
:1037C000F6D818B010BD0000586C002010B50446A3
:1037D00021460248FBF75CFF10BD0000606C002032
:1037E0002DE9F04781460E4617464FF00008D9F8FC
:1037F0000040022E02D36069B04202D80220BDE828
:10380000F08767B100BF4FF0FF3239462046FFF71F
:103810006DFE8046B8F1000F01D04046EFE700BFD3
:1038200031464846FAF7F6FF054605B922E0012D74
:1038300001D10220E3E7681C08B90120DFE700227C
:1038400031462046FFF752FE8046B8F1000F01D006
:103850004046D4E7D4E90410801E814206D2206994
:10386000401C2061207940F0010020712E466069E3
:10387000B042D5D800BF0020C1E70000042804D121
:1038800002490968491C014A11607047302F002025
:1038900010B504462046FAF788F808B1FFF72CF96E
:1038A00000212046F9F791FF10B12046FEF714FDE4
:1038B00001212046F9F789FF10B12046FEF702FDED
:1038C000204601F05BFF204600F044F810BD0000E8
:1038D0002DE9F05F834688464FF00D09002088F8F7
:1038E0000000DBE90267FBF791F8341A67EB01058A
:1038F00000210846091BA8411ADAB4F5350F05D393
:10390000F7F7F8FA11490844002101E0304639463A
:1039100082464FF49603524600210D48FAF75BF8B1
:103920008146B9F1000F02D10120BDE8F09F03E00C
:1039300000210748F9F73EFFB9F10D0F04D15846B1
:1039400001F0AAFE88F800000020EEE7FFFFB400B7
:10395000902E0020F8B5074655E000BF2B48FDF734
:10396000A2FD06460EB1304600E0002004460025C8
:10397000002C40D06B1ED4E902105940584001433E
:1039800002D101F011FB3EE02148006808B9012591
:1039900017E01F49D4E902300A68D2E90212591A25
:1039A00090410ED201251A480068D0E90210AA1EE3
:1039B00051405040014304D0154801681348FDF7B9
:1039C0005EFDBDB101F0F0FA044669462046FFF7FE
:1039D0007FFF58B10E48006810B93846F9F7EDFF7F
:1039E0000B4804609DF8000018B90DE0002008495C
:1039F000086007E008E00648006810B93846F9F7A3
:103A0000E3FF01E000BFA8E700BFF8BD246D03009D
:103A1000982E002070B504460E462546D5E90010C4
:103A2000884770BD10B504462046F6F74BF910B92B
:103A300042F2010010BD2046002803DB1F4A125C41
:103A4000520905E01E4A00F00F031B1FD25C520909
:103A50001146082904D20120884000F0EC0008B982
:103A6000002000E0012010B942F20200E2E7154810
:103A7000806868B16009134951F8200004F01F0202
:103A800001219140084361090E4A42F8210012E0E9
:103A9000204600280DDB00BF00BF00F01F020121FF
:103AA00091404209920002F1E022C2F8001100BFE9
:103AB00000BF00BF00BF0020BCE7000000E400E042
:103AC00018ED00E0F46E002070B50446F6F716F924
:103AD000054614488068D8B9012012498860124808
:103AE0000068124908400F49086010484FF0E02173
:103AF000C1F880010C488038D0F88400094948603A
:103B00004FF0FF310848001D01600020207001E0E7
:103B1000012020701DB900BF62B600BF00BF0020A9
:103B200070BD0000F46E002080E100E0FC06FFBDE7
:103B300038B504460D4624B1012C1FD0032C38D1D2
:103B400032E00020002817DB00F01F020121914025
:103B5000194A430942F8231000BF00BF00BFBFF35A
:103B60004F8F00BF00BF00BF00BF00BF00BFBFF34B
:103B70006F8F00BF00BF00BF00BF1BE000200090A0
:103B80006846F7F75BFA0D48007808B9FCF748F883
:103B90000A48C068401C0949C860012088709DF827
:103BA0000000F7F751FA05E0FDF734FDFCF75EF889
:103BB00000E000BF00BF38BD80E100E0D46C002011
:103BC00070B501460878821122B1012A1CD0022A60
:103BD00026D100E000BF087A8009CE7900EB86008C
:103BE0008E7906F0030600EB8623487900F00F0477
:103BF000887AC0094E7A06F0030600EB4605601984
:103C0000C61F581CB04070BD487A0C7A00EB0420E7
:103C1000CC7904F03F0400EB0443581C8002F2E727
:103C200000BF00BF0020EEE72DE9F04705460E4635
:103C300090463A4890F8230010B11120BDE8F08773
:103C400000240121354880F8231005F08000A8B138
:103C500006240221314880F8231077202F4981F86B
:103C6000280000212D4880F8291080F82A1080F8BB
:103C70002B1080F82C10FF2180F82D1005F07F010B
:103C8000264828300155320E601C244928310A5438
:103C9000C6F30742A01C0A54C6F30722E01C0A54CC
:103CA000201D0E54402D02D0482D04D101E095274F
:103CB00003E0872701E0FF2700BF00BF601D174911
:103CC00028310F54B8F1020F03D0B8F1030F0AD115
:103CD00004E00521114880F8241009E005210F486F
:103CE00080F8241004E001210C4880F8241000BF63
:103CF00000BF05F0800008B1012002E0074890F8FD
:103D00002400814609F10E00C3B2044A383206216C
:103D1000A2F1100000F054FE00208FE70C6F00208D
:103D20002DE9FE4305466878424908704248066816
:103D3000B469287820B1012834D002286CD14CE035
:103D4000687880B1B1464846F8F714FB074600BFD3
:103D5000B846B8F1000F04D000BF4046F6F7DAFCD1
:103D600000BF00BF00BFF6F7B7FF006820604FF448
:103D700000706060304800688069806888B1002009
:103D8000009001900290687808B1012000E00020C6
:103D90008DF80100A069029069463046A2689047FC
:103DA00000BF43E02448006880698068A0B1234ACE
:103DB00007CA8DE80700687808B1012000E00020FC
:103DC0008DF8010004F10C000190A0690290694691
:103DD0003046A268904700BF28E017480068806915
:103DE0008068C0B1154A0C32D2E900109268CDE962
:103DF00001020091687808B1012000E000208DF8F0
:103E0000010004F10C000190A0690290694630465F
:103E1000A268904700BF09E000BF032700BF03204E
:103E2000F6F778FC00BF00BFBDE8FE8300BF00BF0F
:103E3000FAE70000CC2E0020D02E0020D06E030028
:103E40002DE9FC5F80468946154698F8006098F891
:103E50000100000698F8021040EA014098F80310AB
:103E600040EA012098F8041040EA010B0127FE48BF
:103E7000808BB0F50E7F7DD010DC40F21322A0EBDA
:103E80000201904252D004DCD0B1B0F5047F72D16F
:103E90002FE006297AD01329F9D1BAE040F2612245
:103EA000811A904269D006DCA0F24D20002870D023
:103EB0000628ECD174E10A296CD00F29E7D1FEE184
:103EC0002BE2012200214020FFF7AEFE044600BF96
:103ED000A246BAF1000F04D000BF5046F6F71AFC14
:103EE00000BF00BF00BF00274FF40471DE4881838C
:103EF00000BF17B90120BDE8FC9F00BF01220021CF
:103F00004020FFF791FE044600BFA246BAF1000F21
:103F100004D000BF5046F6F7FDFB00BF00BF00BF56
:103F2000002740F21321D048818300BF0FB9012040
:103F3000E1E700BF00BF26F0030040B100BF04204E
:103F4000287000BF0021C84881830220D3E700BF4A
:103F500003224FF4D5714820FFF766FE044600BFE8
:103F6000A246BAF1000F04D000BF5046F6F7D2FBCC
:103F700000BF03E089E0D1E108E04BE100BF00BFF2
:103F8000002740F21921B848818300BF1FB90120E2
:103F9000B1E7D7E072E100BF06F00400A0B9B24873
:103FA000807A20F00700C01CAF49887200BF26F05D
:103FB000030040B100BF0420287000BF0021AA48C0
:103FC0008183022097E700BF0021A7480184807AFF
:103FD00000F00700032802D14FF0804000E00020ED
:103FE00001900222E9200199FFF71EFE044600BF5E
:103FF000A246BAF1000F04D000BF5046F6F78AFB84
:1040000000BF00BF00BF002740F2262196488183F1
:1040100000BF0FB901206EE700BF06F00400B8B37F
:104020009148807A20F00700401C8F49887226F062
:10403000040600BF8C48008C401C81B28A48018471
:10404000008CB0F5FA6F08DD00BF0220287000BFB9
:1040500000218548818302204DE702220021412072
:10406000FFF7E2FD044600BFA246BAF1000F04D0FC
:1040700000BF5046F6F74EFB00BF00BF00BF002751
:104080004FF40E717848818300BF17B9012032E7E1
:1040900013E000BF00BF26F0030040B100BF0420C2
:1040A000287000BF002170488183022023E700BFF1
:1040B00006F001000028BDD18EE000BF26F003000D
:1040C00040B100BF0420287000BF002166488183F2
:1040D000022010E700BF47E06348008C401C81B21B
:1040E00061480184008CB0F5FA6F08DD00BF022042
:1040F000287000BF00215C4881830220FBE65A48FB
:10410000807A00F00700032802D14FF0804000E0E1
:10411000002001900222E9200199FFF785FD044665
:1041200000BFA246BAF1000F04D000BF5046F6F718
:10413000F1FA00BF00BF00BF002740F24D214A48FE
:10414000818300BF0FB90120D5E600BF00BF26F074
:10415000030040B100BF0420287000BF0021424886
:1041600081830220C7E600BF06F001000028B3D11A
:10417000022200217A20FFF757FD044600BFA24625
:10418000BAF1000F04D000BF5046F6F7C3FA00BFE3
:1041900000BF00BF002740F253213348818300BF96
:1041A0000FB90120A7E600BF00BF26F0030040B111
:1041B00000BF0420287000BF00212B48818302200B
:1041C00099E600BF0BF0804030B12748807A20F09C
:1041D00008000830244988722348807A00F00700DC
:1041E000032829D0012251025020FFF71DFD04466B
:1041F00000BFA246BAF1000F04D000BF5046F6F748
:1042000089FA00BF00BF00BF002740F261211648B5
:10421000818300BF0FB901206DE600BF00BF26F00B
:10422000030040B100BF0420287000BF00210E48E9
:10423000818302205FE600BF0B4848300A49C8600E
:10424000012148388182012200214920FFF7ECFC3E
:10425000044600BFA246BAF1000F04D000BF50468A
:10426000F6F758FA00BF01E00C6F002000BF00BF56
:10427000002740F26B212C48818300BF0FB9012039
:1042800039E600BF00BF26F0030040B100BF0420A4
:10429000287000BF00212448818302202BE600BF44
:1042A00008F10108A9F1010000F0FF0900BF002199
:1042B0001D48C18300BF4FF41C71818300BF6B4652
:1042C00010224946404600F0B3F8022801DA0020E7
:1042D00011E600BF00BF00BF9DF8000048B100BF5D
:1042E0009DF80000287000BF00210F488183022044
:1042F00001E600BF0C484830FFF762FC0A494860FD
:104300004FF400710848018100BF0020287000BFF1
:104310000021054881830220EDE5D2E50027002138
:10432000014881830320E6E50C6F00202DE9F84F5A
:1043300006460F4614464FF0010A3C48808B38B1C0
:10434000B0F5267F22D0A0F2A220002867D156E047
:1043500064E096F8008000BF28F0030048B100BF79
:104360000420207000BF0021304881830220BDE876
:10437000F88F00BF761C781EC7B200BF00212B4803
:10438000C18300BF4FF42671818300BF6B464FF499
:1043900000723946304600F04BF8022801DA00205E
:1043A000E5E700BF00BF00BF9DF8000048B100BFB7
:1043B0009DF80000207000BF00211C48818302206E
:1043C000D5E700BF1948808A01281EDD012200219F
:1043D0004C20FFF729FC054600BFA946B9F1000FA4
:1043E00004D000BF4846F6F795F900BF00BF00BFF4
:1043F0004FF0000A40F2A2210C48818300BFBAF1BD
:10440000000F01D10120B2E700BF00BF00202070E3
:1044100000BF0021054881830220A8E799E74FF0FB
:10442000000A0021014881830320A0E70C6F0020CF
:104430002DE9F04704460D4616461F464FF0010889
:104440008448C08B40F2D912811A90427AD005DCA0
:1044500048B1A0F2C710002875D16EE0072973D0CB
:104460001329F9D1DBE0ECE07A48818AC182BDE012
:10447000002178480184FF20764981F82800002136
:1044800074480183032180F823105FE07148008C99
:10449000401C81B26F480184008C44F62061884240
:1044A00009DD00BF0220387000BF00216948C183C8
:1044B0000220BDE8F08702E0641C681EC5B215B199
:1044C0002078FF28F8D045B32078FE281CD1641C42
:1044D000681EC5B204225F4880F82320B54201DD82
:1044E000304600E028460146002004E0225C594B9B
:1044F000DB681A54401C8842F8D356480183C068D0
:104500000844544AD06021E000BF0520387000BF45
:1045100000215048C1830220CBE710234D4A383296
:104520000121A2F1100000F04BFA00BF4FF000088B
:1045300040F2C7114748C18300BFB8F1000F04D152
:104540000120B6E72CE07DE049E000BF414890F84B
:10455000230003289AD029E03E48008B301A1FFA26
:1045600080F9B9F1F00F01DD4FF0F00909F0FF0318
:1045700038480121C268283000F022FA3548C06866
:1045800048443449C8600846008B484481B23148E9
:10459000018300BF4FF0000840F2D911C18300BF72
:1045A000B8F1000F01D1012083E700BF2948008B3B
:1045B000B042D1DB2748C08A401E81B22548C18263
:1045C000022300F138020121283000F0F9F900BF80
:1045D0004FF000084FF4F0711E48C18300BFB8F1DE
:1045E000000F01D1012064E700BF00251948C08AEF
:1045F00000287FF43DAFFF20164981F828000223F0
:1046000001F138020121A2F1100000F0D9F900BF38
:104610004FF000084FF4F6710E48C18300BFB8F1A7
:10462000000F01D1012044E700BF0021094880F8B4
:10463000231000BF0020387000BF0648C18302204D
:1046400037E711E74FF0000800210248C18303203B
:104650002FE700000C6F00202DE9F0470646884642
:1046600014460125D548808BB0F53B7F70D009DC1E
:1046700088B1A0F2C320002842D010287DD0212884
:1046800068D1A3E0A0F20A30002879D0162878D0AB
:104690002628F5D16CE18AE196F800A000BF2AF047
:1046A000030048B100BF0420207000BF0021C348B0
:1046B00081830220BDE8F08700BFC048807A00F007
:1046C0000700012830D0BD48808A01282CDDBB4876
:1046D000012201695920FFF7A7FA074600BFB94632
:1046E000B9F1000F04D000BF4846F6F713F800BF39
:1046F00000BF00BF002540F2C321B048818300BF46
:104700000DB90120D6E700BF96F800A000BF2AF03F
:10471000030040B100BF0420207000BF0021A74863
:1047200081830220C6E700BFA448818AC182D2E00B
:104730000021A2480183042180F82310FF209F4913
:1047400081F828000846808A012804DDFC2103E066
:104750005DE012E02CE1FE21984880F82910022348
:1047600000F138021946283000F02AF900BF002570
:1047700040F2D3219148818300BF1DB9012099E700
:104780008DE0C7E000BF25E08C48008BC0F50070CD
:104790001FFA80F9B9F1F00F01DD4FF0F009874AF7
:1047A000D368128B981809F0FF010123834A38322D
:1047B00000F006F98148008B484481B27F480183AC
:1047C00000BF00254FF43971818300BF0DB901206E
:1047D00070E700BF7948008BB0F5007FD4DB7748E5
:1047E000C06800F500707549C8600321734880F8FF
:1047F0002310032300F138020121283000F0E0F8F3
:1048000000BF00254FF43B716C48818300BF0DB998
:1048100001204FE700BF694890F83A0000F01F01FF
:10482000052915D00B2901D00D2908D100BF05207D
:10483000207000BF00226148828302203AE700BF57
:104840000420207000BF00225C488283022031E7F0
:1048500000215A48018433E05848008C401C81B242
:1048600056480184008C44F62061884208DD00BF70
:104870000220207000BF002150488183022019E7E8
:1048800010234E4A38320121A2F1100000F098F8AE
:1048900000BF002540F20A314848818300BF0DB9AE
:1048A000012007E700BF002007E0315C21B10022B2
:1048B000424981F8232002E0401C4045F5D300BF67
:1048C0003E4890F823000328C6D03C48C08A401ECA
:1048D00081B23A48C1823948C08A00287FF428AFA3
:1048E0003648808A012859DDFF20344981F82800A4
:1048F000FD21324880F82910032300F138020221FB
:10490000283000F05DF800BF00254FF448712B48B7
:10491000818300BF0DB90120CCE600BF00212748EC
:104920000184032180F8231033E02448008C401CCC
:1049300081B222480184008C44F62061884208DD5F
:1049400000BF0220207000BF00211C48818302208C
:10495000B0E61023194A38320121A2F1100000F00C
:104960002FF800BF00254FF44C711448818300BF1D
:104970000DB901209EE600BF002007E0315C21B1A7
:1049800000220E4981F8232002E0401C4045F5D367
:1049900000BF0A4890F823000328C6D000BF0020BB
:1049A000207000BF002105488183022082E673E663
:1049B000002500210148818303207BE60C6F002045
:1049C0002DE9F84305460E461746984600BF1348A2
:1049D00090F8580000906846FBF700FC81460121E2
:1049E000009A01FA02F0C9F80C0500BF00BF00BF31
:1049F0003B46324629460A48CDF80080FBF7ABF922
:104A0000044600BFA146B9F1000F04D000BF4846DC
:104A1000F5F780FE00BF00BFBDE8F8830C6F0020F3
:104A2000186F030010B501E001F05BFBF6F744F9E5
:104A30000028F9D110BD0000FEB505460C496846B6
:104A4000FCF7E5FC0DE06846FCF7DEFC0446266852
:104A500028466168B04708B91120FEBD6846FCF7DA
:104A6000F7FC6846FCF7D0FC0028ECD100BFF4E767
:104A7000746F0300FEB505460A496846FCF7C7FC9B
:104A80000AE06846FCF7C0FC0446266828466168D0
:104A9000B0476846FCF7DCFC6846FCF7B5FC00282C
:104AA000EFD1FEBD906F030010B504460348806946
:104AB00018B1024881692046884710BD3C6C00202F
:104AC0002DE9F04105468846084CE61C0427A878E5
:104AD000A070687860700420207020700220307010
:104AE0003946204601F09CFDBDE8F081A44B002032
:104AF0002DE9F04104460E46074DF01C87B2A07820
:104B0000A87060786870022028703946284601F045
:104B100087FDBDE8F0810000A44B002070B505467C
:104B20000E463146284675DF044624B1112C02D0CA
:104B30002046FFF7B9FF0CB9012070BD0020FCE74B
:104B40002DE9F84F88461546002D35D04FF0000965
:104B50000A20009000BF08EB09012A460020F4F764
:104B6000DBFB0446A1442D1BFCB91448007800B9B6
:104B700020E0012606B90FE000BF4FF47A7707B9AD
:104B800006E0DFF83CA04FEA871B5846D04700BF3D
:104B9000701E061EF1D100BF0098401E00900098C4
:104BA00018B900200549087004E001200349087085
:104BB000002DD0D100BF00BFBDE8F88FD42E00205B
:104BC000516F03002DE9F04707460E4614469A46FA
:104BD000B86A10B90720BDE8F0874FF0000836E04A
:104BE00008EB4801B86A00EB8105A88800F10209CA
:104BF000B9F1FE0F01D90C20EDE709F10100218880
:104C000070542088401C20801620218870542088F1
:104C1000401C208022889119288801F006F92188FB
:104C200008442080A88800280DDDA86808B907205E
:104C3000D1E7AA8823889819A968F2F757FC208839
:104C4000A9880844208008F1010000F0FF0897F8C7
:104C50002C004045C4DC0020BDE70246022082F85B
:104C6000310092F8240010B10720087001E0032001
:104C70000870108A88810020C2F8200402F22640C1
:104C80004860D0688860002070470246012082F8A2
:104C900031000020C2F8200402F2264048600020C3
:104CA000886002200870802088810020704770B5DD
:104CB00004460D466069A860208BA88194F8240002
:104CC00018B1062084F83C0002E0012084F83C0082
:104CD000204601F047F978B10220287504212046CA
:104CE000F9F7D5FC064600BF304600B170BD00BFE5
:104CF000052084F8310002E0032084F8310004F537
:104D00008260C4F820040020F0E770B504460D4628
:104D1000E069A860208CA88194F8240018B10620CE
:104D200084F83C0002E0012084F83C00204601F0B9
:104D300019F978B10220287504212046F9F7A7FC5B
:104D4000064600BF304600B170BD00BF062084F8A3
:104D5000310002E0042084F8310004F58260C4F8D8
:104D600020040020F0E7000070B5054611480068F7
:104D7000407E08B1062070BD00BF0F4800F1080159
:104D8000026828469047044600BF24B9012009491B
:104D9000096848760BE00F2C09D10849084A891A9E
:104DA000C908012242EA01400649FBF783FD20467B
:104DB000E1E700005C2F0020D0950020647D030017
:104DC000CC7C0300FC7A030000BF0A7822F00F02BB
:104DD0000A700A7822F0F0020A7000BF062850D24A
:104DE000DFE800F0030E1B28354200BF0A7822F0EE
:104DF0000F020A700A7822F0F0020A7000BF40E049
:104E000000BF0A7822F00F02521C0A700A7822F0C2
:104E1000F00210320A7000BF33E000BF0A7822F0BF
:104E20000F02521C0A700A7822F0F00220320A7037
:104E300000BF26E000BF0A7822F00F02521C0A7061
:104E40000A7822F0F00230320A7000BF19E000BF89
:104E50000A7822F00F02921C0A700A7822F0F002FF
:104E600010320A7000BF0CE000BF0A7822F00F0277
:104E7000921C0A700A7822F0F00220320A7000BFF9
:104E800000BF00BF7047000010B50CE000BF2C4809
:104E9000806804462B4800782168884700B910BD17
:104EA0002748FCF7D5FA00BF254880680028EDD1D7
:104EB00000BFFBF7EDFD00BF00BFFBF7EFFA0028D6
:104EC000FBD100BF00BF1F480078032803D01D4856
:104ED000007802281DD100BF00BF00BF00BF00BF87
:104EE000BFF34F8F00BF00BF00BF1748006800F43A
:104EF000E06016490843001D1349086000BF00BF69
:104F000000BFBFF34F8F00BF00BF00BF00BF00BF97
:104F1000FDE7FCF749FA10B133DF044600BF00BFDC
:104F200001200B49086000BF00BF00BF00BFBFF3F6
:104F30004F8F00BF00BF00BF00E020BFFDE70000B3
:104F4000006F0020C02E00200CED00E00000FA05EC
:104F50000005004070B504460D462CB901200349F8
:104F600048700020F7F7A8FC70BD0000D46C00204A
:104F700070B51620FEF756FD044600BF254625B144
:104F800000BF2846F5F7C6FB00BF00BF70BD10B5D7
:104F900000BF00F009F818B14FF0FF328260C26024
:104FA0000028F6D110BD000010B50448FCF77FFAC8
:104FB00004460CB1204610BD0020FCE7246D030020
:104FC0002DE9FE4306468846F468357C9648C08A3B
:104FD00030B900BF944991F85800FBF729F900BF98
:104FE000914890F82300022804D08F4890F82300BD
:104FF00001287DD1A81FC5B2A41D706800784C2877
:1050000003D115B1681EC5B2641C02E0681EC5B2AA
:10501000641C15B12078FF28F8D045B97068007875
:105020004C2803D1681CC5B2641E00E00024002C8B
:1050300049D17D4890F82200012844D001208DF804
:105040000100794890F82200012806D0022805D0F6
:10505000042816D005281CD117E000BF00208DF8C9
:1050600000000321704880F8221000BFF5F7C2FE4F
:10507000074627B100BF3846F5F74CFB00BF00BF1D
:1050800010E001208DF800000CE002208DF80000F7
:1050900008E000BF032700BF0320F5F73BFB00BF7C
:1050A00000BF00BF00BF00BF5F4991F85800FBF789
:1050B000BFF800BF03215C4880F8221001686846F1
:1050C0008847BDE8FE83584890F82300022817D18E
:1050D0000121554880F82310277827F0010070B986
:1050E000514890F824000E30C3B24F4A383200E0E5
:1050F0000AE00621A2F10A00FFF762FCE1E700BF27
:105100000021494880F8231006200290464890F874
:105110002200012806D002280BD0042830D0052810
:1051200075D150E00221404880F82210002181838F
:1051300000BF02AA29462046FEF782FE02281EDB97
:1051400000208DF804009DF808008DF8050003216B
:10515000354880F8221000BF014691F85800FBF74F
:1051600067F800BF00BF314A4FF080415068C0F877
:10517000241500BF00BF2C48016801A888474FE0F4
:1051800002AA29462046FFF7D1F802281ADB01209F
:105190008DF804009DF808008DF8050003212248D1
:1051A00080F8221000218182C18280F8231000BF84
:1051B000014691F85800FBF73BF800BF1A48016818
:1051C00001A888472CE002AA29462046FFF744FAA6
:1051D00002281ADB02208DF804009DF808008DF8E3
:1051E00005000321104880F82210002180F82310C8
:1051F0008182C18200BF014691F85800FBF718F880
:1052000000BF0948016801A8884709E0FFE700BF1F
:10521000032700BF0320F5F77DFA00BF00BF00BFE2
:1052200000BF00BF4DE700000C6F0020186F0300A7
:1052300070B586B004460D462E4620788DF80400E1
:1052400060680290217A8DF80C10E1680491217C4D
:105250008DF81410044850F82610044850F8262001
:1052600001A8904706B070BDD86D0020C86D002021
:105270002DE9F04704460E4615461F46286818B12A
:105280002868FCF71FFA28B1A86850B1A868FCF795
:1052900019FA30B9002070774FF010084046BDE889
:1052A000F087D5E90001C4F844054FF4A962115113
:1052B00000BFD5E90201C4F834054FF4A7621151CB
:1052C00000BF4FF48C712046FCF717F92046394691
:1052D00001F0010232B100BF01234FF4AA62135062
:1052E00000BF06E000BF00234FF4AA62135000BFC6
:1052F00000BF01F0020232B100BF01234FF4A862E7
:10530000135000BF06E000BF00234FF4A862135003
:1053100000BF00BF00BF07F0080018B910212046E9
:10532000FCF7F5F83068A0B900BF4FF48C71204647
:10533000FCF7DCF80028F8D0F07FFF281CD0B07F05
:1053400018B1F07FFAF7DDFE16E0F07FFAF763FFA1
:1053500012E0A146012020EA970ABAF1000F04D119
:1053600040214846FCF7D0F804E04020C9F8040387
:1053700000BF00BF00BF00BF4FF0000840468EE7EF
:1053800070B506460C461546A9B204F11A0000F0A5
:1053900015F83078032804D1290C04F1140000F02A
:1053A0000DF870BD00F8011B090A00F8011B090A7D
:1053B00000F8011B090A00F8011B704700F8011BE7
:1053C000091200F8011B70472DE9F04105460F4610
:1053D00014461E46022038717C713868A8B14FF01F
:1053E000820804F0040008B148F0100804F0080036
:1053F00008B148F0200804F0100008B128F0800837
:1054000041462868FBF779FC00BF4FF48271286899
:10541000FBF76CFC04F0800028B128688219114663
:105420000846BDE8F08131462868FBF78DFC002076
:10543000F7E7000010B5044601200349087008464C
:10544000F2F764FE10BD0000D46700202DE9F05F84
:1054500005460E4690461F46DDF828904FEA154A4D
:10546000F8F79CF983464AEA0B42781C00EA0900E7
:105470000E4941F8202007EA090001EB800420686A
:1054800065F3C5002060206868F3891020602068FB
:1054900066F39F202060206820F00300401C2060FD
:1054A000206820F004002060BDE8F09F947C00207C
:1054B0002DE9FC478046894616461C461C4807686D
:1054C000012201A92046F7F709F8C0B1019800F1BF
:1054D000020A002509E056F8252050460AF1010A83
:1054E0003840144941F820206D1CA542F3D30097A1
:1054F000224649464046019BFFF7A8FF00BF0D48E2
:105500000C38007880B1002000906846F5F796FDD1
:1055100000BF00BFFAF7C2FF0028FBD100BF9DF813
:105520000000F5F791FD00BFF9F7C3FDBDE8FC876A
:10553000E82E0020947C00202DE9F04781460C469F
:1055400015469846002608F00100A0B105E0641C4D
:10555000761C39464846F7F735F82778002FF6D1FC
:1055600004E06D1E20214846F7F72CF8B5421BD900
:10557000002DF6D118E01CB12046F1F7DBFF0646FE
:1055800004E06D1E20214846F7F71CF8B54201D90A
:10559000002DF6D105E0641C761C39464846F7F725
:1055A00011F82778002FF6D1BDE8F08770B50446D2
:1055B000204600F043F80546002D38D12078032816
:1055C0002ED1207901282BD14202002104F1300094
:1055D000F9F77AFE4AF6552104F22E20FFF7EEFE87
:1055E000144904F13000FFF7DDFE134904F505709E
:1055F000FFF7D8FE04F506702169FFF7D3FE04F526
:105600000770E168FFF7CEFEE069401CE062607859
:10561000012304F13001E26AF8F740F8002020711C
:10562000607800221146F7F7E9FE00B1012528460F
:1056300070BD000052526141727241612DE9F0412A
:1056400004460027E078F8B1E56A607801232A462D
:1056500004F13001F8F722F808B1012714E0002026
:10566000E070206A281AA16988420DD2A67809E064
:10567000A0690544607801232A4604F13001F8F757
:105680000DF8761E022EF3D23846BDE8F0810246B0
:10569000501A20F07F4070472DE9FE4304464FF03A
:1056A00000083348007801285ED1002C5CD0F9F75F
:1056B000ADF9D4E90232C01A914147D300200090DD
:1056C0006846F5F7BBFC206918B94FF0FF31A160BF
:1056D000E1609DF80000F5F7B7FC60690190A069F2
:1056E0000290244A082101A8F5F77AF9054600BF7F
:1056F0002F4627B100BF3846F5F70CF800BF00BFB2
:10570000002000906846F5F799FC206988B14FF0B9
:10571000FF33D4E9021059405840014309D0D4E97D
:1057200002302169591840F10000C4E90210012635
:1057300000E000269DF80000F5F786FC2EB121461A
:105740000D48FBF79CFE4FF001080DE04FF0FF33D2
:10575000D4E9021059405840014305D0214606487B
:10576000FBF78DFE4FF001084046BDE8FE830000C8
:105770009C2E0020153A0300246D0300F8B5064660
:10578000694620480068F9F767FF044637E020784B
:1057900020B1012810D0022824D11DE06068D0E992
:1057A00002104FF0FF3359405840014303D01648D0
:1057B0006168FBF764FE16E0144960680968884276
:1057C00003D100201149086005E00F486168FBF72C
:1057D0007AFE054600BF06E0FFF7D9FB01200C4921
:1057E000087000E000BF00BF694606480068F9F78E
:1057F00025FF694603480068F9F72EFF0446002C90
:10580000C5D1F8BD206D0300246D0300982E002043
:105810009C2E0020F8B505460E4669460B480068E8
:10582000F9F7FEFE04467CB12570666069460748BC
:105830000068F9F71FFF28B100BF0548F8F79AF88C
:1058400000BF00BF0020F8BD0420FCE7206D03006E
:10585000902E0020704700002DE9F043A3B00546CC
:105860000E4690461F4600203880012229462448D3
:10587000F8F72CFA8146B9F1000F0DD02149224AE0
:10588000891AC908012242EA01402A461FA1FBF7F2
:105890001BF823B0BDE8F0830024194A802103A837
:1058A000F8F7BDF911E001AB02AA1CA103A8F1F7BA
:1058B0005FFE029806F8140006EB44010198487058
:1058C000641C444500DB07E000BF0D4A802103A8AB
:1058D000F8F7A5F90028E6D100BF3C8009490A4A3B
:1058E000891AC908032242EA014023462A460DA12B
:1058F000FAF7F6FF0248F8F781F900BFC9E70000A0
:1059000088650020647D0300CC7C03006F70656EA9
:10591000202573206661696C65640A0025782C2552
:10592000780000006C6F6164202573206366672037
:1059300073697A653A25640A0000000070B586B084
:1059400006460C462146304600F051F908B106B033
:1059500070BD94F82F0018BB207B022802D0207B5A
:1059600003281DD1616AA069814219D1E069606292
:105970006069A06294F82000C0F3401084F82C0005
:10598000002084F82D00207B032804D121463046D6
:1059900000F0C4F93DE02146304600F08DF838E0D3
:1059A000142204F10C0101A8F1F7A0FD94F82F00D6
:1059B000E0B13046FBF706FE054605F0020018B1DF
:1059C00001208DF8000010E005F0040018B102205D
:1059D0008DF8000009E005F0010018B103208DF8F2
:1059E000000002E004208DF8000002E000208DF8A5
:1059F0000000002084F8300094F8200000F004003B
:105A000010B194F82F0018B16846D4E900219047EE
:105A100000BF00BF9BE70146032001F001020AB16D
:105A20004FF4024001F002020AB148F2012001F0F5
:105A300004020AB148F20220704770B505460C46D0
:105A4000A16A606B884235D200BFD5F81805C0B294
:105A5000626B616A8854606B401C6063A06A401E80
:105A6000616B814209D194F8200000F0400020B918
:105A700002212846FBF7BDFD18E0A16A606B884251
:105A800006D194F8200000F0400008B9012070BD54
:105A9000A16A606B884209D194F8200000F04000B0
:105AA00020B1022084F82D000020F0E720212846B4
:105AB000FBF7A2FD0120EAE7F8B506460C460027F1
:105AC000344800904FF482713046FBF788FD4FF464
:105AD00092713046FBF783FD4FF48E713046FBF731
:105AE0007EFD4FF484713046FBF779FD0020606342
:105AF00084F82F00A06A012809D194F8200000F052
:105B0000400020B902213046FBF773FD03E001217C
:105B10003046FBF76EFD20213046FBF76DFD94F813
:105B20002D00022803D000213046FBF765FD2068D8
:105B300038B140F28620A060A1683046FBF756FDE0
:105B400025E002E00098401E00900098002805DD46
:105B50002146304600F04BF80028F3D194F82F008E
:105B600058B13046FBF72EFD054625B12846FFF714
:105B700052FF074600E0032700BF0098002806DC1C
:105B80003046FBF717FD3046FBF718FD0327384674
:105B9000F8BD0000A086010070B505460C46A16A5C
:105BA000606B884206D2626B616A885CC5F81C052E
:105BB00000BF1AE094F82C0028B11C212846FBF7FE
:105BC0001BFD002070BD94F8200000F0400040B1A3
:105BD0001C212846FBF710FD012084F82D00002031
:105BE000F0E714212846FBF707FD0120EAE770B52E
:105BF00005460C4600264FF482712846FBF7E8FC68
:105C000028B14FF482712846FBF7E9FC012694F88D
:105C10002F0078B14FF492712846FBF7E0FC4FF467
:105C20008E712846FBF7DBFC4FF484712846FBF7A6
:105C3000D6FC5FE04FF492712846FBF7C9FC60B1D7
:105C40004FF492712846FBF7CAFC14212846FBF753
:105C5000D3FC012084F82F004CE04FF48E712846CD
:105C6000FBF7B6FC08B34FF48E712846FBF7B7FC80
:105C7000606B401C60634FF492712846FBF7A8FCF0
:105C800060B14FF492712846FBF7A9FC1421284615
:105C9000FBF7B2FC012084F82F002BE021462846B8
:105CA000FFF77AFF30BB002070BD4FF484712846A7
:105CB000FBF78EFCF0B14FF484712846FBF78FFCA4
:105CC0004FF492712846FBF783FC60B14FF4927158
:105CD0002846FBF784FC14212846FBF78DFC0120A5
:105CE00084F82F0006E021462846FFF7A6FE08B9F3
:105CF0000020D9E77EB1002084F82D0094F82F0011
:105D000038B92146284600F0F1F980F0010084F806
:105D10002F000020C8E70120C6E70000F8B50646BE
:105D20000C4600272F4800904FF482713046FBF755
:105D300056FC4FF492713046FBF751FC4FF48E71D4
:105D40003046FBF74CFC4FF484713046FBF747FCC0
:105D500000213046FBF74DFC0020606384F82F00E3
:105D600020213046FBF748FC94F82D00012803D091
:105D700008213046FBF740FC21463046FFF70CFF78
:105D8000206838B140F28620A060A1683046FBF759
:105D90002DFC25E002E00098401E009000980028AD
:105DA00005DD21463046FFF722FF0028F3D194F8A5
:105DB0002F0058B13046FBF705FC054625B12846B3
:105DC000FFF729FE074600E0032700BF00980028E0
:105DD00006DC3046FBF7EEFB3046FBF7EFFB032714
:105DE0003846F8BDA086010030B504461088C01CB6
:105DF000984201D90C2030BD0220158848551088E2
:105E0000401C10800A20158848551088401C1080BE
:105E100015884C551088401C10800020EBE7014687
:105E200008784A7840EA0220704702460A70100A51
:105E300048700220704700002DE9FF4F81B088466E
:105E400016461F46DDE90E4B45464FF0010A03E0BA
:105E5000B5FBF6F50AF1010AB542F9D2574500D96A
:105E6000BA460BF0010098B994B10BF00200022879
:105E700003D117B93020009001E02020009004E009
:105E8000641EDDE90010F6F79DFB0CB1A245F7D3C7
:105E9000012509E0012F01D97F1E04E0B8FBF5F9C7
:105EA000B14500D201E07543F4E700BF00BFB8FB85
:105EB000F5F909FB15880D4810F809100198F6F757
:105EC00081FBB5FBF6F5002DF1D10BF0010048B1D7
:105ED00044B104E0641E20210198F6F773FB0CB175
:105EE000A245F7D305B0BDE8F08F0000466D030072
:105EF000F8B506463546A8B2F8F7C6FE04466CB3B8
:105F0000207A1749097B88420ADAA8B204F10A010B
:105F1000FEF704FE074617B1207A401C20721DE0F0
:105F2000002020720E48007C50B1A8B23B2176DFE1
:105F3000074627B1082F02D03846FEF7B5FD00BF4F
:105F40000748406950B100208DF80000A8B2ADF8B4
:105F50000200034841696846884700BFF8BD000059
:105F60003C6C002010B50446607940B194F82E04D2
:105F700028B9204600F0B6F808B1012010BD002075
:105F8000FCE72DE9FC478046894615469A46DDE93F
:105F90000A675346022249464046CDE9006700F0B1
:105FA00017F8044600BF204608B1BDE8FC8700BFD3
:105FB0005346102229464046CDE9006700F008F814
:105FC000044600BF204600B1EFE700BF0020ECE729
:105FD0002DE9FF5F07468B4696461D460E9C4FF007
:105FE000000920880390C84647E0786800EB8800E5
:105FF00000680190002202A901A864DF064600BFE4
:10600000304610B104B0BDE8F09F00BF9DF8080015
:10601000704530D1B9F1000F01D0002000E002201E
:10602000009020889DF808100144009801440F98C2
:10603000814201DD0C20E5E7B9F1000F0AD120888B
:10604000401C2080208805F800B02088401C20805B
:106050004FF001092088421902A901A864DF064611
:1060600000BF304600B1CDE700BF21889DF8080091
:106070000844208000BF08F1010838884045B4DC9E
:10608000B9F1000F0DD021880398401C081A1FFA9F
:1060900080FABAF1FF0F01DD0C20B3E7039805F891
:1060A00000A00020AEE770B504460D4684B120681C
:1060B00070B12068007858B12068C088A1888842F3
:1060C00006D121684878F7F761FA00F0010018B1AD
:1060D00000202860092602E020682860002630465B
:1060E00070BD7047014691F83004704770B50546A1
:1060F0000C46A16A606B884207D02846FBF75AFA23
:106100002846FBF75BFA002070BD0120FCE7000089
:1061100010B504462078012806D10A2007490870E6
:106120000846F1F7F3FF08E02078022805D10B209C
:10613000024908700846F1F7E9FF10BD44680020E5
:1061400001480088704700003E2F0020F0B5ADB038
:10615000054600BF9DF8A80020F00F00401C2A90C3
:106160009DF8A80020F0F00010302A9000BF2868A9
:10617000F1F7E0F986B232462AA829687CDF0446A6
:1061800000BF2746002F1AD0A1A0A449A44A891A0B
:10619000C9080322CDE9000742EA014040F2311369
:1061A000A0A2A8A1FAF7C0FBFAF778F900BF00BFD8
:1061B00026B100BF3046F4F7ADFA00BF00BF00BF04
:1061C00000202B902C901020ADF8AC003C20ADF8B6
:1061D000AE000020ADF8B0004FF4C870ADF8B200CA
:1061E0002BA87ADF044600BF2746002F1AD088A0CC
:1061F0008A498B4A891AC9080322CDE9000742EA75
:10620000014040F23B1387A28EA1FAF78DFBFAF70B
:1062100045F900BF00BF26B100BF3046F4F77AFA57
:1062200000BF00BF00BF8F498F48F9F735FB044618
:1062300000BF2746002F1AD075A07849784A891ADE
:10624000C9080322CDE9000742EA014040F24513A4
:1062500074A27CA1FAF768FBFAF720F900BF00BF2F
:1062600026B100BF3046F4F755FA00BF00BF00BFAB
:10627000F7217D48F9F701FB044600BF2746D7B157
:1062800063A06649664A891AC9080322CDE9000756
:1062900042EA01404FF4A47362A26AA1FAF744FBF8
:1062A000FAF7FCF800BF00BF26B100BF3046F4F794
:1062B00031FA00BF00BF00BF00202C906B482C902B
:1062C0002CA8F5F751FB064600BF3746D7B150A0C2
:1062D0005249534A891AC9080322CDE9000742EA04
:1062E000014040F253134FA256A1FAF71DFBFAF7F3
:1062F000D5F800BF00BF24B100BF2046F4F70AFA6A
:1063000000BF00BF00BF686808B168688047AC2163
:1063100002A8F1F704F902208DF8080000208DF89A
:106320000A0006208DF80B000121ADF854105049E9
:10633000169101218DF8841040212491002125918E
:106340004C482B9002A94C48F5F761F8064600BF6F
:106350003746D7B12EA03149314A891AC9080322DC
:10636000CDE9000742EA01404FF4B8732DA235A1F0
:10637000FAF7DAFAFAF792F800BF00BF24B100BFCB
:106380002046F4F7C7F900BF00BF00BF01213A481B
:10639000F5F73AF81C2126A8F1F7C1F8002026905D
:1063A0004FF4A03027904FF4F020289003208DF870
:1063B000A4000020ADF8A6008DF8A8002F482B906F
:1063C0002F482C9026A8F5F787F9064600BF3746D8
:1063D000D7B10FA01149124A891AC9080322CDE981
:1063E000000742EA014040F287130EA215A1FAF716
:1063F0009BFAFAF753F800BF00BF24B100BF204654
:10640000F4F788F900BF00BF00BF2DB0F0BD000059
:106410006572725F636F646500000000647D030055
:10642000CC7C03002E2E5C6C69627A6E6F7264699C
:10643000635C7372635C7A626C655F6D6F64756CCC
:10644000652E630025733A2564205A4552524F52F7
:106450005F434845434B28257329206661696C3AA0
:106460002564000091E7020090950020D5BB020052
:10647000382F0020B52203005C910020F922030090
:106480004FCB02000149086070470000402F0020F8
:106490007CB503211148F5F765F8054600BF2E4687
:1064A000002E19D00EA01149114A891AC9080322D9
:1064B000CDE9000642EA014087230EA215A1FAF7B2
:1064C00033FAF9F7EBFF00BF00BF24B100BF20464D
:1064D000F4F720F900BF00BF00BF7CBD5C91002035
:1064E0006572725F636F646500000000647D030085
:1064F000CC7C03002E2E5C6C69627A6E6F726469CC
:10650000635C7372635C7A626C655F6D6F64756CFB
:10651000652E630025733A2564205A4552524F5226
:106520005F434845434B28257329206661696C3ACF
:10653000256400007FB505460C461148006890F8B8
:10654000230010B9082004B070BD2088F42801DDB4
:106550000720F8E70020009001900290039008487F
:106560000068808AADF800000395029401208DF840
:10657000020003490968098C88B26946AEDFE2E788
:10658000482F002070B50446207800B170BD0D483A
:10659000007800B1FAE72089B0F5807F00D9F5E7EF
:1065A000228909486168F0F7A1FF2189074A064856
:1065B000F4F716FA054615B901200249087000BF24
:1065C000E4E70000C02B0020A44A0020A12E030015
:1065D0007FB505460C461148006890F8220010B9B6
:1065E000082004B070BD2088F42801DD0720F8E7FA
:1065F0000020009001900290039008480068808875
:10660000ADF800000395029401208DF802000349C3
:106610000968098C88B26946AEDFE2E7482F00209E
:1066200013B5044601A92046FFF7D2FF1CBD0000A8
:10663000F0B58DB004460E465D4804604FF0FF3063
:106640005B49096808845B4B0FCB08AD0FC500BFE1
:1066500014B90E200DB0F0BD00BF00BF0EB90E2062
:10666000F8E700BF3068E061214608A862DF054610
:1066700000BF284600B1EDE700BF20788DF832005A
:106680000120ADF83000A21C0CA9A8DF054600BF10
:10669000284600B1DEE700BF20216846F0F73FFF43
:1066A0000220ADF8000020788DF80200F420ADF84B
:1066B00004000120ADF806008DF80C009DF80D00D7
:1066C00020F0080008308DF80D009DF80D0020F036
:1066D0000400001D8DF80D0000208DF81100012030
:1066E0008DF8120000BF608804F10C026946F5F7CE
:1066F000B7FF07460FB13846ACE700BF2021684618
:10670000F0F70DFF0320ADF8000020788DF80200AF
:10671000F420ADF804000120ADF806008DF80C005F
:106720009DF80D0020F0100010308DF80D000120B4
:106730008DF811008DF812008DF8130000BF6088ED
:10674000221D6946F5F78CFF07460FB1384681E7F1
:1067500000BF20216846F0F7E2FE0420ADF80000FB
:1067600020788DF80200F420ADF804000120ADF887
:1067700006008DF80C009DF80D0020F01000103080
:106780008DF80D0001208DF811008DF812008DF8A4
:10679000130000BF608804F114026946F5F760FF3A
:1067A00007460FB1384655E700BF002052E700000A
:1067B000482F00201870030004480068B0F920003A
:1067C000401C08B1012070470020FCE7482F002042
:1067D00070B505460E4606B105B970BD3446288829
:1067E000102804D011281CD050282DD127E018499A
:1067F000184A891AC908032242EA014016A1FAF789
:1068000059F8A88800B220842189A888F8F770FE7A
:1068100084F822002189A888F8F76AFE84F823000A
:1068200013E00B490B4A891AC908032242EA0140C6
:106830000FA1FAF73FF84FF0FF30208405E029461A
:106840002046FCF7D5F900E000BF00BF00BFC4E759
:10685000647D0300CC7C0300424C455F4741505FA0
:106860004556545F434F4E4E454354454400000047
:10687000424C455F4741505F4556545F444953433E
:106880004F4E4E45435445440000000072B6044943
:10689000096801EB4102C2EBC11062B6704700000B
:1068A000302F002000B572B6FFF7F0FF4FF47A7179
:1068B000B0FBF1F362B6184600BD00007CB54FF4A2
:1068C00080410020FAF7A4F8044600BF254625B110
:1068D00000BF2846F3F71EFF00BF00BFF9F7CAFD4F
:1068E000F4F790FF044600BF254625B100BF2846B7
:1068F000F3F710FF00BF00BFF4F718FB044600BF1A
:10690000254625B100BF2846F3F704FF00BF00BFAE
:10691000FAF71EFA044600BF254625B100BF2846F7
:10692000F3F7F8FE00BF00BFFAF7E4FC044600BF2F
:10693000254625B100BF2846F3F7ECFE00BF00BF97
:106940000020019001A90120FAF724FB044600BFB2
:10695000254625B100BF2846F3F7DCFE00BF00BF87
:1069600001A8FAF7E7FB044600BF254625B100BFA2
:106970002846F3F7CFFE00BF00BF0F4903C9CDE99A
:10698000000140F6FF70ADF800000C4A69460C4863
:10699000FBF73EF8044600BF254625B100BF284658
:1069A000F3F7B8FE00BF00BF01210548FBF798F8D8
:1069B0000348FBF71DF87CBD107003007D38030011
:1069C0000870030006E0F4F767F8F9F767FD08B907
:1069D000FAF7DEF9F7E7000038B504460B4800681F
:1069E00000EB4001C1EBC0104FF47A71B0FBF1F045
:1069F00007490968084400906846F0F789FF054692
:106A00002C2229462046F0F771FD38BD302F00209A
:106A1000342F00202DE9F05F04460D4616461F4630
:106A2000DDE90A9A2C211148F0F779FDA4F26C7087
:106A30000E494861681E08610846C6608760C0F854
:106A40000490C0F800A04FF0FF3008620846F0F74D
:106A5000F9FC8346FFF726FFABEB000804488045AE
:106A600002D90448C0F80080BDE8F09F308F0020B4
:106A700080009265342F002038B50446E0B26946A4
:106A8000FBF716F905466DB10849094A891AC90884
:106A9000012242EA01402B46224606A1F9F720FFD7
:106AA000002038BDBDF90000FBE70000647D030055
:106AB000CC7C03006E7266785F73616164635F73A0
:106AC000616D706C655F636F6E76657274282564A6
:106AD00029206661696C206572725F636F64653A34
:106AE000256400002DE9F0430246104601231C46B0
:106AF0000D460026374600BF202802D24FF0A0489E
:106B000003E000F01F00DFF82480C44643EA440895
:106B100048EA850848EA062848EA07490CF5E0688B
:106B200048F8209000BFBDE8F0830000000300504B
:106B3000C82B0020E82B002000900040010400003A
:106B400002000000003002400100000001000000CF
:106B50000600020600000000882D0020010006004B
:106B6000010006000000000002000001000000001B
:106B7000C82D0020F02D00200400000000000000BF
:106B80000000000080FFFFFF070700002E0002004A
:106B9000182E00200000000000000000000000008F
:106BA000B86E03004C730300487303004073030086
:106BB00000020000110B0405E06B00200000000043
:106BC0000338FDD870470000770A0000000000007D
:106BD000770A0000000000007ADA000000000000E0
:106BE00000000050000300506E7266785F677069A5
:106BF0006F74655F696E6974006E7266785F677046
:106C0000696F74655F6F75745F696E6974006E7229
:106C100066785F6770696F74655F696E5F696E69DA
:106C200074000000000000000000000000000000F0
:106C30000338FDD870476E7266785F736161646374
:106C40005F696E6974006E7266785F736161646318
:106C50005F6368616E6E656C5F696E6974006E7209
:106C600066785F73616164635F6368616E6E656CB3
:106C70005F756E696E6974006E7266785F736161CC
:106C800064635F73616D706C655F636F6E76657270
:106C900074006E7266785F73616164635F627566CB
:106CA0006665725F636F6E76657274006E72667889
:106CB0005F73616164635F73616D706C65006E72B8
:106CC00066785F73616164635F63616C696272615E
:106CD00074655F6F66667365740000006E72667837
:106CE0005F7370696D5F696E697400009D93020047
:106CF000C59302007370696D5F78666572006E728D
:106D000066785F7370696D5F786665720000000079
:106D1000FFFFFFFF0006FF00000000400000000032
:106D2000E46E002000000000B02E00202BC90200FD
:106D3000010006000000000000000000000000004C
:106D40000338FDD87047303132333435363738396F
:106D50004142434445460000987D03009C7D03006A
:106D60000000000000000000000000000000000023
:106D7000586D0300706D030004000000556E6B6ECB
:106D80006F776E206572726F7220636F64650000AA
:106D9000000000000C78030001000000B87603003A
:106DA00002000000AC740300030000002C77030015
:106DB00004000000807703000500000060760300F7
:106DC00006000000FC750300070000006877030060
:106DD000080000007476030009000000D876030064
:106DE0000A000000F47703000B0000009474030015
:106DF0000C0000008C7603000D0000005C7803009E
:106E00000E000000587703000F0000009477030085
:106E100010000000C8770300110000007078030024
:106E2000120000004478030013000000E077030024
:106E300080000000147603008100000050750300FC
:106E4000820000001075030083000000F07403004E
:106E5000840000002C7503008500000038760300D4
:106E6000860000004077030090000000DC750300FE
:106E700091000000D074030092000000A07603008F
:106E800000820000A877030001820000F47603006E
:106E90000282000010770300008400006C7503007C
:106EA000018400001878030002840000B475030018
:106EB00003840000907503002DC2020075C3020018
:106EC000E9C20200D5C30200B5C2020025C2020019
:106ED00002000000000000000000000003000000AD
:106EE00000000000000000000001000000000000A1
:106EF0000000000001000000000000000000000091
:106F0000020100000000000000000000020100007B
:106F10000000000000000000000000000030004001
:106F20000000000001000000000000FF06FF00005C
:106F3000000000040000000000000000000000004D
:106F400025030300230303001903030000000000CE
:106F50000338FDD870470000707A0020FF01000060
:106F6000707C002000000000000000000000000015
:106F700000000000646F0300746F0300080000004D
:106F8000FC7D03000C7E03000000000000000000F8
:106F9000806F0300906F030008000000EC7D030089
:106FA000FC7D030000000000000000009C6F030057
:106FB000AC6F030008000000001002019C7D03007C
:106FC000A47D0300A47D0300C47D0300C47D0300F1
:106FD000D47D0300D47D0300DC7D0300BC6F03007F
:106FE000DC6F030008000000B82B0020DC7D0300EC
:106FF000E47D0300E47D0300EC7D0300EC6F0300FF
:10700000FC6F030008000000004002402400040060
:1070100000000641000000009ECADC240EE5A9E045
:1070200093F3A3B50000406E0200000000000000D2
:1070300050EADA308883B89F604F15F30000C98E9C
:10704000004040404040404040404141414141407B
:107050004040404040404040404040404040404030
:1070600040050202020202020202020202020202BF
:1070700002202020202020202020200202020202C4
:10708000020290909090909010101010101010101C
:107090001010101010101010101010100202020228
:1070A000020288888888888808080808080808086C
:1070B0000808080808080808080808080202020268
:1070C00040000000417003001F1C1F1E1F1E1F1FD9
:1070D0001E1F1E1F1F1D1F1E1F1E1F1F1E1F1E1FC8
:1070E0006170705F74696D65725F6372656174650C
:1070F00028266D5F7265636F72645F75706C6F6177
:10710000645F746D722C204150505F54494D45525C
:107110005F4D4F44455F52455045415445442C20F6
:107120005265636F726455706C6F61645F746D72E9
:107130005F636229000000006170705F74696D65B3
:10714000725F63726561746528266D5F7265636F37
:1071500072645F75706C6F61645F66696E69736895
:107160005F7061636B65745F7265706F72745F747A
:107170006D722C204150505F54494D45525F4D4F28
:1071800044455F53494E474C455F53484F542C206C
:107190005265636F726455706C6F61645F66696E8F
:1071A0006973685F7061636B65745F7265706F723D
:1071B000745F746D725F6362290000006170705FBC
:1071C00074696D65725F7374617274286D5F726546
:1071D000636F72645F75706C6F61645F66696E691E
:1071E00073685F7061636B65745F7265706F7274F2
:1071F0005F746D722C204150505F54494D45525F71
:107200005449434B53283330292C2028766F696426
:107210002A296D5F7265706F72745F646174615F5B
:1072200073756D636865636B636F64652900000047
:107230006170705F74696D65725F737461727428D8
:107240006D5F73746174655F6D616368696E655FBE
:107250006472697665725F746D722C204150505F64
:1072600054494D45525F5449434B532831303029DE
:107270002C204E554C4C29006170705F74696D650F
:10728000725F63726561746528266D5F73746174E3
:10729000655F6D616368696E655F6472697665726A
:1072A0005F746D722C204150505F54494D45525FC0
:1072B0004D4F44455F52455045415445442C207341
:1072C000746174655F6D616368696E655F6472693E
:1072D0007665725F746D725F636229006170705FC2
:1072E00074696D65725F63726561746528266D5F90
:1072F000677265656E5F6C696768745F6566666511
:1073000063745F746D722C204150505F54494D4539
:10731000525F4D4F44455F52455045415445442CC2
:1073200020426F6172644C696768745F6566666568
:1073300063745F746D725F68616E646C657229005E
:10734000312E3030000000005344430049464C5970
:10735000544F500052657175657374696E6720747F
:107360006F2075706461746520415454204D5455EC
:1073700020746F202575206279746573206F6E20EC
:10738000636F6E6E656374696F6E20307825782048
:10739000287265747279292E0000000073645F62A0
:1073A0006C655F6761705F646174615F6C656E6777
:1073B00074685F757064617465282920287265712E
:1073C0007565737429206F6E20636F6E6E656374CC
:1073D000696F6E20307825782072657475726E65DD
:1073E000642025732E000000546865207265717555
:1073F000657374656420636F6D62696E6174696F33
:107400006E206F6620545820616E642052582070A0
:1074100061636B6574206C656E6774687320697353
:1074200020746F6F206C6F6E672062792025752045
:107430006D6963726F7365636F6E64732E00000015
:1074400073645F626C655F67617474635F657863C2
:1074500068616E67655F6D74755F72657175657380
:10746000742829206F6E20636F6E6E656374696F78
:107470006E20307825782072657475726E65642090
:10748000627573792C2077696C6C207265747279DF
:107490002E0000004E52465F4552524F525F494EF9
:1074A00056414C49445F4441544100004E52465FAE
:1074B0004552524F525F534F4654444556494345F7
:1074C0005F4E4F545F454E41424C45440000000022
:1074D0004E52465F4552524F525F464541545552B7
:1074E000455F4E4F545F454E41424C4544000000BD
:1074F0004E52465F4552524F525F4D555445585F6C
:10750000554E4C4F434B5F4641494C4544000000AB
:107510004E52465F4552524F525F4D555445585F4B
:107520004C4F434B5F4641494C4544004E52465FE9
:107530004552524F525F4D555445585F434F4E444C
:107540005F494E49545F4641494C454400000000A4
:107550004E52465F4552524F525F4D555445585F0B
:10756000494E49545F4641494C4544004E52465F9E
:107570004552524F525F424C455F495053505F5203
:10758000585F504B545F5452554E4341544544004C
:107590004E52465F4552524F525F424C455F4950F2
:1075A00053505F504545525F52454A454354454408
:1075B000000000004E52465F4552524F525F424C0F
:1075C000455F495053505F4C494E4B5F44495343CC
:1075D0004F4E4E4543544544000000004E52465F16
:1075E0004552524F525F4150495F4E4F545F494D93
:1075F000504C454D454E5445440000004E52465FA8
:107600004552524F525F4E4F545F535550504F5258
:10761000544544004E52465F4552524F525F4D4FC3
:1076200044554C455F4E4F545F494E495449414C77
:10763000495A4544000000004E52465F4552524FA1
:10764000525F4D4F44554C455F414C524541445962
:107650005F494E495449414C495A45440000000095
:107660004E52465F4552524F525F4E4F545F464F07
:10767000554E44004E52465F4552524F525F494E5E
:1076800056414C49445F5354415445004E52465F65
:107690004552524F525F444154415F53495A45004D
:1076A0004E52465F4552524F525F494F5F50454ED2
:1076B00044494E47000000004E52465F4552524F2B
:1076C000525F5356435F48414E444C45525F4D49CB
:1076D0005353494E470000004E52465F4552524FA9
:1076E000525F494E56414C49445F4C454E475448C1
:1076F000000000004E52465F4552524F525F4452C6
:10770000565F5457495F4552525F414E41434B00CB
:107710004E52465F4552524F525F4452565F545745
:10772000495F4552525F444E41434B004E52465FC3
:107730004552524F525F494E5445524E414C000003
:107740004E52465F4552524F525F53544F5241473B
:10775000455F46554C4C00004E52465F4552524FD5
:10776000525F4E554C4C00004E52465F4552524FB0
:10777000525F494E56414C49445F504152414D0081
:107780004E52465F4552524F525F4E4F5F4D454DF0
:10779000000000004E52465F4552524F525F464F26
:1077A0005242494444454E004E52465F4552524F64
:1077B000525F4452565F5457495F4552525F4F568D
:1077C000455252554E0000004E52465F4552524FB0
:1077D000525F494E56414C49445F41444452000077
:1077E0004E52465F4552524F525F5245534F55528B
:1077F000434553004E52465F4552524F525F494EE9
:1078000056414C49445F464C414753004E52465FF7
:1078100053554343455353004E52465F4552524FD2
:10782000525F424C455F495053505F4348414E4E72
:10783000454C5F414C52454144595F45584953546A
:10784000530000004E52465F4552524F525F434F25
:107850004E4E5F434F554E54000000004E52465F5F
:107860004552524F525F54494D454F555400000008
:107870004E52465F4552524F525F42555359000097
:107880007761726E696E67006465627567000000FB
:107890001B5B313B33306D001B5B306D0000000023
:1078A0001B5B313B33316D001B5B313B33326D0071
:1078B0001B5B313B33336D001B5B313B33346D005D
:1078C0001B5B313B33356D001B5B313B33366D0049
:1078D0001B5B313B33376D00696E666F0000000043
:1078E0006572726F7200000073645F626C655F6343
:1078F00066675F73657428292072657475726E659A
:1079000064202573207768656E20617474656D70DE
:1079100074696E6720746F2073657420424C455FF4
:1079200047415454535F4346475F5345525649437A
:10793000455F4348414E4745442E000073645F62F3
:107940006C655F6366675F73657428292072657470
:1079500075726E6564202573207768656E2061748A
:1079600074656D7074696E6720746F207365742020
:10797000424C455F434F4D4D4F4E5F4346475F5628
:10798000535F555549442E0073645F626C655F63B5
:1079900066675F73657428292072657475726E65F9
:1079A00064202573207768656E20617474656D703E
:1079B00074696E6720746F2073657420424C455F54
:1079C00047415454535F4346475F415454525F54B8
:1079D00041425F53495A452E0000000073645F62C4
:1079E0006C655F6366675F736574282920726574D0
:1079F00075726E6564202573207768656E206174EA
:107A000074656D7074696E6720746F20736574207F
:107A1000424C455F434F4E4E5F4346475F474150A0
:107A20002E00000073645F626C655F6366675F735E
:107A3000657428292072657475726E6564202573DB
:107A4000207768656E20617474656D7074696E6707
:107A500020746F2073657420424C455F4741505F2E
:107A60004346475F524F4C455F434F554E542E009F
:107A700073645F626C655F6366675F736574282912
:107A80002072657475726E65642025732077686551
:107A90006E20617474656D7074696E6720746F20F8
:107AA00073657420424C455F434F4E4E5F434647DB
:107AB0005F474154542E00004661696C6564207430
:107AC0006F20646973636F6E6E65637420636F6E9D
:107AD0006E656374696F6E2E20436F6E6E6563749E
:107AE000696F6E2068616E646C653A20256420457C
:107AF00072726F723A20256400000000546865209D
:107B0000626F6F746C6F6164657220686173207757
:107B1000726974652070726F74656374656420693E
:107B200074732073657474696E6773207061676520
:107B30002E20546869732070726F6869626974736B
:107B40002073657474696E6720746865206164765B
:107B50006572746973696E67206E616D652E20545D
:107B6000686520626F6F746C6F61646572206D75FB
:107B7000737420626520636F6D70696C6564207733
:107B8000697468204E52465F424C5F5345545449D5
:107B90004E47535F504147455F50524F5445435401
:107BA0003D3020746F20616C6C6F77207365747446
:107BB000696E6720746865206164766572746973A4
:107BC000696E67206E616D652E0000006E72665FE3
:107BD000626C655F6761747400000000626C655FD1
:107BE0006E757300636C6F636B000000434C4F4312
:107BF0004B0000004750494F54450000505253007D
:107C000055415254000000005541525445000000B7
:107C100053414144430000005350494D00000000CF
:107C20005457490050574D00574454005254430094
:107C300054494D45520000006170705F6275747464
:107C40006F6E00006170705F74696D657200000096
:107C50007077725F6D676D7400000000736F7274EF
:107C60006C697374000000007274745F6C6F675FFE
:107C70006261636B656E6400617070006E72665F56
:107C8000736468006E72665F7364685F626C65003F
:107C90006E72665F7364685F736F63000C7E0300CF
:107CA000B82B0020AC030000A87E0200307F030048
:107CB000642F0020C4760000B69C0200406F0300D1
:107CC00000000000687C0300D82E0020CC7B03005D
:107CD00000000404DC7B030000000000E47B0300E0
:107CE00000000000EC7B030000000000F47B0300B8
:107CF00000000000FC7B030000000000007C03008B
:107D000000000000087C030000000000107C03005D
:107D100000000000187C030000000000207C03002D
:107D200000000000247C030000000000287C030009
:107D3000000000002C7C030000000000307C0300E9
:107D400000000000387C030000000000447C0300B9
:107D500000000000507C0300000000005C7C030079
:107D600000000000787C0300000004047C7C030019
:107D700000000303847C030000000303907C0300E5
:107D800000000303E02E00206873002090730020A1
:107D9000907300202C00000051AE020061BE020072
:107DA00000000000A9BD02000000000021BE02008A
:107DB0000000000029B502005C910020CDF802000F
:107DC00090950020D1670300A44D00200DBA020059
:107DD000B495002019BF020000000000554F0300B9
:107DE00000000000E5BA020000000000811203005C
:107DF00000000000B513030000000000313B030049
:107E00000000000025C602000000000001185AFF13
:107E10000109362001361601190211031204120558
:107E2000120616070F08FF0910100A070B070C743B
:107E30000D010E020F03100411100A12051339145C
:107E400036150616141705181219121A121B121CD1
:107E5000121D100A21012220232024022512261699
:107E60002708280829122A122B122C122D162E331D
:107E70002F303012311232123312341235123612C0
:107E80003712381239123A123B123C123D123E128E
:107E90003F1440FF5012602A6282DC0C02148211EF
:107EA000198213780D120E120F398208081D07135C
:107EB0003B14241504820A364082012E1AFF015316
:107EC00006FFEA40182901091A38091E5809132427
:107ED000BBC00168C1141201030C2C09C602503149
:107EE00064A06B03024B011510014011024504A967
:107EF000B55AFFAB14E078031A80041AD8041A8824
:107F0000041A98041A90041AA0041AA8041AB004B7
:107F10001AB8041AC0041AC8041AD0040110128036
:107F20001492650112020422FFFF14040090D00392
:040000050002720182
:00000001FF
